:100000000C9402280C9486CE0C945BCE0C9430CECB
:100010000C9405CE0C94DACD0C94AFCD0C9484CD19
:100020000C9459CD0C9433280C9433280C94332819
:100030000C9433280C9427930C9433280C94332875
:100040000C9433280C9495A70C9433280C943328E3
:100050000C9433280C9433280C9434500C9413D003
:100060000C9433280D94DF030D9479040C943328F9
:100070000C9433280C9433280C9433280C94332894
:100080000C9433280C9433280C9433280C94332884
:100090000C9433280C9433280C9433280C94332874
:1000A0000C9433280C9433280C9433280C94332864
:1000B0000C9433280C9433280C9433280C94332854
:1000C0000C9433280C9433280C9433280C94332844
:1000D0000C9433280C9433280C9433280C94332834
:1000E0000C943328C0C9C3C9B2C9B6C9BCC9FAC9BE
:1000F000C7C9CBC9D1C9D5C9D9C9DFC9E3C9E7C9FE
:10010000FAC9EDC9F1C9F5C92FCF34CF39CF43CFE3
:100110004DCFC6CF57CF5FCF67CF71CF7BCF85CFC6
:1001200094CF9ECFC6CFA8CFB2CFBCCF5CF55CF545
:1001300063F563F563F56AF56AF56AF577F571F5C8
:1001400071F571F5DA00DC00E800E200D600DE00AF
:10015000D800DE00D400E400DE00E000084AD73B0F
:100160003BCE016E84BCBFFDC12F3D6C74319ABD86
:1001700056833DDA3D00C77F11BED9E4BB4C3E91AA
:100180006BAAAABE000000803F05A84CCDB2D44E99
:10019000B93836A9020C50B9918688083CA6AAAA9B
:1001A0002ABE000000803F000D9444040D943C04DE
:1001B0000D9440040D9412040D9418040D945104F0
:1001C0000D944E040D9434040D9448040D94130CB6
:1001D0000D9429040D94D7080D9486094E414E497B
:1001E0004E495459494E46CDCCCC3D0AD7233C17F5
:1001F000B7D13877CC2B329595E6241FB14F0A0042
:100200000020410000C84200401C4620BCBE4CCA31
:100210001B0E5AAEC59D74434F4D4D554E4943413B
:1002200054494F4E0044525952554E004552524F78
:10023000525300494E464F004543484F00556E6BA0
:100240006E6F776E20636F6D6D616E643A20220071
:100250004163746976652045787472756465723A95
:1002600020003A2000207A5F6D696E3A20202D32FE
:10027000207A5F6D61783A2020350A0050726F62F3
:1002800065205A204F6666736574000000A0C100A7
:10029000809743000000004F6666736574732061A9
:1002A00070706C696564004572723A20546F6F20FB
:1002B0006661722100546F6F206661722066726FF2
:1002C0006D207265666572656E636520706F696E1C
:1002D000740A00FF01FF426564204C6576656C6915
:1002E0006E6720004661696C656420746F20656EDE
:1002F00061626C6520426564204C6576656C696E50
:10030000670A00426564204C6576656C20436F7215
:1003100072656374696F6E204D61747269783A001A
:1003200043290A0061626C656420286D696E20743F
:10033000656D702000436F6C64206578747275641D
:10034000657320617265200020643A0020693A00DC
:1003500020703A0020643A0020693A0020703A0088
:1003600050726F6265205A204F66667365743A203A
:10037000004D31343520533C696E6465783E206F02
:100380007574206F662072616E67652028302D318C
:10039000290A007A5F70726F62653A20007A5F6D99
:1003A00061783A20007A5F6D696E3A2000795F6D5E
:1003B00061783A2000795F6D696E3A2000785F6D50
:1003C00061783A2000785F6D696E3A20005265705E
:1003D0006F7274696E6720656E6473746F702073DA
:1003E00074617475730A002F2F2000454D455247E4
:1003F000454E43595F504152534552004341534586
:100400005F4C494748545F4252494748544E455310
:100410005300544F47474C455F4C4947485453009D
:10042000534F4654574152455F504F574552004233
:1004300055494C445F50455243454E54004C455637
:10044000454C494E475F44415441005A5F50524F1A
:100450004245004155544F4C4556454C0050524979
:100460004E545F4A4F420050524F4752455353003B
:100470004155544F5245504F52545F54454D5000D2
:10048000564F4C554D455452494300454550524FE7
:100490004D0053455249414C5F584F4E5F584F46AF
:1004A00046004649524D574152455F4E414D453AEF
:1004B0004D61726C696E20204649524D574152453C
:1004C0005F56455253494F4E3A312E312E382E3613
:1004D000322045585452554445525F545950453A7C
:1004E00053696E676C6545787472756465722053E4
:1004F0004F555243455F434F44455F55524C3A6810
:10050000747470733A2F2F636F64652E616C65701D
:10051000686F626A656374732E636F6D2F646966BA
:10052000667573696F6E2F4D41524C494E20505283
:100530004F544F434F4C5F56455253494F4E3A31FB
:100540002E30204D414348494E455F545950453A5D
:100550004C756C7A426F742054415A2036204558AD
:100560005452554445525F434F554E543A312055ED
:100570005549443A38343566303033632D6165620D
:10058000642D346535332D613662392D3764303949
:1005900038346664653630390A004C756C7A426FBF
:1005A000742054415A2036204F66662E002F2F614A
:1005B0006374696F6E3A70617573650A00426564B1
:1005C00020646F6E652E0020573A004265642068F3
:1005D000656174696E672E0042656420636F6F6C9D
:1005E000696E672E00436F6F6C696E6720646F6E73
:1005F000652E0048656174696E6720646F6E652EB4
:100600000020573A0045787472756465722025732E
:10061000006F6B00380233022C02250217026F664E
:10062000660044454255473A0045787472756465E2
:100630007220257300000125301D0C1824311C0B7D
:1006400017232F1B0A1E16040308060202222B1A68
:100650004142033809FF3628294527444350726F29
:100660007465637465642050696E0A0025697300BF
:1006700025696D20256973002569682025696D202D
:1006800025697300256964202569682025696D2026
:10069000256973002569792025696420256968200A
:1006A00025696D20256973005072696E7420746924
:1006B0006D653A20005344207072696E74696E67EC
:1006C000206279746520004E6F742053442070724C
:1006D000696E74696E670A004D31323500456E648B
:1006E0002066696C65206C6973740A0042656769ED
:1006F0006E2066696C65206C6973740A004E6F2009
:100700006D6F76652E00526573756D696E6720702A
:1007100072696E74004C756C7A426F742054415A41
:1007200020362072656164792E00436C69636B200A
:10073000746F20726573756D652E2E2E00205A3AE7
:10074000200020593A200042656420583A20005386
:100750006C6565702E2E2E0047322F473320626164
:100760006420706172616D65746572730A00207433
:100770006F6F206C6F6E6720657874727573696F28
:100780006E2070726576656E7465640A0020636F12
:100790006C6420657874727573696F6E2070726511
:1007A00076656E7465640A00746F20726573756D8A
:1007B00065005761697420666F72207072696E748B
:1007C000005052494E542050415553454400436116
:1007D00072642072656D6F76656400436172642097
:1007E000696E7365727465640000060900FE060197
:1007F0008902FE20FFFE07FE06FE0000000600073D
:100800000106060602008080808000800303030644
:100810000103A0A0A00507070600FF5050F850F8FC
:1008200050500509090600FE2070A8A07028A87085
:10083000200608080600FF40A84810204854080574
:1008400007070600FF609090609890680103030618
:1008500002038080800207070602FF4080808080BC
:1008600080400207070602FF80404040404080056C
:1008700005050600008850F85088050505060000AB
:100880002020F820200204040602FEC0404080051B
:100890000101060002F8020202060200C0C00406BE
:1008A00006060100101020408080040606060100A4
:1008B00060909090906003060606010040C04040A2
:1008C00040E00406060601006090102040F0040697
:1008D00006060100F020601010E005060606000084
:1008E00010305090F810040606060100F080E01069
:1008F00010E00406060601006080E09090600406A7
:1009000006060100F0101020404004060606010013
:100910006090609090600406060601006090907000
:100920001060020505060200C0C000C0C002070733
:100930000602FEC0C000C04040800505050600005C
:100940001860806018050303060001F800F805052B
:1009500005060000C0300830C0040707060100602B
:100960009010604000400506060600007090A8B098
:100970008070050606060000205088F88888050665
:1009800006060000F088F08888F0040606060100DC
:10099000609080809060040606060100E0909090D0
:1009A00090E0040606060100F080E08080F0040676
:1009B00006060100F080E080808004060606010043
:1009C000609080B090600406060601009090F09060
:1009D0009090030606060100E040404040E0050616
:1009E000060600003810101090600406060601008C
:1009F00090A0C0A090900406060601008080808030
:100A000080F005060606000088D8A8A88888040695
:100A10000606010090D0B0909090050606060000F2
:100A2000708888888870040606060100E09090E0CF
:100A300080800407070601FF609090D0B06010042A
:100A40000606060100E09090E0909004060606017C
:100A500000609040209060050606060000F8202007
:100A600020202004060606010090909090906004DB
:100A70000606060100909090F060600506060600EC
:100A8000008888A8A8D88805060606000088502097
:100A90002050880506060600008888502020200483
:100AA0000606060100F010204080F003060606014D
:100AB00000E080808080E00406060601008080401F
:100AC000201010030606060100E020202020E0058B
:100AD00003030600032050880501010600FEF8020A
:100AE0000202060204804004040406010070909093
:100AF000700406060601008080E09090E004040483
:100B00000601007080807004060606010010107057
:100B100090907004040406010060B0C070040606E2
:100B2000060100205040E040400406060601FE6039
:100B300090907010600406060601008080E090909E
:100B4000900306060601004000C04040E00308088C
:100B50000601FE200060202020A0400406060601B9
:100B6000008080A0C0A090030606060100C040409F
:100B70004040E0050404060000D0A8A8880404044E
:100B8000060100E09090900404040601006090903B
:100B9000600406060601FEE09090E08080040606F0
:100BA0000601FE709090701010040404060100A06D
:100BB000D0808004040406010070C030E004060602
:100BC0000601004040E0405020040404060100906B
:100BD0009090700404040601009090606005040485
:100BE00006000088A8A85004040406010090606074
:100BF000900406060601FE90909070906004040434
:100C0000060100F02040F0030707060100204040E5
:100C1000804040200107070602FF8080808080809E
:100C20008003070706010080404020404080040206
:100C30000206010350A0FFFFFFFFFFFFFFFFFFFFC2
:100C4000FFFFFFFFFFFFFFFFFFFFFFFFFFFFFFFFB4
:100C5000FFFFFFFFFFFFFF00000006000701060681
:100C60000602008000808080800406060601FF20C6
:100C700070A0A070200507070600FF304840F04034
:100C800040F8050505060000A8508850A80506068E
:100C90000600008850F820F8200107070602FF80B0
:100CA0008080008080800407070601FF70806090CC
:100CB0006010E0030101060105A006070706000019
:100CC000788494A494847803050506010160A060EB
:100CD00000E00505050600002850A0502804030385
:100CE000060100F01010040101060102F0060707DA
:100CF0000600007884B4A4A48478040101060105E8
:100D0000F00403030601026090600507070600FF78
:100D10002020F8202000F803050506010140A0204E
:100D200040E0030505060101C0204020C002020288
:100D300006020440800405050601FF9090B0D080B3
:100D400005060606000078E8E86828280101010683
:100D50000202800202020602FE408003050506012F
:100D60000140C04040E003050506010140A04000ED
:100D7000E0050505060000A0502850A0050808065B
:100D800000FF40C04050703078100508080600FF92
:100D900040C04050680810380508080600FFC02011
:100DA0004030F03078100407070601002000206072
:100DB000809060050707060000402020507088885A
:100DC00005070706000010202050708888050707D7
:100DD0000600002050205070888805070706000094
:100DE0002850205070888805070706000050002012
:100DF0005070888805070706000020502050708832
:100E00008805060606000078A0F0A0A0B80408082F
:100E10000601FE6090808090602040040707060174
:100E2000004020F080E080F0040707060100204029
:100E3000F080E080F00407070601002050F080E019
:100E400080F00407070601005000F080E080F00306
:100E500007070601008040E0404040E00307070626
:100E600001002040E0404040E00307070601004049
:100E7000A0E0404040E0030707060100A000E0407A
:100E80004040E00506060600007048E84848700447
:100E9000070706010050A090D0B090900407070605
:100EA0000100402060909090600407070601002038
:100EB0004060909090600407070601002050609009
:100EC00090906004070706010050A0609090906029
:100ED000040707060100500060909090600505052A
:100EE00006000088502050880408080601FF107092
:100EF000B0B0D0D0E08004070706010040209090F9
:100F00009090600407070601002040909090906048
:100F10000407070601002050909090906004070796
:100F200006010050009090909060050707060000B1
:100F30001020885020202004060606010080E09042
:100F400090E0800406060601006090A0A090A00436
:100F50000707060100402000709090700407070604
:100F600001002040007090907004070706010020E7
:100F700050007090907004070706010050A00070A8
:100F80009090700406060601005000709090700466
:100F90000707060100205020709090700504040699
:100FA000000070A8B0780406060601FE708080700C
:100FB000204004070706010040200060B0C0700414
:100FC000070706010020400060B0C0700407070654
:100FD000010020500060B0C07004060606010050F9
:100FE0000060B0C070030707060100804000C040E9
:100FF00040E0030707060100204000C04040E00336
:10100000070706010040A000C04040E003060606B6
:101010000100A000C04040E0040707060100306066
:10102000107090906004070706010050A000E09047
:101030009090040707060100402000609090600433
:101040000707060100204000609090600407070633
:1010500001002050006090906004070706010050D6
:10106000A0006090906004060606010050006090A9
:1010700090600505050600002000F8002004040427
:1010800006010070B0D0E004070706010040200010
:101090009090907004070706010020400090909007
:1010A000700407070601002050009090907004061D
:1010B000060601005000909090700409090601FE98
:1010C0002040009090907090600408080601FE8017
:1010D00080E09090E080800408080601FE500090B7
:1010E00090907090601000C90210012C0140012204
:1010F0000170011801B0010E01F00104015002FA63
:1011000000B002F0003003E600D003DC009004D20F
:10111000007005C800A006BE000008B400B009AA0F
:1011200000D00BA000600E960060118C00001582AC
:101130000020197800C01D6E00A0226400B0275A5C
:1011400000902C500000314600E0343C0010383252
:1011500000903A2800603C1E00A03D1400803E0A2A
:1011600000203F00004572723A204D494E54454DD3
:101170005020424544004D494E54454D5020747214
:1011800069676765726564004572723A204D494E21
:1011900054454D50204531004572723A204D494E1C
:1011A00054454D50204530004572723A204D41580B
:1011B00054454D5020424544004D415854454D50F2
:1011C00020747269676765726564004572723A20BF
:1011D0004D415854454D50204531004572723A20DA
:1011E0004D415854454D5020453000202F0020429D
:1011F000403A0020403A007C3C3E5E2B3D3F2F5B56
:101200005D3B2C2A225C004C696E65204E756D6238
:101210006572206973206E6F74204C617374204C6A
:10122000696E65204E756D6265722B312C204C61A4
:101230007374204C696E653A200053544F505045EA
:10124000442E20005072696E7465722073746F7042
:101250007065642064756520746F206572726F72AA
:10126000732E2046697820746865206572726F72EB
:1012700020616E6420757365204D39393920746F93
:1012800020726573746172742E202854656D7065C8
:101290007261747572652069732072657365742E4E
:1012A00020536574206974206166746572207265CC
:1012B0007374617274696E67290A004E6F20436807
:1012C00065636B73756D2077697468206C696E65F2
:1012D000206E756D6265722C204C617374204C69B0
:1012E0006E653A2000636865636B73756D206D6988
:1012F000736D617463682C204C617374204C696E4B
:10130000653A20004D313130004D333100534420D7
:1013100072656164206572726F720A00446F6E6557
:10132000207072696E74696E672066696C650A0068
:1013300020496E76616C69642065787472756465A5
:101340007220000000A0C10000A0C1000000000049
:101350000096430080974300008743486F6D6520E7
:1013600058592066697273740A00486F6D65205879
:1013700059206669727374002F2F616374696F6EF0
:101380003A726573756D650A004D36303020486FCE
:1013900074656E6420746F6F20636F6C6420746F6B
:1013A000206368616E67652066696C616D656E7447
:1013B0000A006265640A002C2073797374656D20DD
:1013C00073746F7070656421204865617465725F25
:1013D00049443A200048656174696E672066616916
:1013E0006C6564204245440048656174696E6720FD
:1013F0006661696C65640048656174696E67206642
:1014000061696C65640048656174696E6720666136
:10141000696C6564204530001000AD0330016A013D
:1014200050022B0170030A019004F500B005E5009D
:10143000D006D800F007CE001009C500300ABE0063
:10144000500BB700700CB100900DAB00B00EA600B1
:10145000D00FA200F0109D001012990030139500DB
:101460005014920070158E0090168B00B0178700F4
:10147000D0188400F0198100101B7E00301C7B0006
:10148000501D7900701E7600901F7300B020700010
:10149000D0216E00F0226B00102469003025660018
:1014A000502663007027610090285E00B0295C0020
:1014B000D02A5900F02B5600102D5400302E510028
:1014C000502F4E0070304B0090314800B032450034
:1014D000D0334200F0343E0010363B003037370046
:1014E0005038330070392E00903A2900B03B230069
:1014F000D03C1B00F03D1100103F0100F03F000008
:101500004D3530320A4D353030004C6F61642073F8
:10151000657474696E67730053746F7265207365C8
:101520007474696E677300526573746F72652066B8
:1015300061696C7361666500416476616E636564C0
:101540002053657474696E6773004D61696E000A9B
:10155000003B20454550524F4D20496E6465783A16
:1015600020005570646174696E67207A6F666673D7
:10157000657420696E20454550524F4D3A20000E4B
:10158000000E000E000E000E000E000E000E007F7A
:10159000C03F801F000E00040004000E001F003F2B
:1015A000807FC00E000E000E000E000E000E000E1A
:1015B000000E0007F8000C0C001002002001006073
:1015C00001804000804003E04001C04000804000B6
:1015D000004000006000002000001000000C0C0023
:1015E00007F80001FE000303000400800800401813
:1015F00000601000207C0020380020100020000037
:101600002000002000006000004000008003030074
:1016100001FE00FFFFFF7F80FFC0FFC0FFC07F8093
:101620007F80FFC0FFC0FFC03F001E000C005A209B
:101630004F6666736574005A204F66667365740062
:10164000466C6F7700466C6F770046616E20737052
:1016500065656420310046616E20737065656420A5
:10166000310042656400426564004E6F7A7A6C65B1
:10167000004E6F7A7A6C6500537065656400537034
:10168000656564004D61696E004D6F766520580098
:101690004D6F76652059004D6F7665205A0045786C
:1016A000747275646572004D6F766520302E316DF1
:1016B0006D004D6F766520316D6D004D6F76652044
:1016C00031306D6D004D6F7665206178697300452E
:1016D00078747275646572004D6F7665205A004D9E
:1016E0006F76652059004D6F7665205800457874F7
:1016F0007275646572004D6F7665205A004D6F7685
:10170000652059004D6F76652058004D6F76656DE8
:10171000656E740053442063617264206F6B0A002D
:101720006F70656E526F6F74206661696C65640AD4
:1017300000766F6C756D652E696E697420666169DF
:101740006C65640A00534420696E6974206661699F
:101750006C0A006175746F25692E67004D32340084
:101760004D32332025730057726974696E67207497
:101770006F2066696C653A20006F70656E20666147
:10178000696C65642C2046696C653A20006F706551
:101790006E206661696C65642C2046696C653A2030
:1017A0000046696C652073656C65637465640A0046
:1017B0002053697A653A200046696C65206F706530
:1017C0006E65643A20006F70656E206661696C65B5
:1017D000642C2046696C653A20002066696C653A85
:1017E0002000646F696E67006672657368004E6FF3
:1017F000772000454E4420535542524F5554494E90
:10180000450A002220706F73002220706172656E9D
:10181000743A2200535542524F5554494E45204385
:10182000414C4C207461726765743A22004B494CFC
:101830004C45442E2000747279696E6720746F20C5
:1018400063616C6C207375622D67636F64652066DD
:10185000696C6573207769746820746F6F206D619F
:101860006E79206C6576656C732E204D4158206C26
:101870006576656C2069733A004572726F723A0042
:1018800025753A2530327500253032753A253032CB
:10189000750025756420253032753A253032750083
:1018A00000060900FE000000000001090008FE001B
:1018B0000005080806000040F0C8888898781005E0
:1018C0000808060000C0F88888888888F80505059B
:1018D0000600012030F830200508080600002070BE
:1018E000F820202020E00509090600FF2070A8A8A4
:1018F000B8888870200509090600FFE080C0B0A8FC
:10190000283028280509090600FFF8A88888888853
:1019100088A8F8050A0A0600FE205050505088A8F2
:10192000A8887003030306000340A04000060900D6
:10193000FE0701920321207FFF07FF07FF00000041
:10194000060000010707060200808080808000807A
:10195000030202060105A0A005070706000050507B
:10196000F850F850500507070600002078A07028AE
:10197000F020050707060000C0C810204098180591
:1019800007070600006090A040A8906802030306C5
:101990000104C040800307070601002040808080CA
:1019A00040200307070601008040202020408005DA
:1019B000050506000120A870A82005050506000100
:1019C0002020F820200203030602FFC0408005010A
:1019D00001060003F8020202060200C0C005050568
:1019E00006000108102040800507070600007088E7
:1019F000888888887003070706010040C04040407F
:101A000040E0050707060000708808708080F80530
:101A10000707060000F81020100808F00507070661
:101A2000000010305090F81010050707060000F86D
:101A300080F008088870050707060000708080F0B5
:101A4000888870050707060000F80810202020206D
:101A500005070706000070888870888870050707EA
:101A600006000070888878080870020505060200E4
:101A7000C0C000C0C00206060602FFC0C000C040D1
:101A80008004070706000010204080402010050356
:101A900003060002F800F804070706010080402052
:101AA00010204080050707060000708808102000FD
:101AB0002005070706000070880868A8A8700507B9
:101AC00007060000708888F88888880507070600E0
:101AD00000F08888F08888F0050707060000708805
:101AE0008080808870050707060000F08888888855
:101AF00088F0050707060000F88080F08080F80570
:101B00000707060000F88080F08080800507070640
:101B10000000708880B88888700507070600008874
:101B20008888F888888801070706020080808080FE
:101B300080808005070706000038101010109060A4
:101B40000507070600008890A0C0A0908805070739
:101B5000060000808080808080F80507070600006E
:101B600088D8A8888888880507070600008888C85C
:101B7000A8988888050707060000708888888888E4
:101B800070050707060000F08888F0808080050750
:101B90000706000070888888A89068050707060077
:101BA00000F08888F0A0908805070706000078807C
:101BB00080700808F0050707060000F820202020A4
:101BC0002020050707060000888888888888700517
:101BD00007070600008888888888502005070706C0
:101BE00000008888888888A85005070706000088B4
:101BF000885020508888050707060000888888508C
:101C0000202020050707060000F80810204080F873
:101C1000030707060100E08080808080E00505055D
:101C20000600018040201008030707060100E0209D
:101C300020202020E0050303060004205088050131
:101C400001060000F80202020602058040050505B3
:101C50000600007008788878050707060000808075
:101C6000B0C88888F005050506000070808088707F
:101C700005070706000008086898888878050505A4
:101C80000600007088F880700507070600003048DD
:101C9000E0404040400506060600FF70888878084E
:101CA000700507070600008080B0C8888888010793
:101CB00007060200800080808080800308080601FB
:101CC000FF200020202020A04004070706000080FD
:101CD0008090A0C0A090030707060100C0404040CC
:101CE0004040E0050505060000D0A8A8A8A8050505
:101CF00005060000B0C88888880505050600007044
:101D0000888888700506060600FFF08888F08080C5
:101D10000506060600FF7888887808080505050688
:101D20000000B0C880808005050506000070807046
:101D300008F00407070600004040E040404030053E
:101D400005050600008888889868050505060000D6
:101D500088888850200505050600008888A8A850B6
:101D60000505050600008850205088050606060077
:101D7000FF888888780870050505060000F810209F
:101D800040F8030707060100204040804040200142
:101D90000707060200808080808080800307070696
:101DA0000100804040204040800502020600026899
:101DB000900000000600005A005900580009200059
:101DC0000000000000000000000000007FFFE000B5
:101DD00000000000000000000000007000E00000B3
:101DE0000000000000000000000061F8600000003A
:101DF00000000000000000000041F820000000008A
:101E0000000000000000000040F020000000000082
:101E10000000000000000040602000000000000002
:101E20000000000000005801A07F800000000000BA
:101E300000004104005C63A0FFC00000000000003F
:101E4000002082005EF7A0FFC0000000000000003C
:101E50002082005EF7A0FFC00000000000000041EB
:101E600004005C63A07F8000000000000000820886
:101E7000005801A07F800000000000000104100055
:101E8000406020FFC000000000000001041000407E
:101E9000F020FFC00000000000000082080041F8B0
:101EA00020FFC00000000000000041040061F86055
:101EB0003F00000000000000000000007000E01E75
:101EC0000000000000000001FFFF807FFFE00C0029
:101ED00000000000000001FFFF8000000000000083
:101EE0000000000000000000007FFFE00000000094
:101EF00000000000000000007000E0000000000092
:101F000000000000000000630C6000000000000002
:101F1000000000000000470E20000000000000004C
:101F200000000000004F0F20000000000000000033
:101F3000000000005F0FA000000000000000000093
:101F40000000005E07A07F8000000000000000414C
:101F50000400406020FFC00000000000000020825C
:101F60000040F020FFC000000000000000208200C0
:101F700040F020FFC00000000000000041040040CD
:101F800060207F80000000000000008208005E07E3
:101F9000A07F80000000000000010410005F0FA07F
:101FA000FFC0000000000000010410004F0F20FFE0
:101FB000C000000000000000820800470E20FFC0A3
:101FC00000000000000000410400630C603F0000BE
:101FD0000000000000000000007000E01E00000093
:101FE0000000000001FFFF807FFFE00C0000000008
:101FF00000000001FFFF800000004F6666004F6E8A
:102000002000456E6473746F702061626F7274009B
:1020100053746570732F6D6D004A65726B00416378
:1020200063656C65726174696F6E0056656C6F6391
:10203000697479005A204F6666736574004164764E
:10204000616E6365642053657474696E67730043E1
:10205000616E6E6F7420656E746572207375626454
:1020600069723A2000022E2E004D61696E00202018
:102070004E6F7A7A6C653A200020004261636B00F3
:102080004D696E696D756D2054656D7020697320A2
:102090003132302E0048656174696E67206661696F
:1020A0006C65640045787472756465206D6F726547
:1020B00000526573756D65207072696E74005245CB
:1020C00053554D45204F5054494F4E533A00202010
:1020D0004E6F7A7A6C653A20006368616E676500BE
:1020E0006F66207468652066696C616D656E74004A
:1020F0005761697420666F72207374617274005046
:1021000052494E54205041555345440020204E6FB3
:102110007A7A6C653A2000200066696C616D656EA4
:102120007420756E6C6F6164005761697420666F0E
:1021300072005052494E542050415553454400209E
:10214000204E6F7A7A6C653A20002000506C6561F1
:10215000736520776169742E2E2E0048656174695D
:102160006E67206E6F7A7A6C65005052494E54202B
:102170005041555345440020204E6F7A7A6C653AA1
:102180002000200068656174206E6F7A7A6C652E7D
:1021900000507265737320627574746F6E20746F73
:1021A000005052494E542050415553454400202080
:1021B0004E6F7A7A6C653A2000746F20636F6E748C
:1021C000696E75652E2E2E00616E642070726573C7
:1021D0007320627574746F6E00496E73657274203B
:1021E00066696C616D656E74005052494E542050A2
:1021F00041555345440020204E6F7A7A6C653A2051
:1022000000200066696C616D656E74206C6F61649E
:10221000005761697420666F72005052494E542015
:102220005041555345440020204E6F7A7A6C653AF0
:102230002000200066696C616D656E74206578749D
:1022400072756465005761697420666F7200505240
:10225000494E5420504155534544004E6F20636110
:102260007365206C696768740A00526573656E64F3
:102270003A20002042002050006F6B004B494C4C2C
:1022800045442E20004B494C4C20636175736564B6
:1022900020627920746F6F206D75636820696E61AC
:1022A00063746976652074696D65202D206375728D
:1022B00072656E7420636F6D6D616E643A200050BC
:1022C0006C65617365207265736574005052494E88
:1022D0005445522048414C544544005072696E7434
:1022E00065722068616C7465642E206B696C6C2863
:1022F000292063616C6C6564210A00656E717565E7
:102300007565696E6720220000004842000048425F
:1023100000004040000000005761726E696E673A2D
:1023200020486F6D696E672042756D702044697634
:1023300069736F72203C20310A000202040000A081
:10234000400000A040000000400000A0430080A129
:1023500043000087431FFFFFFFFFFFFF60000000F7
:102360000001FF400000000000FF800000000000AE
:102370007F83CF00000C303F87FF80000C301F862A
:102380007980000C000F8C30C7838C30E78C30CF05
:10239000C7CC31F38C30DCECEC33B98C30D86C6CBE
:1023A00033198C30D06C0C33198C30D86C0C331939
:1023B0008C30DC6C0E3B198C30CF7C079F198C3035
:1023C000C77C038F1940000000000002600000007D
:1023D0000000061FFFFFFFFFFFF82020506C616E1A
:1023E0006E657242756666657242797465733A20ED
:1023F000002046726565204D656D6F72793A200048
:10240000436F6D70696C65643A204A756C202036A4
:1024100020323031380A00207C20417574686F7298
:102420003A2028416C657068204F626A6563747356
:1024300020496E632E2C204C756C7A426F742047B5
:102440006974205265706F7369746F7279290A001C
:102450004A756C202036203230313831313A3135EE
:102460003A333900204C617374205570646174658F
:10247000643A2000312E312E380A004D61726C69A9
:102480006E0020536F6674776172652052657365C4
:10249000740A00205761746368646F672052657323
:1024A00065740A002042726F776E206F7574205237
:1024B000657365740A002045787465726E616C20DE
:1024C00052657365740A00506F77657255700A0023
:1024D00073746172740A006572726F722077726928
:1024E00074696E6720746F2066696C650A00456EBA
:1024F0006473746F70732025632025632025632027
:1025000025630020503A00205A3A0020593A002012
:10251000583A00656E6473746F7073206869743A1A
:102520002000446F6E6520736176696E672066696E
:102530006C652E0A004D3239000201050800FF06C5
:102540000121023520FFFF07FF06FF090050221678
:1025500056808080800080153353A0A0A00257577A
:102560005050F850F850500257572070A070287003
:102570002013355580A040A02002475740A0A0401E
:10258000A0A0502513538080801226564080808062
:102590008040122656804040404080024555906061
:1025A000F060900255552020F820201133536040F0
:1025B00080044151F011335340E040024656101060
:1025C0002040808012365640A0A0A0A0401236566F
:1025D00040C0404040E00246566090106080F002EB
:1025E0004656F020601090600246562060A0F02011
:1025F00020024656F080E01090600246566080E06F
:10260000909060024656F0102020404002465660EE
:102610009060909060024656609090701060122515
:1026200055C0C000C0C011365660600060408012C6
:102630003656204080804020034353F000F012368D
:102640005680402020408012365640A02040004056
:10265000015858304898A8A89040300246566090DB
:1026600090F09090024656E090E09090E00246563E
:10267000609080809060024656E090909090E002DA
:102680004656F080E08080F0024656F080E0808080
:1026900080024656609080B090600246569090F05E
:1026A000909090123656E040404040E0024656700E
:1026B000202020A04002465690A0C0A0A090024634
:1026C000568080808080F002465690F0F090909086
:1026D00002465690D0F0B0B090024656609090906E
:1026E0009060024656E09090E080800147576090ED
:1026F00090D0B06010024656E09090E09090024674
:1027000056609040209060123656E0404040404075
:10271000024656909090909060024656909090900D
:102720006060024656909090F0F09002465690906D
:1027300060609090025656888850202020024656AD
:10274000F010204080F0123656E080808080E00259
:102750004656808040201010123656E0202020205F
:10276000E016325240A0014151F016225280400240
:102770004454709090700246568080E09090E01231
:102780003454608080600246561010709090700241
:10279000445460B0C060024656205040E0404001C2
:1027A000455560907010600246568080E090909091
:1027B0001236564000C04040E0113757200020201C
:1027C00020A040024656808090E09090123656C07D
:1027D00040404040E0025454D0A8A8A8024454E02D
:1027E00090909002445460909060014555E090E0D4
:1027F00080800145557090701010024454A0D08024
:102800008012345460C020C00246564040E0405020
:102810002002445490909070123454A0A0A0400222
:10282000545488A8A85002445490606090014555C3
:102830009090709060024454F02040F0024757306E
:102840004020C02040302216568080808080800248
:102850004757C02040304020C006425250A0FFFFE2
:10286000FFFFFFFFFFFFFFFFFFFFFFFFFFFFFFFF78
:10287000FFFFFFFFFFFFFFFFFFFFFFFFFFFFFF095E
:1028800000502216568000808080800146562070BD
:10289000A0A070200246562050E04050A00255559E
:1028A00088705070880256568850F820F8202217F9
:1028B00057808080008080800247577080E0907051
:1028C00010E0173151A002565670A8C8C8A870145D
:1028D000355560A06000E003435350A050123353BD
:1028E000E02020143151E002565670E8D8E8D87044
:1028F000173151E015335340A04012355540E040A8
:1029000000E014355540A02040E0143555C020C0EB
:1029100020C01622524080014555909090E08002E0
:10292000565678E8E8682828241151801122524030
:102930008014355540C04040E014355540A040005B
:10294000E0034353A050A0024757808080A060F06E
:10295000200247578080A0D0102070024757804047
:102960008060A0F02012365640004080A040024710
:102970005740206090F0909002475720406090F0C0
:10298000909002475760906090F0909002475750A7
:10299000A06090F0909002475790006090F0909067
:1029A00002475760906090F0909002465670A0A049
:1029B000F0A0B00147576090808090604002475778
:1029C0004020F080E080F00247572040F080E08017
:1029D000F00247576090F080E080F0024757900087
:1029E000F080E080F01237578040E0404040E01235
:1029F00037572040E0404040E012375740A0E040C9
:102A00004040E0123757A000E0404040E0025656F8
:102A10007048E848487002475750A090D0B0909056
:102A200002475740206090909060024757204060D6
:102A3000909090600247576090609090906002473D
:102A40005750A0609090906002475790006090901F
:102A50009060123353A040A002465670B0B0D0D060
:102A6000E0024757402090909090600247572040E6
:102A70009090909060024757609090909090600284
:102A800047579000909090906002575710208850C0
:102A900020202002465680E09090E080024656605A
:102AA00090A0A090A0024757402000709090700224
:102AB0004757204000709090700247572050007098
:102AC00090907002475750A0007090907002465648
:102AD00050007090907002475760906070909070B6
:102AE000025454F068B0781135556080806040021F
:102AF000475740200060B0C0600247572040006048
:102B0000B0C06002475760900060B0C06002465697
:102B1000500060B0C060123757804000C04040E0B5
:102B2000123757204000C04040E012375740A00005
:102B3000C04040E0123656A000C04040E002475777
:102B4000A040A01070906002475750A000E0909005
:102B50009002475740200060909060024757204005
:102B60000060909060024757609000609090600213
:102B7000475750A0006090906002465690006090C9
:102B800090601235554000E0004002445470B0D0CF
:102B9000E002475740200090909070024757204035
:102BA0000090909070024757609000909090700253
:102BB00046569000909090700148582040009090A8
:102BC0007090600147578080E090E0808001475717
:102BD0009000909070906001050700FE0500FB01D9
:102BE000F220FFFE05FE05FE020040021525808052
:102BF000800080053242A0A002556550F850F85080
:102C00000146562070C030E02002556590102040EB
:102C10004802556560806890680512228080022510
:102C2000354080808040022535804040408004331C
:102C300043A040A003334340E040012232408004DF
:102C40003141E002112180025565081020408002C8
:102C500045556090909060022535C040404040024C
:102C60004555E0106080F0024555E0106010E0022C
:102C700045552060A0F020024555F080E010E002AC
:102C800045556080E09060024555F01020404002BC
:102C900045556090609060024555609070106003EB
:102CA0001323800080021424800080800235452098
:102CB00040804020033343E000E00235458040205F
:102CC0004080024555E0106000400255657088B8AC
:102CD000A870024555609090F090024555E090E054
:102CE00090E00235456080808060024555E090901C
:102CF00090E0023545E080E080E0023545E080E08C
:102D000080800245557080B090700245559090F0DB
:102D10009090023545E0404040E0024555301010AB
:102D2000906002455590A0C0A090023545808080FB
:102D300080E002556588D8A8888802455590D0B0B3
:102D400090900245556090909060024555E09090BB
:102D5000E080014656609090906010024555E090EA
:102D600090E09002455570806010E0023545E040EB
:102D7000404040024555909090906002455590909B
:102D8000A0A04002556588A8A8A85002455590907B
:102D90006090900245559090701060023545E0209B
:102DA0004080E0022535C0808080C00255658040AB
:102DB000201008022535C0404040C005324240A0E6
:102DC000024151F0052232804002445470909070CC
:102DD00002455580E09090E00234446080806002BB
:102DE0004555107090907002445460B0C060023538
:102DF000452040E0404000465670909070106002C0
:102E0000455580E0909090021525800080808000DC
:102E10002737400040404040800245558090A0E068
:102E2000900215258080808080025464F0A8A8A8B4
:102E3000024454E0909090024454609090600046A8
:102E400056E09090E0808000465670909070101090
:102E5000023444A0C0808002445470C030E0023587
:102E60004540E04040200244549090907002445409
:102E70009090A040025464A8A85050023444A0404E
:102E800040A0004656909090701060024454F0208C
:102E900040F002354560408040600215258080800A
:102EA0008080023545C0402040C005425250A0FFFE
:102EB000FFFFFFFFFFFFFFFFFFFFFFFFFFFFFFFF22
:102EC000FFFFFFFFFFFFFFFFFFFFFFFFFFFFFFFF12
:102ED000020040FFFFFFFFFFFFFFFFFFFFFFFFFFBD
:102EE000FFFFFFFFFFFFFFFFFFFFFFFFFFFFFFFFF2
:102EF000FFFFFFFFFFFFFFFFFFFFFFFFFFFFFFFFE2
:102F0000FFFFFFFFFFFFFFFFFFFFFFFFFFFFFFFFD1
:102F1000FFFFFFFFFFFFFFFFFFFFFFFFFFFFFFFFC1
:102F2000FFFFFFFFFFFFFFFFFFFFFFFFFFFFFFFFB1
:102F3000FFFF01060D00FE09016602D620FFFE0B11
:102F4000FE0AFE0D006022196980808080808080EA
:102F50000080183363A0A0A00357675050F850F8C2
:102F600050500259692078A0A0702828F0200259FA
:102F70006948A85010204050A89002586840A0A06E
:102F800040A0989068281363808080113B6B20409C
:102F9000408080808080404020113B6B80404020FA
:102FA0002020202040408006556520A870A82004DD
:102FB00055652020F8202011336360408006516160
:102FC000F811336340E040025969080810102040AE
:102FD0004080800259692050888888888850200263
:102FE00059692060A02020202020F80259697088AB
:102FF000880810204080F8025969F80810207008ED
:10300000088870025969101030505090F810100262
:103010005969F88080B0C8080888700259697088BA
:103020008080F088888870025969F8081010202084
:10303000404040025969708888887088888870028A
:10304000596970888888780808887011386840E065
:1030500040000040E04011386840E040000060401F
:1030600080025969081020408040201008045464F0
:10307000F80000F8025969804020100810204080B4
:103080000259697088880810202000200259697050
:10309000888898A8A8B080780259692050888888C4
:1030A000F8888888025969F048484870484848F0CC
:1030B000025969708880808080808870025969F028
:1030C00048484848484848F0025969F8808080F0EC
:1030D000808080F8025969F8808080F0808080804C
:1030E0000259697088808080988888700259698840
:1030F000888888F888888888123969E0404040408C
:10310000404040E0025969381010101010109060D3
:10311000025969888890A0C0A09088880259698067
:1031200080808080808080F80259698888D8A8A82B
:103130008888888802596988C8C8A8A89898888803
:10314000025969708888888888888870025969F06F
:10315000888888F080808080015A6A708888888892
:103160008888A87008025969F0888888F0A090883B
:1031700088025969708880807008088870025969CF
:10318000F820202020202020200259698888888863
:1031900088888888700259698888888850505020AB
:1031A0002002596988888888A8A8A8A85002596967
:1031B000888850502050508888025969888850501B
:1031C0002020202020025969F8081010204040805B
:1031D000F8113B6BE0808080808080808080E002FE
:1031E0005969808040402010100808113B6BE02096
:1031F0002020202020202020E00853632050880138
:103200005161F82A226280400256667008788898D8
:1032100068025969808080F088888888F002566644
:1032200070888080887002596908080878888888C2
:1032300088780256667088F880887002596930482C
:103240004040F040404040005868708888887808C6
:103250008870025969808080B0C888888888123850
:10326000684000C040404040E0004A6A1000301012
:1032700010101090906002596980808090A0C0A0CA
:103280009088123969C040404040404040E00256BA
:1032900066D0A8A8A8A888025666B0C8888888887A
:1032A000025666708888888870005868F088888818
:1032B000F08080800058687888888878080808023C
:1032C0005666B0C88080808002566670886010881C
:1032D000700258684040F0404040483002566688CE
:1032E00088888898680256668888885050200256D8
:1032F000668888A8A8A85002566688502020508862
:103300000058688888889868088870025666F8109F
:10331000204080F8015B6B1820202020C020202056
:103320002018221969808080808080808080015BE5
:103330006BC0202020201820202020C00853634884
:10334000A890FFFFFFFFFFFFFFFFFFFFFFFFFFFF53
:10335000FFFFFFFFFFFFFFFFFFFFFFFFFFFFFFFF7D
:10336000FFFFFF0D0060221969800080808080804F
:1033700080800358682070A8A0A0A8702002596916
:1033800030484040E0404048B00356668870505096
:10339000708802596988885050F820F82020221936
:1033A00069808080800080808080124A6A6090807E
:1033B000609090601090601A3262A0A0035969700A
:1033C00088A8D8C8D8A88870045767700878887803
:1033D00000F80356662850A0A05028045363F8084C
:1033E00008163161E00359697088E8D8D8E8D888B0
:1033F000700A5161F8174464609090600357672029
:1034000020F8202000F807356540A02040E007356F
:103410006540A04020C02A22624080005868888809
:10342000888898E8808002596978E8E8E8E86828A0
:103430002828262161C0202262408007356540C0CF
:103440004040E0045767708888887000F80356662B
:10345000A050282850A0025A6A40C04040E00818F6
:10346000283808025A6A40C04040E0102808103846
:10347000025A6A40A04020A048182838080259691A
:10348000200020204080888870025A6A4020002056
:10349000508888F88888025A6A102000205088884E
:1034A000F88888025A6A30480020508888F888884E
:1034B000025A6A28500020508888F88888025A6A80
:1034C00050500020508888F88888025A6A2050207E
:1034D00020508888F8888802596958A0A0A0B0E0D8
:1034E000A0A0B8005B6B708880808080808870208E
:1034F00040025A6A402000F88080F08080F8025A2A
:103500006A102000F88080F08080F8025A6A304803
:1035100000F88080F08080F8025A6A505000F880ED
:1035200080F08080F8123A6A804000E040404040DD
:1035300040E0123A6A204000E04040404040E01243
:103540004A6A609000E04040404040E0123A6AA081
:10355000A000E04040404040E0025969F04848483F
:10356000E8484848F0025A6A2850008888C8A89855
:103570008888025A6A40200070888888888870028B
:103580005A6A10200070888888888870025A6A30C9
:10359000480070888888888870025A6A28500070AD
:1035A000888888888870025A6A5050007088888895
:1035B0008888700355658850205088015B6B0870BF
:1035C0009898A8A8A8C8C87080025A6A40200088A5
:1035D000888888888870025A6A10200088888888BD
:1035E000888870025A6A304800888888888888707D
:1035F000025A6A50500088888888888870025A6AFF
:103600001020008888502020202002596980F088EE
:103610008888F0808080025969609090A0A090888E
:1036200088B002596940200070087888986802596B
:10363000691020007008788898680259693048003D
:10364000700878889868025969285000700878884E
:103650009868025969505000700878889868025A32
:103660006A3048300070087888986802566670287A
:1036700070A0A85000586870888080887020400230
:1036800059694020007088F88088700259691020BC
:10369000007088F88088700259693048007088F896
:1036A0008088700259695050007088F880887012C4
:1036B0003969804000C040404040E01239692040F4
:1036C00000C040404040E0124969609000C0404066
:1036D0004040E0123969A0A000C040404040E002F4
:1036E0005A6A50206010708888888870025969284A
:1036F0005000B0C8888888880259694020007088C6
:1037000088888870025969102000708888888870BD
:103710000259693048007088888888700259692881
:1037200050007088888888700259695050007088ED
:1037300088888870035767202000F80020200158EF
:1037400068087098A8A8C87080025969402000884D
:103750008888889868025969102000888888889825
:1037600068025969304800888888889868025969D1
:10377000505000888888889868005B6B102000880B
:1037800088889868088870005A6A8080B0C88888DD
:10379000C8B08080005B6B505000888888986808AB
:1037A0008870000000000000000000000000000021
:1037B0000000000000000000000000000000000009
:1037C00000000000000C000000000000000C0000E1
:1037D00000000000001200000000000000230000B4
:1037E000000000000021000000000000004C8000EC
:1037F00000000000005E8000000000000092400019
:103800000000000000A14000000000000121200095
:1038100000000000027F9000000000000200100085
:103820000000000007FFF80000000000040008008E
:10383000000000000800040000000000080006006E
:10384000000000001000020000000000301E010017
:1038500000000000207F81000000000041FFE080A8
:103860000000000043FCF08000000000873B78402F
:10387000000000018EDBFC60000000010FEBCC209B
:10388000000000021FEDB610000000021FDEB6109F
:103890000000000439CD7F080000000436E0FF0876
:1038A000000000087EC0BB84000000187F005D8619
:1038B000000000107FC0ED82000000203CC07301BA
:1038C000000000203B337F01000000701BE77E03F7
:1038D000800000C81DEEDE04C00000880FDEDC049E
:1038E000400001240FDF3C092000012607DBF81906
:1038F0002000027203E7F0139000025101FFE02262
:1039000090000489007F802448000904801E00483C
:1039100024000BFE400000DFF40010004000008097
:1039200002001FFFFFFFFFFFFE000000000000007D
:103930000000000000000000000000000000000087
:1039400000001022103C3C0E1F0010221004221117
:1039500004001022100822110400102210083C114B
:103960000400102210102211040010221020221135
:1039700004001E1C1E3C3C0E040000000000000061
:103980000000000000000000000000000000000037
:103990000000000000000000000000000000000027
:1039A0000000000000000000000000000000000017
:1039B0000000000000000000000000000000000007
:1039C00000000000000000000000000000000000F7
:1039D00000000000000000000000000000000000E7
:1039E00020746F6F206C6F6E6720657874727573CA
:1039F000696F6E2070726576656E7465640A00206A
:103A0000636F6C6420657874727573696F6E207073
:103A1000726576656E7465640A0024F4D43050C310
:103A20008E20C2A24017828B7011127A910D816C88
:103A3000D90AA861E108C7586607615143061E4BC1
:103A40005D05C145A7041A411104093D9803713968
:103A500031034036DB0265339102D4305402802EAC
:103A60001D02632CEE01752AC501B028A0011027A4
:103A700081018F2564012B244B01E0223401AC210C
:103A80001F018D200D01801FFC00841EED00971D7D
:103A9000DF00B81CD200E61BC600201BBC00641A65
:103AA000B200B219A8000A19A0006A189900D1172B
:103AB000910040178B00B516840031167E00B315B7
:103AC00079003A157300C7146F0058146A00EE139A
:103AD00066008813630025135E00C7125B006C123A
:103AE000570015125400C111510070114F002111DF
:103AF0004B00D61049008D104700461044000210BC
:103B00004200C00F4000800F3E00420F3C00060FF5
:103B10003B00CB0E3800930E37005C0E3500270EAD
:103B20003400F30D3200C10D3100900D3000600DF6
:103B30002E00320D2D00050D2C00D90C2B00AE0CE3
:103B40002900850C29005C0C2700350C27000E0C81
:103B50002600E80B2400C40B2400A00B23007D0BDF
:103B600023005A0B2100390B2100180B2000F80A02
:103B70001F00D90A1E00BB0A1E009D0A1D00800AF4
:103B80001D00630A1C00470A1B002C0A1B00110AB7
:103B90001A00F7091A00DD091900C4091900AB0958
:103BA0001900920917007B091800630917004C09D6
:103BB000160036091600200916000A091500F50836
:103BC0001500E0081400CC081400B8081400A4087C
:103BD0001400900813007D0812006B0813005808A9
:103BE00012004608120034081100230811001208C0
:103BF000110001081100F0071000E0071000D007C5
:103C00001000C0071000B0070F00A10710009107B7
:103C10000E0083070F0074070F0065070E0057079B
:103C20000E0049070E003B070D002E070E0020076F
:103C30000D0013070D0006070D00F9060C00ED0638
:103C40000D00E0060C00D4060C00C8060C00BC06F3
:103C50000C00B0060C00A4060B0099060C008D06A3
:103C60000B0082060B0077060B006C060B0061064A
:103C70000A0057060B004C060A0042060A003806E6
:103C80000A002E060A0024060A001A060A00100678
:103C9000090007060A00FD050900F4050900EB0507
:103CA0000900E2050900D9050900D0050900C7058A
:103CB0000900BE050900B5050800AD050800A50509
:103CC00009009C050800940508008C05080084057F
:103CD00008007C050800740508006C0507006505F0
:103CE00008005D050700560508004E05070047055A
:103CF00007004005080038050700310507002A05C0
:103D00000700230507001C050600160507000F0520
:103D100007000805060002050700FB040600F5047D
:103D20000700EE040600E8040600E2040700DB04D6
:103D30000600D5040600CF040600C9040600C3042B
:103D40000600BD040600B7040600B1040500AC047B
:103D50000600A6040600A00405009B0406009504C6
:103D60000500900406008A0405008504050080040F
:103D700006007A04050075040500700405006B0454
:103D8000050066040500610405005C040500570495
:103D90000500520405004D040500480405004304D5
:103DA00005003E0404003A04050035040500300413
:103DB00004002C04050027040400230405001E044D
:103DC00004001A04040016040500110404000D0484
:103DD0000400090405000404040000040400FC03BA
:103DE0000400F8030400F4030400F0030400EC03EF
:103DF0000400E8030400E4030400E0030400DC031F
:103E00000400D8030400D4030400D0030400CC034E
:103E10000400C8030300C503030024F404D9201BD5
:103E2000C40C5C0E9804C4095F0265077101F405B7
:103E3000F900FB04B30048048700C103690058037C
:103E4000550003034500BE023A00840231005302CC
:103E50002A002902250004022000E4011C00C801F8
:103E60001900AF01170098011400840113007101BB
:103E700010006101100051010E0043010D003601D8
:103E80000B002B010B0020010B00150109000C0198
:103E9000090003010800FB000800F3000800EB0024
:103EA0000700E4000600DE000600D8000600D2008D
:103EB0000600CC000500C7000500C2000500BD00DB
:103EC0000400B9000400B5000400B1000400AD0016
:103ED0000400A9000400A5000300A20003009F0045
:103EE00004009B000300980003009500020093006B
:103EF0000300900003008D0002008B000300880087
:103F000002008600020084000300810002007F009E
:103F100002007D0002007B000200790002007700B1
:103F200001007600020074000200720001007100BE
:103F300002006F0002006D0001006C0002006A00C8
:103F400001006900020067000100660001006500D1
:103F500001006400020062000100610001006000D5
:103F600001005F0002005D0001005C0001005B00D9
:103F700001005A00010059000100580001005700DB
:103F800001005600010055000100540001005300DB
:103F900000005300010052000100510001005000D8
:103FA00001004F0001004E0000004E0001004D00D6
:103FB00001004C0001004B0000004B0001004A00D2
:103FC00001004900010048000000480001004700CE
:103FD00001004600000046000100450000004500C9
:103FE00001004400010043000000430001004200C2
:103FF00000004200010041000000410001004000BB
:1040000001003F0000003F0001003E0000003E00B4
:1040100001003D0000003D0001003C0000003C00AC
:1040200000003C0001003B0000003B0001003A00A2
:1040300000003A000100390000003900010038009A
:104040000000380000003800010037000000370091
:104050000100360000003600000036000100350087
:10406000000035000000350001003400000034007D
:104070000000340001003300000033000000330072
:104080000100320000003200000032000100310067
:10409000000031000000310001003000000030005D
:1040A0000000300001002F0000002F0000002F0052
:1040B00000002F0001002E0000002E0000002E0046
:1040C00001002D0000002D0000002D0000002D003B
:1040D00001002C0000002C0000002C0000002C002F
:1040E00001002B0000002B0000002B0000002B0023
:1040F00001002A0000002A0000002A0000002A0017
:10410000010029000000290000002900000029000A
:1041100000002900010028000000280000002800FD
:1041200000002800000028000100270000002700F0
:1041300000002700000027000000270001002600E3
:1041400000002600000026000000260000002600D7
:1041500001002500000025000000250000002500CA
:1041600000002500000025000100240000002400BC
:1041700000002400000024000000240001002300AF
:1041800000002300000023000000230000002300A3
:104190000000230000002300010022000000220094
:1041A0000000220000002200000022000000220087
:1041B000010021000000210000002100000021007A
:1041C000000021000000210000002100010020006B
:1041D000000020000000200000002000000020005F
:1041E00000002000000020000000200001001F004F
:1041F00000001F0000001F0000001F0000001F0043
:1042000000001F0000001F0001001E0000001E0033
:1042100000001E0000001E0000004D383420582011
:1042200059205A20450043616E6E6F74206F70658F
:104230006E2073756264697220006563686F3A006E
:10424000544845524D414C2052554E4157415920FA
:1042500042454400546865726D616C2052756E6110
:1042600077617900544845524D414C2052554E419A
:1042700057415920453100544845524D414C205238
:10428000554E41574159204530000000220025007D
:1042900028002B002E00310034000201000005012F
:1042A00008010B0100002100240027002A002D0036
:1042B0003000330001010000040107010A01050577
:1042C0000505070508080808020202020A0A08088C
:1042D00004040404010101010101010103030303BA
:1042E00003030303040707070C0C0C0C0C0C0C0C49
:1042F0000202020206060606060606060B0B0B0B5A
:104300000B0B0B0B0102102020080810204010207E
:104310004080020102010804020101020408102089
:104320004080804020100804020180040201804087
:1043300020100804020108040201010204081020F0
:1043400040800102040810204080436F6F6C646F4E
:10435000776E0046616E207370656564203100469B
:10436000616E2073706565642031004265640042AF
:104370006564004E6F7A7A6C65004E6F7A7A6C6570
:10438000004D61696E005654726176206D696E0051
:104390005654726176206D696E00565472617620B3
:1043A0006D696E00566D696E00566D696E00566DD2
:1043B000696E00566D6178204500566D6178204524
:1043C00000566D6178204500566D6178205A005680
:1043D0006D6178205A00566D6178205A00566D61E3
:1043E00078205900566D6178205900566D6178200B
:1043F0005900566D6178205800566D61782058003C
:10440000566D61782058004D6F74696F6E00416D74
:104410006178204500416D6178204500416D6178EB
:10442000205A00416D6178205A00416D6178205911
:1044300000416D6178205900416D6178205800413C
:104440006D6178205800412D74726176656C004171
:104450002D74726176656C00412D726574726163B2
:104460007400412D72657472616374004163636509
:104470006C00416363656C004D6F74696F6E00562C
:10448000652D6A65726B0056652D6A65726B005604
:10449000652D6A65726B00567A2D6A65726B0056DF
:1044A0007A2D6A65726B0056792D6A65726B0056BB
:1044B000792D6A65726B0056792D6A65726B0056AC
:1044C000782D6A65726B0056782D6A65726B00569E
:1044D000782D6A65726B004D6F74696F6E0045735D
:1044E000746570732F6D6D004573746570732F6DF7
:1044F0006D005A73746570732F6D6D005A73746517
:1045000070732F6D6D005973746570732F6D6D002E
:104510005973746570732F6D6D0058737465707383
:104520002F6D6D005873746570732F6D6D004D6F36
:1045300074696F6E00205A3A0020593A0020436F88
:10454000756E7420583A0020453A00205A3A0020EF
:10455000593A00583A003A004361703A0053657482
:1045600074696E672054726176656C20416363657F
:104570006C65726174696F6E3A200053657474697A
:104580006E67205265747261637420416363656C69
:1045900065726174696F6E3A200053657474696E58
:1045A00067205072696E7420416363656C65726147
:1045B00074696F6E3A200053657474696E67205099
:1045C00072696E7420616E642054726176656C202D
:1045D000416363656C65726174696F6E3A20002097
:1045E0005A00205900580020204D61783A200020C0
:1045F0005A00205900580020204D696E3A20004F83
:104600006E20004F666600536F667420656E64739B
:10461000746F70733A20004B6420002364656669F0
:104620006E65202044454641554C545F004B69203F
:104630000023646566696E65202044454641554CFB
:10464000545F004B70200023646566696E6520200E
:1046500044454641554C545F0050494420417574CF
:104660006F74756E652066696E6973686564212074
:1046700050757420746865206C617374204B702CC5
:10468000204B6920616E64204B6420636F6E7374ED
:10469000616E74732066726F6D2062656C6F772037
:1046A000696E746F20436F6E6669677572617469B5
:1046B0006F6E2E680A00504944204175746F7475FE
:1046C0006E65206661696C6564212074696D656F33
:1046D00075740A00544845524D414C2052554E4184
:1046E00057415900546865726D616C2052756E6156
:1046F0007761790048656174696E67206661696CED
:1047000065640048656174696E67206661696C65FF
:104710006400504944204175746F74756E6520665D
:1047200061696C6564212054656D70657261747592
:10473000726520746F6F20686967680A00204B6497
:104740003A2000204B693A2000204B703A20000AA2
:1047500020436C617373696320504944200A002030
:1047600054753A2000204B753A2000206D61783A4C
:104770002000206D696E3A200020643A20002062FB
:104780006961733A20000000200023002600290000
:104790002C002F0032000001000003010601090176
:1047A00020706F736974696F6E206F7574206F6607
:1047B0002072616E67652E0A003F50726F6265203D
:1047C000000A0A426564204C6576656C20436F726E
:1047D00072656374696F6E204D61747269783A0016
:1047E000202B000A436F7272656374656420426512
:1047F00064204865696768742076732E204265647A
:1048000020546F706F6C6F67793A0A00202B000A92
:104810004265642048656967687420546F706F67EB
:1048200072617068793A0A2020202B2D2D2D2042AC
:1048300041434B202D2D2B0A2020207C202020209E
:10484000202020202020207C0A204C207C2020209A
:1048500020282B29202020207C20520A2045207C43
:1048600020202020202020202020207C20490A20D9
:1048700046207C20282D29204E20282B29207C20F2
:10488000470A2054207C2020202020202020202087
:10489000207C20480A2020207C20202020282D2930
:1048A000202020207C20540A2020207C2020202032
:1048B000202020202020207C0A2020204F2D2D2069
:1048C00046524F4E54202D2D2B0A2028302C3029B3
:1048D0000A004D65616E206F662073616D706C65B6
:1048E0006420706F696E74733A200020643A20006F
:1048F00020623A200045716E20636F6566666963C9
:1049000069656E74733A20613A20003474682070CF
:10491000726F626520706F696E742C2064697374A5
:10492000616E63652066726F6D20706C616E653AB2
:104930002000202844525952554E29004732392030
:104940004175746F20426564204C6576656C696EB4
:10495000670028422961636B00284629726F6E74D4
:10496000002852296967687400284C29656674001C
:104970003F4E756D626572206F662070726F626562
:1049800020706F696E747320697320696D706C613B
:10499000757369626C65202832206D696E696D756A
:1049A0006D292E0A003F2856296572626F736520B3
:1049B0006C6576656C20697320696D706C617573C8
:1049C00069626C652028302D34292E0A0045313A61
:1049D000200045303A20005A3A2000593A20005829
:1049E0003A20004D53312C4D53322050696E730ADA
:1049F000004572726F722077726974696E672074F5
:104A00006F20454550524F4D210A00290A0020626F
:104A1000797465733B206372632000536574746915
:104A20006E67732053746F726564202800202863BA
:104A3000616C63756C6174656429210A0020213DF5
:104A40002000454550524F4D20435243206D69731D
:104A50006D61746368202D202873746F72656429FA
:104A60002000290A002062797465733B2063726319
:104A700020002073746F7265642073657474696EAE
:104A800067732072657472696576656420280020FA
:104A90004D61726C696E3D563437290A00284545D0
:104AA00050524F4D3D00454550524F4D2076657256
:104AB00073696F6E206D69736D6174636820005255
:104AC00065776970696E670050726F62696E672002
:104AD0006661696C65640050726F62696E6720661A
:104AE00061696C65640050524F4245204641494C13
:104AF00020434C45414E204E4F5A5A4C450A0052D5
:104B000065776970696E670A005265776970696ECA
:104B1000670050726F62696E67206661696C6564D8
:104B20000050726F62696E67206661696C6564002F
:104B300050524F4245204641494C20434C45414E3E
:104B4000204E4F5A5A4C450A005265776970696E7B
:104B5000670A0050726F62696E67206661696C65F2
:104B6000640A0050726F62696E67206661696C65E5
:104B70006400205A3A200020593A200042656420FF
:104B8000583A200000000A0B02090C0D0E0807031A
:104B90000401000000000000000000000000000010
:104BA0000000000000000000000000000000000005
:104BB00012111000000000000000000000000000C2
:104BC00000000000000000000000486F6D65202517
:104BD0007325732573206669727374002066697289
:104BE00073740A005A0059005800486F6D65200020
:104BF00048617264636F6465642044656661756CC6
:104C0000742053657474696E6773204C6F616465BA
:104C1000640A00282300002823000064000000101C
:104C2000270000000096430000964300004040002B
:104C300000C8410000C9420000C9420000C8440049
:104C4000804F4420204D383531205A005A2D507263
:104C50006F6265204F666673657420286D6D293A12
:104C60000A0020440020490020204D3330342050D9
:104C70000020440020490020204D333031205000D6
:104C80005049442073657474696E67733A0A002052
:104C9000460020420020480020204D31343520536A
:104CA000004D6174657269616C206865617475702E
:104CB00020706172616D65746572733A0A0020201C
:104CC0004D3432302053004175746F2042656420AA
:104CD0004C6576656C696E673A0A00205A00205967
:104CE0000020204D323036205800486F6D65206F0F
:104CF00066667365743A0A00204500205A00205900
:104D00000020580020420020540020204D32303531
:104D1000205300416476616E6365643A20533C6DB4
:104D2000696E5F66656564726174653E20543C6DB2
:104D3000696E5F74726176656C5F666565647261E9
:104D400074653E20423C6D696E5F7365676D656E8C
:104D5000745F74696D655F75733E20583C6D617852
:104D60005F78795F6A65726B3E205A3C6D61785F4F
:104D70007A5F6A65726B3E20453C6D61785F655F66
:104D80006A65726B3E0A0020540020520020204DBC
:104D9000323034205000416363656C657261746920
:104DA0006F6E2028756E6974732F7332293A205004
:104DB0003C7072696E745F616363656C3E20523C47
:104DC000726574726163745F616363656C3E2054E5
:104DD0003C74726176656C5F616363656C3E0A006A
:104DE000204500205A0020590020204D323031202B
:104DF00058004D6178696D756D20416363656C6520
:104E0000726174696F6E2028756E6974732F7332C6
:104E1000293A0A00204500205A0020590020204D40
:104E20003230332058004D6178696D756D206665AC
:104E3000656472617465732028756E6974732F736D
:104E4000293A0A00204500205A0020590020204D10
:104E50003932205800537465707320706572207564
:104E60006E69743A0A0020204D3230302044300AF6
:104E70000020204D323030204400204469736162AC
:104E80006C65640A0046696C616D656E74207365BB
:104E90007474696E67733A0020204D3134392043B1
:104EA000203B20556E69747320696E2043656C73D6
:104EB0006975730A002020473231202020203B20D2
:104EC000556E69747320696E206D6D0A004B494CF4
:104ED0004C45442E20004D36303020423000507278
:104EE000696E7420706175736564004D31323500F0
:104EF000004D3234005072696E742061626F7274BA
:104F00006564004E6F2053442063617264005072E8
:104F1000696E742066726F6D2053440053746F7015
:104F2000207072696E7400526573756D65207072C1
:104F3000696E740041626F7574204669726D7761A5
:104F40007265005061757365207072696E740043FC
:104F500068616E67652066696C616D656E7400439B
:104F60006F6E66696775726174696F6E0054656D06
:104F70007065726174757265004D6F76656D656EF2
:104F8000740054756E6500496E666F2073637265B8
:104F9000656E004D6F7665206178697300446973B2
:104FA00061626C65207374657070657273004D3852
:104FB00034004175746F20686F6D650047323800AA
:104FC0004D61696E0046696C652064656C65746549
:104FD000643A0044656C6574696F6E206661696C43
:104FE00065642C2046696C653A20006F70656E2000
:104FF0006661696C65642C2046696C653A20000026
:10500000C6AF248311241FBECFEFD1E2DEBFCDBFD8
:1050100000E00CBF14E0A0E0B2E0EAEBFDE302E048
:105020000BBF02C007900D92A430B107D9F725E15C
:10503000A4E0B4E001C01D92A839B207E1F718E27C
:10504000C1E0D8E200E006C021970109802FFE01EF
:105050000F944E1EC030D10780E00807A9F70E94C8
:1050600095880D94CC1E0C9400002F923F924F9285
:105070005F926F927F928F929F92AF92BF92CF92E8
:10508000DF92EF92FF920F931F93CF93DF93CDB7F1
:10509000DEB7CC54D1090FB6F894DEBF0FBECDBF3A
:1050A0008091B8048D3409F461C3843511F40C94F3
:1050B000E83A873411F00C942A3B8091B604909121
:1050C000B7048A31910509F429C2B4F484309105FA
:1050D0003CF482309105A4F597FF2BC00C94443B1F
:1050E0008430910509F4D3C10C9711F00C94443B22
:1050F0000E943A530C94443B8E31910509F45BC2F3
:105100003CF48C31910509F440C20CF40EC242C249
:105110008B35910509F4BDC28C35910509F4BEC2E9
:105120008A35910511F00C94443B1092B4040C9410
:10513000443B80910B0281110C94473B0C94443BFF
:1051400020910B02222311F40C94443B11E00297AE
:1051500009F010E00E948C5319821A821B821C8273
:105160001D821E821F82188682E50E94FF448823CA
:1051700009F43EC10E9499446B017C018091AA14FC
:105180009091AB14A091AC14B091AD1488AB99ABD5
:10519000AAABBBAB8090AE149090AF14A090B014AB
:1051A000B090B11420916C1430916D1440916E1434
:1051B00050916F142CAB3DAB4EAB5FAB8091701434
:1051C00090917114A0917214B091731488AF99AF3B
:1051D000AAAFBBAF20E030E0A901C701B6010F9430
:1051E0002617882309F41AC128A939A94AA95BA955
:1051F0006CA97DA98EA99FA90F94261781110BC0B8
:10520000A501940168AD79AD8AAD9BAD0F942617C9
:10521000882309F403C120E030E0A901C701B601E9
:105220000F942617881F8827881F18130BC020E0AB
:1052300030E040E85FE32C962CAF3DAF4EAF5FAF60
:105240002C970AC080E090E0A0E8BFEB2C968CAFD2
:105250009DAFAEAFBFAF2C9728A939A94AA95BA9CA
:105260006CA97DA98EA99FA90F945E1B24966CAF93
:105270007DAF8EAF9FAF2497A501940168AD79AD46
:105280008AAD9BAD0F945E1B28966CAF7DAF8EAF41
:105290009FAF289724962CAD3DAD4EAD5FAD2497C2
:1052A000CA01B9010F948B172B013C0128962CAD34
:1052B0003DAD4EAD5FAD2897CA01B9010F948B1774
:1052C0009B01AC01C301B2010F945F1B0F94CA1D77
:1052D0006CAF7DAF8EAF9FAF20E030E040E05FE38A
:1052E0000F948B172B013C01A7019601C701B60152
:1052F0000F948B176B017C01A3019201C301B201D2
:105300000F948B179B01AC01C701B6010F945E1B74
:105310000F94CA1D9B01AC012C966CAD7DAD8EAD7A
:105320009FAD2C970F948B176B017C012CA93DA985
:105330004EA95FA968A979A98AA99BA90F945F1BA7
:1053400020E030E040E05FE30F948B172B013C013D
:1053500028966CAD7DAD8EAD9FAD289790582CAD45
:105360003DAD4EAD5FAD0F943B1C9B01AC01C70141
:10537000B6010F948B179B01AC01C301B2010F94CE
:105380005F1B28A939A94AA95BA90F945E1B6983F1
:105390007A838B839C8328AD39AD4AAD5BADC50163
:1053A000B4010F945F1B20E030E040E05FE30F9416
:1053B0008B172B013C012CAD3DAD4EAD5FAD24965E
:1053C0006CAD7DAD8EAD9FAD24970F943B1C9B01C2
:1053D000AC01C701B6010F948B179B01AC01C3014F
:1053E000B2010F945F1BA50194010F945E1B12C0C4
:1053F00089E40E94FF44882331F00E949944698324
:105400007A838B839C838AE40E94FF44882331F053
:105410000E9499446D837E838F83988720E030E0DB
:10542000A90169817A818B819C810F942617811152
:105430000BC020E030E0A9016D817E818F819885CD
:105440000F942617882349F0612FCE0101960E9400
:105450006FF90E944A910C94443BE9E7F8E184918A
:105460008F010F5F1F4F882321F00F949602F801E0
:10547000F6CFE8E5F7E084918F010F5F1F4F882397
:1054800011F40C94443B0F949602F801F4CF80E59C
:105490000E94FF44882329F00E9468446B017C012C
:1054A00003C0C12CD12C760183E50E94FF448823E0
:1054B00061F00E94994420E030E04AE754E40F9400
:1054C0008B170F94A81C6B017C010E9425A780916B
:1054D0003E02811105C060E08FE497E00E94F9452B
:1054E0000E944A918091AB049091AC04A091AD04CC
:1054F000B091AE04C80ED91EEA1EFB1E0E9407D052
:10550000DC01CB018C199D09AE09BF09B7FD02C0B2
:105510000C94443B80E00E94BC83F0CF81E08093F8
:105520000B021092B3100C94443B0E94D3F38111F0
:105530000C94443B80E090E0A8ECB2E489839A8329
:10554000AB83BC8380E090E0A6E9B3E48D839E83C7
:10555000AF83B88780E090E0A0EAB1E489879A87BA
:10556000AB87BC8780E50E94FF44882319F00E9426
:10557000784401C060E068A3BE016F5F7F4FCE0139
:1055800080960F94130E0C94443B80E00E94635A63
:105590000C94443B81E08093B50424982C9A08989D
:1055A000109A0E9496D01092B504249A2C98089ACA
:1055B00010980C94443BC090AA14D090AB14E09087
:1055C000AC14F090AD1488E50E94FF44811108C02E
:1055D00020E030E0A901C701B6010F945F1B02C0B3
:1055E0000E94994468A379A38AA39BA3C090AE1498
:1055F000D090AF14E090B014F090B11489E50E94FF
:10560000FF44811108C020E030E0A901C701B601C4
:105610000F945F1B02C00E9499446B017C01698357
:105620007A838B839C8388A099A0AAA0BBA02CE03E
:1056300032E048E951ECC501B4010F94851D87FFA4
:1056400002C00C94443B21E230E040E953E4C50140
:10565000B4010F942617181614F40C94443B29E156
:1056600034E040E151ECC701B6010F94851D87FF7E
:1056700002C00C94443B21E230E840E953E4C70106
:10568000B6010F942617181614F40C94443B0C948E
:10569000F83B81E08093B4040C94443B0E9425A71E
:1056A000A5E1B3E0B9ABA8ABBAEAEB2EB4E1FB2EAF
:1056B0001DE7C12E14E1D12E312C00E010E0E8A945
:1056C000F9A98191F9ABE8AB0E94FF448823C1F1AD
:1056D0000E9499442B013C01133049F0D6012D91D1
:1056E0003D914D915C910F945E1B2B013C01F701A4
:1056F0002081318142815381C301B2010F945E1B2D
:105700004B015C012DEB37E346E855EB0F94851D0B
:1057100087FD0AC02DEB37E346E855E3C501B40128
:105720000F942617181664F4133011F001E002C02C
:1057300033243394D7014D925D926D927C921397EE
:105740001F5FB4E0EB0EF11CE4E0CE0ED11C143070
:1057500009F0B5CF002319F00E94645903C031103D
:105760000E9462590E94CFC70C94443B8091B604BA
:105770009091B7048937910511F40C94AE340CF074
:10578000DBC08C34910509F454C40CF059C0893144
:10579000910509F4DDC21CF58431910509F468C254
:1057A0007CF48131910509F458C22CF4029708F475
:1057B000D0C10C94443B429709F471C60C94443B0D
:1057C0008631910509F49BC20CF495C2873191058D
:1057D00009F49BC2489709F49CC20C94443B8F3156
:1057E000910509F41AC394F48B31910509F4C2C2EE
:1057F0000CF4BCC28C31910509F4F8C24E9711F03B
:105800000C94443B0F943C100C94443B8A32910519
:1058100009F4A9C344F4809711F00C94443B0E940E
:10582000ACC80C94443B8934910509F4F5C38B341E
:10583000910511F00C94443B0E94CCB20C94443B73
:105840008A36910509F44DC5B4F58435910509F4FE
:1058500026C6E4F48135910509F402C64CF48D3472
:10586000910511F00C94443B0E9483B20C94443B8C
:105870008235910509F40FC68335910511F00C941A
:10588000443B81E08093B3040C94443B8C359105F8
:1058900009F457C634F48535910509F437C60C94DC
:1058A000443B8836910509F4C8C38936910509F44B
:1058B000A6C40C94443B8237910509F4CBC6ACF4E2
:1058C0008D36910509F4DCC434F48B36910509F466
:1058D00034C50C94443B8E36910509F4EFC38F36E2
:1058E000910509F4FEC30C94443B8637910509F4F5
:1058F0000AC794F48337910509F4B2C68537910538
:1059000011F00C94443B60E08091A9049091AA04AA
:105910000E9417460C94443B8737910509F432C71F
:105920008837910511F00C94443B81E080934D142D
:1059300080934C140C94443B8F32F1E09F0711F498
:105940000C94A8370CF080C08D3C910511F40C9498
:105950009435ACF58E3B910509F4AEC4ACF48C38AB
:10596000910509F42EC434F48D37910509F4FDC472
:105970000C94443B8139910509F4F5C78B399105A5
:1059800009F457C40C94443B893C910511F40C94E0
:1059900070353CF4883C910511F40C942A350C9434
:1059A000443B8B3C910511F40C9491358C3C910552
:1059B00011F00C94443B0E9400C70C94443B823E7F
:1059C000910511F40C94C13524F5833D910511F432
:1059D0000C94B13584F48E3C910511F00C94443B49
:1059E00065E1C62E63E0D62E7CE2E72E74E0F72E4A
:1059F00010E00C949F358C3D910511F40C94B43556
:105A00008D3D910511F00C94443B0E946EC50C94A1
:105A1000443B8C3231E0930711F40C9410363CF483
:105A20008232914011F40C9403360C94443B8D3235
:105A3000A1E09A0711F40C9439368E32914011F49A
:105A40000C9454370C94443B843FE1E09E0711F4DE
:105A50000C941339D4F5803921E0920711F40C9499
:105A6000AB37ECF48E3541E0940711F40C94E23A34
:105A70003CF48033914011F40C94D7360C94443BA1
:105A80008F35B1E09B0711F40C94E53A83369140D1
:105A900011F00C94443B0E9425880C94443B8239BD
:105AA000F1E09F0711F40C94B23714F40C94AE3764
:105AB000843A31E0930711F40C94B6378C3A914054
:105AC00011F40C9436380C94443B883552E0950719
:105AD00011F40C948D39B4F4863FB1E09B0711F4B6
:105AE0000C94193914F40C941639873FF1E09F0790
:105AF00011F40C941C398C31924011F40C94283917
:105B00000C94443B8C3833E0930711F40C94C83A5E
:105B100094F4833553E0950711F40C9433398B38A2
:105B2000934011F00C94443B85E1E82E83E0F82E7D
:105B300010E00C94A13A803AB3E09B0709F460C1ED
:105B4000873E934011F00C94443B0E9411880C94C2
:105B5000443BA090A904B090AA0480E50E94FF44B1
:105B6000882359F00E9468446B017C0111E0672B87
:105B7000682B692B31F410E004C010E0C12CD12C4B
:105B8000760183E50E94FF448823F1F00E94994446
:105B900020E030E04AE754E40F948B170F94A81CE0
:105BA0006B017C01111112C0672B682B692B71F4FA
:105BB000A114B10459F0D5018C91882339F061E02A
:105BC000C5010E94174607C0112391F360E08AE2E5
:105BD00097E00E94F94581E08093A8040E9425A7E0
:105BE0000E944A91C114D104E104F104F1F08091C2
:105BF000AB049091AC04A091AD04B091AE04C80E7A
:105C0000D91EEA1EFB1E0E9407D0DC01CB018C19B5
:105C10009D09AE09BF09B7FF1CC08091A804882365
:105C2000C1F080E00E94BC83EECF8091A80488235D
:105C300021F080E00E94BC83F8CF80911C1160E0CD
:105C4000823019F485E197E002C086E097E00E9477
:105C5000F9451092A8040C94443B60E08DEF96E067
:105C60000E94F94517981698159814980C94443B7F
:105C7000ECEEF6E084918F010F5F1F4F882321F037
:105C80000F949602F801F6CF1092071440E050E00E
:105C9000BA0183EB91E10F94ED048BE1E3EBF1E1C9
:105CA000DE01159601900D928A95E1F78091B11170
:105CB0009091B2119C838B8382EB93E09A838983CA
:105CC00040E050E0BE016F5F7F4F85EA93E00E94A5
:105CD00027B5CE0101960E944183EDEDF6E0849157
:105CE0008F010F5F1F4F882311F40C94443B0F94D6
:105CF0009602F801F4CF0E94C3710C94443B1092B9
:105D00005B1110925C110C94443B0F948B110C941A
:105D1000443B19821A821B821C8218A219A21AA261
:105D20001BA28091A704882341F040E0BE016F5F71
:105D30007F4FCE0180960E94046380915C1188237E
:105D400019F081E080935B110E94CCB20C94443B2B
:105D500010925B110E946EB288ED96E09093ED0771
:105D60008093EC070E9483560C94443B0F9471116E
:105D70000C94443B80915C11882351F1E5EBF6E0F3
:105D800084918F010F5F1F4F882321F00F9496029B
:105D9000F801F6CF6091FE137091FF13809100140B
:105DA000909101144AE00F94EF028FE20F94960253
:105DB0006091FA137091FB138091FC139091FD1385
:105DC0004AE00F94EF028AE00F9496020C94443B51
:105DD000E7ECF6E084918F010F5F1F4F882311F4E9
:105DE0000C94443B0F949602F801F4CF40E060E03D
:105DF0008091A9049091AA040E947E6E0C94443B69
:105E00008091A9049091AA0421E020935A1140E0C6
:105E100060E00E947E6E0C94443B0E9498B2ACE31A
:105E2000CA2ED12CE12CF12CA70196010F94011B55
:105E3000762E672ECA01B901A70196010F94011BA6
:105E40006B017C01CA01B90128E130E040E050E07B
:105E50000F94011B4B015C01C9016DE671E00F94C9
:105E6000271E8E010F5F1F4F6115710599F06F920C
:105E70007F92DF92CF929F928F929F938F937F9387
:105E80006F9384E996E09F938F931F930F930F94E2
:105E9000BF1612C00097B1F06F927F92DF92CF923F
:105EA0009F928F929F938F9384E896E09F938F9316
:105EB0001F930F930F94BF160FB6F894DEBF0FBE5B
:105EC000CDBF36C081149104A104B10479F06F9262
:105ED0007F92DF92CF929F928F9288E796E09F9376
:105EE0008F931F930F930F94BF16E6CFC114D10465
:105EF000E104F10469F06F927F92DF92CF9280E724
:105F000096E09F938F931F930F930F94BF16D4CF58
:105F10006F927F928CE696E09F938F931F930F93DF
:105F20000F94BF160F900F900F900F900F900F903F
:105F300060E0C8010E941746EAE3F2E484917F0121
:105F40009FEFE91AF90A882321F00F949602F701CE
:105F5000F5CFB80188EA96E00E94C5918AE00F94D7
:105F600096020C94443B83E50E94FF44882311F47D
:105F70000C94443B0E948844E82E80E50E94FF4434
:105F8000811114C081E0E11001C080E08093B5046C
:105F9000882331F024982C9A0898109A0C94443B4A
:105FA000249A2C98089A10980C94443B80E50E94FF
:105FB000FF44882341F00E9478448B0177FF02C0A0
:105FC0000C94443B02C00DE010E0902FE5E3F6E0B6
:105FD00088E28E0F2491921729F031968E13FACF12
:105FE0000C944F3CE9E7F8E184918F010F5F1F4F5C
:105FF000882321F00F949602F801F6CFEDE5F6E044
:1060000084918F010F5F1F4F882311F40C94443B40
:106010000F949602F801F4CF80915B1181110C94DA
:10602000443B80E50E94D04481110C946C3C0C945C
:10603000443B0E946EB20C94443B88E690E00E9480
:10604000255681110C94443B8091AF0483FF02C01C
:106050000C94443B83E50E94FF44882311F40C9484
:10606000443B0E9499440F94A31C70939D04609339
:106070009C0480E00E9445520E94994420919E0415
:1060800030919F044091A0045091A1040F94851D6C
:10609000181614F00C94443B83ED92E09F938F9379
:1060A00089E296E09F938F931F920E9405B30F9011
:1060B0000F900F900F900F900C94443B8EE40E9431
:1060C000FF44882311F40C94443B0E94784460936D
:1060D000DD057093DE058093DF059093E0050C9459
:1060E000443B83E50E94D044882359F083E50E9415
:1060F000FF44882319F00E94884401C080E0809307
:10610000AF04EAE3F2E484918F010F5F1F4F88230D
:1061100021F00F949602F801F6CFE2E2F6E08491C6
:106120008F010F5F1F4F882321F00F949602F80113
:10613000F6CFC090AF04CC2099F1F4E1AF2EF6E099
:10614000BF2EE12CF12C80E0D12C96010E2C02C048
:10615000359527950A94E2F720FF17C09924939468
:10616000980E882319F08CE20F949602F501259180
:106170003491F901849189010F5F1F4F882321F029
:106180000F9496029801F5CF892DFFEFEF1AFF0AC1
:1061900022E0A20EB11C35E0E316F104B1F60CC00A
:1061A000EEE1F6E084918F010F5F1F4F882321F00D
:1061B0000F949602F801F6CF8AE00F9496020C94A1
:1061C000443B8091AF0483FF02C00C94443B83E5C1
:1061D0000E94FF44882311F40C94443B0E9499448C
:1061E0000F94A31C6739710514F066E970E0709391
:1061F0009B0460939A040E94FA510C94443B89E6F4
:1062000090E00E94255681110C94EB3FE1E1F6E00D
:1062100084918F010F5F1F4F882321F00F94960206
:10622000F801F6CF0E94B14F8AE00F9496020C94C9
:10623000EB3F83E50E94FF44882311F40C94443B18
:106240000E948844182F8D3308F01CE310939904A2
:106250000E9407D06B017C01212F30E0A8EEB3E053
:106260000F944F1BC60ED71EE81EF91EC092950450
:10627000D0929604E0929704F09298040C94443BD8
:106280008DE690E00E94255681110C94443B80914C
:10629000AF0483FF02C00C94443B83E50E94FF449B
:1062A00088AB81110C94773C82E50E94FF448111F8
:1062B0000C94773C0C94443B8091AF0483FF02C064
:1062C0000C94443B83E50E94FF4488AF81110C94F9
:1062D000F13D82E50E94FF4481110C94F13D0C9444
:1062E000443B80E50E94FF44882341F00E9488449B
:1062F000182F823010F00C94443B01C010E083E56D
:106300000E94FF44882329F00E947844362F272FCB
:1063100002C03FEF20E0E12FF0E0EE0FFF1FED5550
:10632000FB4F832F922F8F3F910519F010F08FEFC5
:1063300090E0918380830C94443B80E50E94FF446D
:10634000882341F00E9478446230710510F00C946B
:10635000443B02C060E070E0660F771FFB01ED5523
:10636000FB4F118210820C94443B8CE40E94D04479
:10637000882319F00E94994404C060E070E080E036
:1063800090EC6CA37DA38EA39FA380E090E0A8EC8B
:10639000B2E489839A83AB83BC8380E090E0A6E972
:1063A000B3E48D839E83AF83B88780E090E0A0EA5A
:1063B000B1E489879A87AB87BC8788E50E94FF4450
:1063C000882379F088E50E94FF44882319F00E9411
:1063D000994403C060E070E0CB0169837A838B83CA
:1063E0009C8389E50E94FF44882379F089E50E9417
:1063F000FF44882319F00E94994403C060E070E0D4
:10640000CB016D837E838F8398878AE50E94FF444A
:10641000882379F08AE50E94FF44882319F00E94BE
:10642000994403C060E070E0CB0169877A878B876D
:106430009C8718A219A21AA21BA28091A7048111FD
:106440000C94443B00E020E0AE01405E5F4FBE0193
:106450006F5F7F4FCE0184960E940E620C94443B86
:106460000E9490520E9425A70E944B831092A40480
:106470001092A3041092A6041092A50468EE73E093
:1064800080E090E00E9409E660E08AE995E00E94E1
:10649000F9450C94443B1092B3040C94443B83E5BF
:1064A0000E94FF448823A1F00E94994420E030E03C
:1064B0004AE754E40F948B170F94A81C60930202D0
:1064C0007093030280930402909305020C94443B62
:1064D00088E50E94D04481110C94563F89E50E94C2
:1064E000D04481110C94563F8AE50E94D04481111A
:1064F0000C94563F85E40E94D04481110C94563F81
:106500000E9425A70E944B830C94443B83E50E9484
:10651000D044882311F40C94443B0E94994420E019
:1065200030E04AE754E40F948B170F94A81C609353
:10653000890470938A0480938B0490938C040C9448
:10654000443B95E1C92E93E0D92E2AEBE22E24E1BB
:10655000F22E10E0D6018D916D010E94D044882367
:1065600009F46DC0133009F063C00E9499444B01D7
:106570005C0120E030E040EA51E40F94261787FFE9
:106580004EC0A50194016091C6147091C71480910A
:10659000C8149091C9140F943B1C2B013C019B0122
:1065A000AC0160918504709186048091870490917C
:1065B00088040F948B1760938504709386048093EE
:1065C000870490938804A3019201609175047091EF
:1065D000760480917704909178040F948B176093E0
:1065E0007504709376048093770490937804609197
:1065F00065047091660480916704909168040F941B
:106600002A17A30192010F948B170F94A81C609373
:106610006504709366048093670490936804809285
:10662000C6149092C714A092C814B092C91407C09F
:106630000E949944F70160837183828393831F5F73
:10664000F4E0EF0EF11C143009F084CF0E9448AF43
:106650000C94443B0E9425A70E94CFC70C94443B56
:10666000E2EAF4E084918F010F5F1F4F882321F04D
:106670000F949602F801F6CF60E082E994E00E9460
:106680008BC761E08BE894E00E948BC761E080E8F3
:1066900094E00E948BC761E080E794E00E948BC782
:1066A00060E087E694E00E948BC761E08DE594E0AE
:1066B0000E948BC761E083E594E00E948BC761E094
:1066C0008BE494E00E948BC761E08DE394E00E942C
:1066D0008BC761E08FE294E00E948BC760E080E2AC
:1066E00094E00E948BC760E082E194E00E948BC737
:1066F00060E08CEF93E00E948BC761E08BEE93E04B
:106700000E948BC7C1C785E40E94FF44882319F00B
:106710000E94AB5C03C085E40E94D044882361F0F2
:10672000EAE3F2E484918F010F5F1F4F882321F089
:106730000F949602F801F6CF81E40E94FF4488236B
:1067400019F00E94AB5C03C081E40E94D04488230E
:1067500061F0E7EEF3E084918F010F5F1F4F882314
:1067600021F00F949602F801F6CF0091A904109140
:10677000AA04D8018D918D01882309F41DCD0F94B1
:106780009602F7CF81E08093B50424982C9A08985C
:10679000109AEDECF3E084918F010F5F1F4F882377
:1067A00021F00F949602F801F6CFE5ECF3E0849126
:1067B0008F010F5F1F4F882321F00F949602F8017D
:1067C000F6CF1E9903C009EE12E002C00EEE12E0F1
:1067D000F80181918F01882319F00F949602F8CF68
:1067E0008AE00F949602EDEBF3E084918F010F5F46
:1067F0001F4F882321F00F949602F801F6CF0299DB
:1068000003C009EE12E002C00EEE12E0D8018D9135
:106810008D01882319F00F949602F8CF8AE00F9427
:106820009602E5EBF3E084918F010F5F1F4F882301
:1068300021F00F949602F801F6CF1D9903C009EEDE
:1068400012E002C00EEE12E0F80181918F01882360
:1068500019F00F949602F8CF8AE00F949602EDEAB1
:10686000F3E084918F010F5F1F4F882321F00F9475
:106870009602F801F6CF019903C009EE12E002C0BA
:106880000EEE12E0D8018D918D01882319F00F943E
:106890009602F8CF8AE00F949602E5EAF3E084913D
:1068A0008F010F5F1F4F882321F00F949602F8018C
:1068B000F6CF1C9B03C009EE12E002C00EEE12E000
:1068C000F80181918F01882319F00F949602F8CF77
:1068D0008AE00F949602EDE9F3E084918F010F5F57
:1068E0001F4F882321F00F949602F801F6CF3799B5
:1068F00003C009EE12E002C00EEE12E0D8018D9145
:106900008D01882319F00F949602F8CF8AE00F9436
:106910009602E3E9F3E084918F010F5F1F4F882314
:1069200021F00F949602F801F6CF009B03C009EE08
:1069300012E002C00EEE12E0F80181918F0188236F
:1069400019F00F949602F8CF8AE00F9496021092F5
:10695000B504249A2C98089A109896C610924D1453
:1069600010924C1491C683E50E94FF44882319F0CD
:106970000E94784402C060E070E08B011127023071
:106980001105CCF0E9E7F8E184918F010F5F1F4F0B
:10699000882321F00F949602F801F6CFE1E7F3E0A7
:1069A00084918F010F5F1F4F882309F46DC60F94E8
:1069B0009602F801F5CF88E40E94FF448823A9F0ED
:1069C0000E947844683771053CF06332F1E07F073C
:1069D0002CF062E271E002C068E770E0F801EE0FAF
:1069E000FF1FEB5AFB4F7183608386E40E94FF44D4
:1069F0008823A9F00E947844F801EE0FFF1FEF5A98
:106A0000FB4F718360836F3F710519F014F06FEFD6
:106A100070E077FF02C060E070E07183608382E421
:106A20000E94FF44882309F42FC60E9478446530F1
:106A3000710534F0683871052CF067E870E002C029
:106A400065E070E0000F111FF801E35BFB4F7183FD
:106A500060831AC688EC90E00E942556811114C606
:106A600084E40E94D0448823C1F10E94994411E03B
:106A700020E030E0A9010F942617811101C010E039
:106A800010934C04112349F10E949944E09194041D
:106A900024E0E29FF0011124E85BFB4F60837183E7
:106AA0008283938320E030E0A901609148047091D3
:106AB000490480914A0490914B040F942617811148
:106AC0000CC080E090E0A0E4B0E480934804909390
:106AD0004904A0934A04B0934B040E9485A5D4C5F1
:106AE000E8E3EE2EE4E0FE2E05E113E0F4E0DF2E15
:106AF000D00ED8018D918D010E94D044882349F099
:106B00000E9499440F94A81CF701608371838283CB
:106B10009383F4E0EF0EF11CD012EBCF0E94DEAEB7
:106B2000B3C50E9469C7B0C50E9496C6ADC51F5FB8
:106B3000F4E0EF0EF11C133011F40C94B22BD601DB
:106B40008D916D010E94D044882389F30E9499445D
:106B5000F7016083718382839383812F0E94E555BF
:106B6000E6CF0E94B8C590C583E50E94FF44882304
:106B700009F48AC50E94784470939402609393024A
:106B800083C580E50E94D044882309F47DC50E9416
:106B90007844F62E062F172F83E50E94FF448823A2
:106BA00021F00E9478446B0103C0CC24CA94DC2CF1
:106BB000C6010196039708F067C517FD65C50E94D9
:106BC00025A72FEFC216D20631F0CA94CD2871F452
:106BD00001E010E00DC08F2D0E94B1CE31E020E029
:106BE000892B09F030E0032F122F02C000E010E0E3
:106BF0008F2D0E94B1CE8017910709F445C580E022
:106C00000E94BC83F5CF8AE50E94FF4481110C9459
:106C1000753F83E50E94FF4481110C94753F34C594
:106C200083E50E94FF44882319F00E94784402C043
:106C300064E071E079A368A380E50E94FF448823A3
:106C400039F00E947844693843E1740730F402C097
:106C500068EE73E07A83698304C088E893E19A83DD
:106C60008983BE01605E7F4FCE0101960E94497309
:106C70000BC585E40E94FF44811110C080E50E948D
:106C8000D044882391F00E94994460932204709329
:106C90002304809324049093250407C00E94884411
:106CA000882361F3E9E7F8E171C089E40E94D044E8
:106CB000882381F00E9499442CEA35EC47E25EE398
:106CC0000F948B1760931E0470931F04809320040D
:106CD0009093210484E40E94D044882381F00E9490
:106CE00099442CEA35EC47E25EE30F943B1C609339
:106CF0001A0470931B0480931C0490931D04EAE310
:106D0000F2E484918F010F5F1F4F882321F00F94CD
:106D10009602F801F6CF409122045091230460912D
:106D20002404709125048CE593E00E948F912CEA55
:106D300035EC47E25EE360911E0470911F04809180
:106D40002004909121040F943B1CAB01BC0188E509
:106D500093E00E9472912CEA35EC47E25EE3609189
:106D60001A0470911B0480911C0490911D040F94CF
:106D70008B17AB01BC0184E593E00E9472918AE01D
:106D80000F94960281C40F949602F80184918F01AA
:106D90000F5F1F4F8111F7CF04E013E0D8018D91F1
:106DA0008D01882309F408CA0F949602F7CF80E575
:106DB0000E94D044882351F00E94994460931604A5
:106DC00070931704809318049093190489E40E9427
:106DD000D044882381F00E9499442CEA35EC47E2A4
:106DE0005EE30F948B1760931204709313048093E7
:106DF00014049093150484E40E94D044882381F005
:106E00000E9499442CEA35EC47E25EE30F943B1C68
:106E100060930E0470930F048093100490931104F8
:106E2000EAE3F2E484918F010F5F1F4F882321F082
:106E30000F949602F801F6CF409116045091170472
:106E4000609118047091190480E593E00E948F917D
:106E50002CEA35EC47E25EE3609112047091130472
:106E600080911404909115040F943B1CAB01BC015C
:106E70008CE493E00E9472912CEA35EC47E25EE3E9
:106E800060910E0470910F04809110049091110490
:106E90000F948B17AB01BC0188E493E00E947291C0
:106EA0008AE00F949602F0C383E50E94D044182F25
:106EB000882371F00E9499440F94A31C70930102DF
:106EC0006093000221E0672B09F020E020930D047D
:106ED00080E50E94D044882359F02091000230912F
:106EE0000102232B11F00E94AB5C80930D04CCC3F4
:106EF0001111CAC3EAE3F2E484918F010F5F1F4FBF
:106F0000882321F00F949602F801F6CF80910D04AA
:106F1000811103C068EF72E002C06BEE72E085E39E
:106F200093E00E94C591609100027091010284E299
:106F300093E00E94AC91E0E2F3E084918F010F5F57
:106F40001F4F882309F4A0C30F949602F801F5CFD0
:106F50000E94B3BF99C30E9425A796C381E00E94F7
:106F6000425592C380E00E9442558EC38091AA147C
:106F70009091AB14A091AC14B091AD1489839A8315
:106F8000AB83BC838091AE149091AF14A091B014E8
:106F9000B091B1148D839E83AF83B8878091B21472
:106FA0009091B314A091B414B091B51489879A87C5
:106FB000AB87BC8786E50E94D044882321F083E01C
:106FC00093E00E940AF583E50E94D044882331F0C3
:106FD0000E94AB5C182F0E944C5A01C010E0F09048
:106FE0000C04111103C0EAE3F2E41AC0F110FBCF64
:106FF000E9E7F8E184918F010F5F1F4F882321F0AB
:107000000F949602F801F6CFE4EEF2E084918F013E
:107010000F5F1F4F882339F30F949602F801F6CFC4
:1070200084918F010F5F1F4F882321F00F949602E8
:10703000F801F6CFF11003C060E073E002C06CEF1E
:1070400072E086ED92E00E94C5918AE00F9496026C
:107050004CE050E06AEA74E1CE0101960F945E1EA6
:10706000892B09F411C30E94CFC70EC30E94D3F32A
:1070700081110AC32BE8822E22E0922EEAEAF4E183
:10708000F9ABE8AB9E012F5F3F4F590103ED12E0D2
:10709000190133E0300F3CABF40165917591859196
:1070A0009491A8A9B9A9CD90DD90ED90FD90B9ABD0
:1070B000A8ABA70196010F945E1B2B013C0120E0B9
:1070C00030E040EA51EC0F94851D87FD10C020E0B0
:1070D00030E040EA51E4C301B2010F9426171816BC
:1070E00034F0F10140825182628273820EC0F80155
:1070F00084911816B4F7F7FAF094F7F8F094D101E8
:10710000CD92DD92ED92FC921397D101CD90DD905E
:10711000ED90FD901D0120E030E040EA51ECC70108
:10712000B6010F94851D87FF03C0E9E7F8E10BC0A6
:1071300020E030E040EA51E4C701B6010F94261781
:10714000181674F5F2CF84918F010F5F1F4F8823BB
:1071500021F00F949602F801F6CFE5EBF2E084916E
:107160008F010F5F1F4F882321F00F949602F801C3
:10717000F6CF61E087EA92E00E94F9450E942A7A00
:1071800088E290E099A388A388EC90E09DA38CA36B
:10719000BE01605E7F4FCE0184960E94497374C227
:1071A000B4E08B0E911C0F5F1F4FECA9E01374CF5E
:1071B0009CE2E92E94E0F92E10E0F5018191919185
:1071C000A191B1915F01F70181939193A193B19343
:1071D0007F01812F0E94E5551F5F133071F70E94D8
:1071E000CFC760E087E992E00E94F94583E992E029
:1071F0009DA38CA304E610E019A308A3BE016C5D57
:107200007F4FCE0180960E9449738AEB92E09DA346
:107210008CA319A308A3BE016C5D7F4FCE0180969D
:107220000E94497331C20E9488ED2EC20E9477E805
:107230002BC20F94540128C283E50E94D0448823B6
:1072400021F00E94AB5C91E089270E944DFD1CC299
:1072500083E50E94D044882309F416C20E94AB5CE7
:1072600080930B0411C2EAE3F2E484918F010F5F73
:107270001F4F882321F00F949602F801F6CFECE718
:10728000F2E084918F010F5F1F4F882321F00F944C
:107290009602F801F6CF8AE50E94D044882369F16E
:1072A0000E9499446B017C0120E030E040E050EC0A
:1072B0000F94851D87FF03C0E5E6F2E013C020E0D0
:1072C00030E040EA50E4C701B6010F9426171816C3
:1072D0009CF3C0929614D0929714E0929814F09276
:1072E00099140BC084918F010F5F1F4F882309F4FD
:1072F000CBC10F949602F801F5CF409196145091AE
:107300009714609198147091991482E692E00E940B
:107310008F918AE00F949602B7C180E090E0A8ECCC
:10732000B2E489839A83AB83BC8380E090E0A6E9D2
:10733000B3E48D839E83AF83B88780E090E0A0EABA
:10734000B1E489879A87AB87BC870E94D3F38823EF
:1073500019F081E00E94635A85E40E94D04488239A
:1073600019F00E94994404C060E070E080E090EC65
:107370006CA77DA78EA79FA78AE50E94FF4488235C
:1073800079F08AE50E94FF44882319F00E9499440D
:1073900003C060E070E0CB0169877A878B879C87A8
:1073A00088E50E94FF44882379F088E50E94FF4425
:1073B000882319F00E94994403C060E070E0CB017B
:1073C00069837A838B839C8389E50E94FF448823A9
:1073D00079F089E50E94FF44882319F00E949944BE
:1073E00003C060E070E0CB016D837E838F8398875C
:1073F00085E50E94D044882319F00E94994404C076
:1074000060E070E088EC92EC68A779A78AA79BA758
:107410008CE40E94D044882319F00E94994403C050
:1074200060E070E0CB016CA37DA38EA39FA382E4F8
:107430000E94FF44882321F00E947844162F01C047
:1074400015E0F0901C118091A704811171C001E03A
:10745000212FAE01485D5F4FBE016F5F7F4FCE01B0
:107460008C960E940E62882309F462C081E08093AA
:10747000A8048091A804882309F446C060E0812F05
:107480000F9431128091AA108823D1F10093AE108D
:1074900083E99CE70E9464B38091A804882321F0CB
:1074A00081E00E94BC83F8CF109207041092080478
:1074B0001092090410920A041092AA100E944552D8
:1074C0000F94D6110093AE108DE39CE70E9464B335
:1074D0000E9407D0DC01CB0188539045AF4FBF4FCE
:1074E0008093070490930804A0930904B0930A04BE
:1074F0001092AA100093A80461E0812F0F9431121A
:1075000081E00E94BC83B5CF80E090E0A0EAB1E4C6
:1075100088A399A3AAA3BBA38091A704882341F0C1
:10752000412FBE01605E7F4FCE0184960E940463AE
:10753000F1E0FF12A9C00E94CCB2A6C01F5F1430B8
:1075400069F0D7018D917D010E94D0448823B1F369
:107550000E947844812F0E94BFA6F0CF82E40E944F
:10756000D044882329F00E94784484E00E94BFA67A
:1075700083E50E94D044882309F486C010E00E946D
:107580007844812F0E94BFA61F5F1530C1F77CC0D1
:1075900083E50E94FF44882321F00E9478448B01F8
:1075A00002C000E010E080E50E94FF44882321F043
:1075B0000E947844CB0102C080E090E0B8010E94B4
:1075C000B0A662C00E9441BF5FC00E9440885CC0FC
:1075D000F090B604FF2029F1EAE3F2E484918F01F0
:1075E0000F5F1F4F882321F00F949602F801F6CF0A
:1075F00084E50F9496026F2D70E080E090E04AE001
:107600000F94EF0280E20F94960204E013E0F80179
:1076100081918F01882311F40C94DC300F94960231
:10762000F6CF10927C14EAE3F2E484918F010F5FAD
:107630001F4F882321F00F949602F801F6CF609136
:107640007C1470E080E592E00E94AC918AE00F9497
:1076500096021AC0EAE3F2E484918F010F5F1F4F94
:10766000882321F00F949602F801F6CF609104046C
:10767000709105048DE392E00E94C59182E20F941F
:1076800096028AE00F9496020E940786A4C40E9484
:107690008C538CE694E10E94B2850E944A918091BD
:1076A000AF0483FD86C0C0907814D0907914E09028
:1076B0007A14F0907B142091B6143091B714409155
:1076C000B8145091B914C701B6010F942617882336
:1076D00009F46FC00E940483882301F1C092B6149C
:1076E000D092B714E092B814F092B914EAE3F2E43D
:1076F00084918F010F5F1F4F882321F00F94960212
:10770000F801F6CFEDE8F7E084918F010F5F1F4F8E
:10771000882321F00F949602F801F6CFC0907814D8
:10772000D0907914E0907A14F0907B142091B614E4
:107730003091B7144091B8145091B914C701B601F3
:107740000F945E1B9F77E0917C1424E0E29FF00190
:107750001124E95FFD4F20813181428153810F94D3
:107760008B1720E030E048E453E40F94851D181691
:1077700004F5C092B614D092B714E092B814F09207
:10778000B914EAE3F2E484918F010F5F1F4F88235D
:1077900021F00F949602F801F6CFEEE6F7E084911F
:1077A0008F010F5F1F4F882321F00F949602F8017D
:1077B000F6CF6091930270919402072E000C880B13
:1077C000990B0F942C172091990230919A024091B5
:1077D0009B0250919C020F948B172AE037ED43E2F5
:1077E0005CE30F948B170E9493550E9423454CCF66
:1077F00080E00E944C5A0E943D5485E40E94FF4460
:10780000882319F00E94AB5C03C085E40E94D04439
:1078100021E0482FBE016F5F7F4FCE0180960E940E
:1078200078F56B017C019B01AC010F940B1E81115B
:1078300031C02CEA35EC47E257E368A179A18AA16F
:107840009BA10F945F1BAB01BC0187E497E00E94F2
:1078500072912CEA35EC47E257E369817A818B819A
:107860009C810F945F1BAB01BC0182E497E00E94F6
:1078700072912CEA35EC47E257E3C701B6010F9449
:107880005F1BAB01BC018DE397E00E9472918AE01F
:107890000F9496020E9423540E94CFC7F5CE802FEA
:1078A0000E9408B16E2D802F0E94D9CEF12CB70115
:1078B000802F0E9408CF0630110529F4F092A6040B
:1078C000E092A504E1CE0830110509F0DDCEF0927A
:1078D000A404E092A304D8CE0E948844853620F008
:1078E00084E68093A204D0CE8093A204CDCE0E94E1
:1078F00099440F94A31C70939D0460939C0480E0B2
:107900000E94455260919C0470919D04072E000CCA
:10791000880B990B0F942C1720919E0430919F0493
:107920004091A0045091A1040F94851D18160CF0ED
:1079300052C183ED92E09F938F9385E096E09F93F1
:107940008F931F920E9405B30F900F900F900F908E
:107950000F9081E0809306021CAA1DAA1EAA1FAAEE
:107960001CAE1DAE1EAE1FAE10E021961FAE2197BD
:107970004CE325964FAF25975CE129965FAF299799
:1079800086E42D968FAF2D97C12CD12C70E8E72E71
:10799000EFEBFE2E812C912C540160919C04709190
:1079A0009D04072E000C880B990B0F942C17062FA3
:1079B000772E682E592E262F372F482F592FB60194
:1079C000C7010F9426178823C9F020919E04309197
:1079D0009F044091A0045091A104602F772D862D23
:1079E000952D0F942617182F111F1127111F98A9D5
:1079F000992341F0112331F011E0DBC00C2D7D2CD7
:107A00006E2C5F2C0E9407D06B017C01DC01CB0146
:107A10002CAD3DAD4EAD5FAD821B930BA40BB50BF2
:107A2000B7FD3BC0D701C60188519C4FAF4FBF4F38
:107A30008CAF9DAFAEAFBFAF0E94B14FE1E0F6E0BB
:107A400084911F019FEF291A390A882321F00F948E
:107A50009602F101F5CF81149104A104B104B9F0AB
:107A6000D501C40188519C4FAF4FBF4FBC01CD0120
:107A70006C197D098E099F0928EE33E040E050E043
:107A80000F94011BCA01B9010E94EAA503C08FE34C
:107A90000F9496028AE00F94960280E00E94BC83C5
:107AA0000E944A91A0919E04A8AF20909F0430901C
:107AB000A0044090A1042A2F322D432D542D602F75
:107AC000772D862D952D0F945E1B9F7720E030E05B
:107AD00040E251E481149104A104B10429F40F940B
:107AE000261787FF07C004C00F94851D181614F4CD
:107AF00046015701112309F442C02CA93DA94EA902
:107B00005FA9211531054105510541F0D701C60195
:107B1000821B930BA40BB50BB7FD31C028AD322DE2
:107B2000432D542D21966FAD219725967FAD259736
:107B300029968FAD29972D969FAD2D970F945E1B9B
:107B400020E030E040EC5FE30F94261787FD54CF30
:107B5000D701C601805A9541AF4FBF4F8CAB9DAB4B
:107B6000AEABBFAB98AD21969FAF219725962FAEB8
:107B7000259729963FAE29972D964FAE2D97809148
:107B800006028823B1F081149104A104B10429F400
:107B9000C02ED72CE62CF52C00CFA8EECA1AA3E0F5
:107BA000DA0AE108F108C818D908EA08FB08F7FC66
:107BB000EFCF80910602882309F466CD60E011239F
:107BC00029F085EE95E00E94F9455ECD83EF95E0C2
:107BD0000E94F94559CDF8A9F111BBCE8EED92E086
:107BE000AACEA7D60F94A31C6739710514F066E9D5
:107BF00070E070939B0460939A040E94FA51609124
:107C00009A0470919B04072E000C880B990B0F941B
:107C10002C1720919004309191044091920450913E
:107C200093040F94261787FF04C060E088ED95E069
:107C300003C060E08BEC95E0DCD781E08093060226
:107C400080917C14809394041CAA1DAA1EAA1FAACA
:107C50001CAE1DAE1EAE1FAE18AA21961FAE2197F8
:107C6000BCE32596BFAF2597ECE12996EFAF2997A6
:107C7000F6E42D96FFAF2D97C12CD12C50E8E52EC0
:107C80006FEBF62E812C912C540160919A04709127
:107C90009B04072E000C880B990B0F942C17162FA2
:107CA000072F782E692E262F372F482F592FB601F0
:107CB000C7010F942617882309F120919004309171
:107CC00091044091920450919304612F702F872D5D
:107CD000962D0F942617881F8827881F88AB28ADFC
:107CE000222381F0882371F080910602882309F411
:107CF000CBCC60E08DEB95E07CD7C6CC1C2D0D2D58
:107D00007E2C6F2C0E9407D06B017C01DC01CB0123
:107D10002CAD3DAD4EAD5FAD821B930BA40BB50BEF
:107D2000B7FD3BC0D701C60188519C4FAF4FBF4F35
:107D30008CAF9DAFAEAFBFAF0E94B14FE7ECF5E0A7
:107D400084912F019FEF491A590A882321F00F943B
:107D50009602F201F5CF81149104A104B104B9F0A7
:107D6000D501C40188519C4FAF4FBF4FBC01CD011D
:107D70006C197D098E099F0928EE33E040E050E040
:107D80000F94011BCA01B9010E94EAA503C08FE349
:107D90000F9496028AE00F94960280E00E94BC83C2
:107DA0000E944A9120909004309091044090920457
:107DB000509093049101A201612F702F872D962D71
:107DC0000F945E1B9F7720E030E040EA50E481147E
:107DD0009104A104B10429F40F94261787FF07C06A
:107DE00004C00F94851D181614F446015701A8A964
:107DF000AA2309F43FC02CA93DA94EA95FA92115CA
:107E000031054105510541F0D701C601821B930B95
:107E1000A40BB50BB7FD2EC09101A20121966FAD49
:107E2000219725967FAD259729968FAD29972D9679
:107E30009FAD2D970F945E1B20E030E040EC5FE398
:107E40000F94261787FD50CFD701C601805A954160
:107E5000AF4FBF4F8CAB9DABAEABBFAB21962FAE40
:107E6000219725963FAE259729964FAE29972D96B7
:107E70005FAE2D9780910602882309F435CF8114D7
:107E80009104A104B10429F4C12ED02EE72CF62CC4
:107E9000FCCE98EEC91A93E0D90AE108F108C81897
:107EA000D908EA08FB08F7FE1FCFEECF0E9425A7EE
:107EB00088E576D5882319F0179A10928D0489E504
:107EC0006FD5882319F0169A10928E048AE568D52A
:107ED000882319F0159A10928F0485E461D58823C0
:107EE00009F4D2CB0E944983CFCB23D520E030E0E8
:107EF00040E050EC0F94261787FD13C01AD520E000
:107F000030E040E050E40F94851D181624F011D5A0
:107F10006B017C010BC0C12CD12CE12C40E4F42E70
:107F200005C0C12CD12CE12C30ECF32E2091C214D1
:107F30003091C3144091C4145091C514C701B601C7
:107F40000F948B170F94A31C20918F04222351F0C0
:107F500020912A0430912B04620F731F70932B041D
:107F600060932A0480E51CD5882329F00E94AB5C2D
:107F7000882309F489CBA70196016091961470912A
:107F8000971480919814909199140F945F1B6093AB
:107F90009614709397148093981490939914EAE32D
:107FA000F2E484918F010F5F1F4F882321F00F941B
:107FB0009602F801F6CF4091961450919714609173
:107FC00098147091991480E693E00E948F918AE052
:107FD0000F94960259CBC45BDF4F0FB6F894DEBF07
:107FE0000FBECDBFDF91CF911F910F91FF90EF900A
:107FF000DF90CF90BF90AF909F908F907F906F90C9
:108000005F904F903F902F900895CF92DF92EF9224
:10801000FF920F931F93CF93DF9300D01F92CDB7A2
:10802000DEB78091AF109091B010A091B110B091D7
:10803000B210B7FF08C01092AF101092B01010929B
:10804000B1101092B2108091CA059091CB05A09109
:10805000CC05B091CD054091AF105091B01060911A
:10806000B1107091B21084179507A607B70744F4B2
:108070008093AF109093B010A093B110B093B21052
:1080800080913D02882379F14091AF105091B0105A
:108090006091B1107091B2108091CE059091CF0592
:1080A000A091D005B091D1056A017B01C80ED91EFF
:1080B000EA1EFB1EC701B6010F942C172AE037ED0C
:1080C00043E25CE30F948B1769837A838B839C83F1
:1080D000CE0101960E944CE3BC018091D4059091A1
:1080E000D5050E94437A8091D5041091D60581115F
:1080F00006C01123D1F180913D028823B1F1409156
:10810000AF105091B0106091B1107091B210809189
:10811000CE059091CF05A091D005B091D1056A010F
:108120007B01C80ED91EEA1EFB1EC701B6010F94C3
:108130002C172AE037ED43E25CE30F948B17E091B4
:10814000D205F091D305309721F06083718382834B
:108150009383112329F0E091D705F091D805199563
:108160008091D50481110E942E7A8091D5048823B4
:1081700029F0E091D705F091D80519950F900F904F
:108180000F900F90DF91CF911F910F91FF90EF9083
:10819000DF90CF900895CF92DF92EF92FF920F93EE
:1081A0001F93CF93DF9300D01F92CDB7DEB780919E
:1081B000AF109091B010A091B110B091B210B7FF74
:1081C00008C01092AF101092B0101092B11010921F
:1081D000B2108091CA059091CB05A091CC05B091C9
:1081E000CD054091AF105091B0106091B1107091D9
:1081F000B21084179507A607B70744F48093AF1011
:108200009093B010A093B110B093B21080913D0242
:10821000882379F14091AF105091B0106091B11066
:108220007091B2108091CE059091CF05A091D005AC
:10823000B091D1056A017B01C80ED91EEA1EFB1E52
:10824000C701B6010F942C172AE037ED43E25CE337
:108250000F948B1769837A838B839C83CE0101965D
:108260000E9401E4BC018091D4059091D5050E9443
:10827000437A8091D5041091D605811106C011234F
:10828000D1F180913D028823B1F14091AF1050911E
:10829000B0106091B1107091B2108091CE059091A4
:1082A000CF05A091D005B091D1056A017B01C80E20
:1082B000D91EEA1EFB1EC701B6010F942C172AE037
:1082C00037ED43E25CE30F948B17E091D205F09118
:1082D000D305309721F060837183828393831123C8
:1082E00029F0E091D705F091D80519958091D50432
:1082F00081110E942E7A0F900F900F900F90DF91B6
:10830000CF911F910F91FF90EF90DF90CF90089544
:10831000CF92DF92EF92FF920F931F93CF93DF9351
:1083200000D01F92CDB7DEB78091AF109091B01002
:10833000A091B110B091B210B7FF08C01092AF1069
:108340001092B0101092B1101092B2108091CA0524
:108350009091CB05A091CC05B091CD054091AF1087
:108360005091B0106091B1107091B21084179507C0
:10837000A607B70744F48093AF109093B010A09372
:10838000B110B093B21080913D02882379F14091F1
:10839000AF105091B0106091B1107091B2108091F7
:1083A000CE059091CF05A091D005B091D1056A017D
:1083B0007B01C80ED91EEA1EFB1EC701B6010F9431
:1083C0002C1720E030E048EC52E40F948B176983BF
:1083D0007A838B839C83CE0101960E9482E4BC0148
:1083E0008091D4059091D5050E94437A8091D5045F
:1083F0001091D605811106C01123D1F180913D0263
:108400008823B1F14091AF105091B0106091B1103C
:108410007091B2108091CE059091CF05A091D005BA
:10842000B091D1056A017B01C80ED91EEA1EFB1E60
:10843000C701B6010F942C1720E030E048EC52E45D
:108440000F948B17E091D205F091D305309721F06E
:108450006083718382839383112329F0E091D70590
:10846000F091D80519958091D50481110E942E7A3A
:108470000F900F900F900F90DF91CF911F910F9160
:10848000FF90EF90DF90CF900895CF92DF92EF9220
:10849000FF920F931F93CF93DF9300D01F92CDB71E
:1084A000DEB78091AF109091B010A091B110B09153
:1084B000B210B7FF08C01092AF101092B010109217
:1084C000B1101092B2108091CA059091CB05A09185
:1084D000CC05B091CD054091AF105091B010609196
:1084E000B1107091B21084179507A607B70744F42E
:1084F0008093AF109093B010A093B110B093B210CE
:1085000080913D02882379F14091AF105091B010D5
:108510006091B1107091B2108091CE059091CF050D
:10852000A091D005B091D1056A017B01C80ED91E7A
:10853000EA1EFB1EC701B6010F942A1720E030E0A7
:1085400048EC52E40F948B1769837A838B839C8366
:10855000CE0101960E9482E4BC018091D4059091E5
:10856000D5050E94437A8091D5041091D6058111DA
:1085700006C01123E1F180913D028823C1F14091B1
:10858000AF105091B0106091B1107091B210809105
:10859000CE059091CF05A091D005B091D1056A018B
:1085A0007B01C80ED91EEA1EFB1EC701B6010F943F
:1085B0002A1720E030E048EC52E40F948B170F9418
:1085C000A81CE091D205F091D305309721F060838B
:1085D000718382839383112329F0E091D705F09171
:1085E000D80519958091D50481110E942E7A809129
:1085F000D504882329F0E091D705F091D805199585
:108600000F900F900F900F90DF91CF911F910F91CE
:10861000FF90EF90DF90CF9008950F931F93CF932B
:108620008091AF109091B010A091B110B091B210A4
:10863000B7FF08C01092AF101092B0101092B11096
:108640001092B2108091CA059091CB05A091CC05F3
:10865000B091CD054091AF105091B0106091B11024
:108660007091B21084179507A607B70744F480935A
:10867000AF109093B010A093B110B093B21080914E
:108680003D02882331F14091AF105091B0106091BC
:10869000B1107091B2108091CE059091CF05A0914C
:1086A000D005B091D1058A019B01080F191F2A1F1F
:1086B0003B1FC901B8010F942C170F94A31CCB01C9
:1086C0000E94D3E5BC018091D4059091D5050E940C
:1086D000437A8091D504C091D605811106C0CC2380
:1086E000A1F180913D02882381F14091AF1050911A
:1086F000B0106091B1107091B2108091CE05909140
:10870000CF05A091D005B091D1058A019B01080F3A
:10871000191F2A1F3B1FC901B8010F942C17E091A4
:10872000D205F091D305309721F060837183828365
:108730009383CC2329F0E091D705F091D8051995C2
:108740008091D50481110E942E7A8091D504CF9119
:108750001F910F91089561CF60DF882329F0E09188
:10876000D705F091D805199408958091AF10909194
:10877000B010A091B110B091B210B7FF08C0109224
:10878000AF101092B0101092B1101092B2108091F0
:10879000CA059091CB05A091CC05B091CD05409133
:1087A000AF105091B0106091B1107091B210841759
:1087B0009507A607B70744F48093AF109093B010C5
:1087C000A093B110B093B21080913D02882399F02C
:1087D0002091CE053091CF058091AF109091B010CF
:1087E000820F931F0E94D3E5BC018091D405909124
:1087F000D5050E94437A8091D5042091D605811138
:1088000006C0222311F180913D028823F1F04091AE
:10881000CE055091CF058091AF109091B010840F8C
:10882000951FE091D205F091D305309711F0918317
:108830008083222329F0E091D705F091D80519957E
:108840008091D50481110E942E7A8091D5040895DB
:108850008CCF8BDF882329F0E091D705F091D805E4
:1088600019940895CF93DF9360E085E00E94AB797F
:10887000D091BA04C0E0D11109C080913D02882393
:10888000E9F021E041E061EC77E015C0D13049F436
:1088900080913D02882391F020E041E062EB77E097
:1088A0000AC0D23059F480913D02882339F020E08B
:1088B00041E068EA77E08C2F0E947D73CF5FDF5F35
:1088C000C530C9F683E08093B904DF91CF91089554
:1088D0008091020590910305009731F04AE050E045
:1088E00060E070E00D94421560E070E0CB01089507
:1088F0008091020590910305009731F04AE050E025
:1089000060E070E00D941A1460E070E0CB0108950F
:10891000EFDF97FD0AC0ECDF6F3F71058105910520
:1089200009F02CF4E5DF862F089580E008958FEF9D
:1089300008950F931F93CF938091020590910305A3
:10894000009711F1FC018F01C1912C2F2F7DA9F00F
:10895000C53411F0C536B9F7F801108260E070E057
:1089600080910205909103050F94B312F801C08322
:10897000562F472F382F292F0BC060E070E0CF9182
:108980001F910F910D94B31250E040E030E020E0D1
:10899000652F742F832F922FCF911F910F910895E0
:1089A00081548A3150F5482F50E0FA0193E0F59553
:1089B000E7959A95E1F7E25CF74F208130E0877008
:1089C000B90102C0759567958A95E2F760FF15C0F9
:1089D000FA01EC5DF74F2081222339F080910404E5
:1089E00090910504820F911D02C080E090E0909369
:1089F00003058093020581E0089580E00895D0DFAB
:108A0000882341F081E02091020530910305232B5A
:108A100009F480E00895FC0123812111F7C5089530
:108A20002091FC109091FD1081E0291301C080E09D
:108A3000089580E1EAEAF4E1ACE6B4E101900D9238
:108A40008A95E1F7089580E1ECE6F4E1AAEAB4E161
:108A500001900D928A95E1F7089543E952E064E6AA
:108A600070E080E090E00F94FB0B4AEB52E064E68C
:108A700070E080E090E00D94FB0B0F931F93CF9379
:108A8000DF93982F862F8A01D22F692F0E94CF7AE9
:108A9000909146148091DA05891748F19091481415
:108AA0008091D905981718F1C4E1F80184918823C1
:108AB00031F00E94A090C81B0F5F1F4FF6CFCC2350
:108AC00029F080E20E9463B2C150F9CF8091DA05AB
:108AD0009AE79093491480934A148D2F0E94B7907F
:108AE00080E2DF91CF911F910F910C9463B2DF91DF
:108AF000CF911F910F91089589EE97E00E9416B2D1
:108B000081E08093DE0408950F931F930E9407D0A5
:108B10000091DA041091DB042091DC043091DD0433
:108B2000DC01CB01801B910BA20BB30BB7FD0FC077
:108B30008091030185FB992790F981E08927909125
:108B4000030196FF8260629B84608093D9048091C8
:108B5000D90481709091D90491FD82609091D804DC
:108B6000891731F18130A9F028F0823041F083304B
:108B700059F01CC0913089F0923099F017C09923B8
:108B800061F0933071F012C0913059F0923071F46D
:108B900004C0992331F0933049F49091D7049F5F3A
:108BA00003C09091D70491509093D7048093D80438
:108BB0001F910F910895EEE3F2E080E09191911101
:108BC00004C0982F981B50E206C0863111F08F5FC9
:108BD000F5CF96E1F7CF282F30E0492F480FF90164
:108BE000E25CFD4F463118F450838F5FF4CF108262
:108BF0000895FC0167FF03C01092B31060E020915C
:108C0000B31030E0462F062E000C550B42175307C9
:108C10006CF06093B31042E450E0BF018EE392E049
:108C20000F949616C8DF83E080933D02089520914B
:108C3000B31021110BC0BC0142E450E08EE392E07E
:108C40000F94B21EB8DF83E080933D0208954F92E7
:108C50005F926F927F928F929F92AF92BF92CF92CC
:108C6000DF92EF92FF920F931F93CF93DF93CDB7D5
:108C7000DEB760970FB6F894DEBF0FBECDBF109180
:108C80000C021F3F01F10E9407D0C090C004D09099
:108C9000C104E090C204F090C304DC01CB018C1944
:108CA0009D09AE09BF09B7FD0EC02091FD1080914E
:108CB000FC1030E08F5F8F70082E000C990B281786
:108CC000390709F027C220DF8091D90482FF39C01B
:108CD0008091D604811137C081E08093D6049091B1
:108CE000A80489278093D5041092A80483E0809378
:108CF0003D021092D9040E9407D0DC01CB018C50B8
:108D00009E4FAF4FBF4F8093DA049093DB04A09344
:108D1000DC04B093DD0448E853E162E070E080E0F9
:108D200090E00F94FB0B16E0115069F08EEF90E18C
:108D30000E94D28F62E070E080E090E00E94CFCF8E
:108D4000F3CF1092D60419B11295117081E0182753
:108D50008091D404412F50E0282F30E04217530770
:108D6000A1F0112309F426C20E94C3718091D4049A
:108D7000823021F060E08BED97E03BDF1093D4046C
:108D800083E080933D020E941F900E9407D06B01F8
:108D90007C018091D0049091D104A091D204B09133
:108DA000D304A7019601281B390B4A0B5B0B57FF15
:108DB00005C08091AB10882309F44FC2D701C601CA
:108DC0008C599F4FAF4FBF4F8093D0049093D104E5
:108DD000A093D204B093D3048091D70418162CF436
:108DE0008091D704823074F408C08091D704992709
:108DF00081950CF4909502972CF48091D504811103
:108E00009BC0ABC08091CF04882309F46EC08091D1
:108E1000D704181654F48091D704082E000C990B2F
:108E200097FD0196959587950CC08091D704082EE3
:108E3000000C990B97FD01969595879591958195D5
:108E400091098090CB049090CC04A090CD04B09078
:108E5000CE0481149104A104B104D1F1BC01990F95
:108E6000880B990B0F942C172B013C01C701B601FD
:108E7000681979098A099B090F942A179B01AC018B
:108E8000C301B2010F943B1C20E030E04AE754E4F8
:108E90000F948B174B015C0120E030E040E253E47B
:108EA0000F94851D87FF0FC020E030E046E952E4B3
:108EB000C501B4010F94851D87FD0AC02AE030E08A
:108EC00040E050E009C024E630E040E050E004C05B
:108ED00021E030E040E050E0C092CB04D092CC04DE
:108EE000E092CD04F092CE0404C021E030E040E0F6
:108EF00050E0A091D7040A2E000CBB0B0F94491B25
:108F000022E030E040E050E00F94231B8091AF104E
:108F10009091B010A091B110B091B210820F931F38
:108F2000A41FB51F8093AF109093B010A093B11001
:108F3000B093B2101092D704D701C6018856954C51
:108F4000AF4FBF4F8093C7049093C804A093C90448
:108F5000B093CA0481E080933D0220913B0230919E
:108F60003C0244E72A3B340741F480919D02882368
:108F700009F42BC1815080939D022F513F4771F41A
:108F80008091CD149091CE14891740F490919D0258
:108F9000992309F42AC1915090939D022FB7F89418
:108FA00080917F0B9091800BA091810BB091820BEF
:108FB0002FBF3AE0B695A795979587953A95D1F743
:108FC000009721E0A207B10520F08FEF9FEFA0E00E
:108FD000B0E09695879520913D02211105C0309112
:108FE000AB10311136C159C0009741F04091C50412
:108FF0005091C6044817590708F04FC08091AB1034
:10900000811113C0223050F0243028F0243031F484
:1090100010923D0203C081E080933D020E942FB375
:1090200081E08093C4048093AB1084E00E9486901A
:1090300081E080933214E0913B02F0913C0219955B
:109040001092D5041092C4048091AB10882351F083
:109050000E9427B191E0811101C090E09093AB1084
:109060009111DBC08090C5049090C604A12CB12C56
:109070000E9407D0DC01CB018C199D09AE09BF0904
:1090800088169906AA06BB0640F40E9407D06C1900
:109090007D097093C6046093C50480913B02909152
:1090A0003C028A5B944721F08091AE10882379F0CE
:1090B00048E9C40E4AE3D41EE11CF11CC092C70467
:1090C000D092C804E092C904F092CA040FC0809103
:1090D000C7049091C804A091C904B091CA04C81AE9
:1090E000D90AEA0AFB0AF7FE0E942A7A8091AB109D
:1090F0008111B3C080913D02813049F008F4ADC0C8
:10910000843008F0AAC081E080933D02A6C010928E
:109110003D02A3C054E01502F0011124E75EFC4FAC
:1091200020E030E040E752E46081718182819381E8
:109130000F943B1C6D877E878F87988B8091AA1434
:109140009091AB14A091AC14B091AD1489839A8323
:10915000AB83BC838091AE149091AF14A091B014F6
:10916000B091B1148D839E83AF83B8878091B21480
:109170009091B314A091B414B091B51489879A87D3
:10918000AB87BC87CE0101960E943991E12C8E01FC
:10919000035F1F4F26EB34E1AE01475F5F4FBE0117
:1091A0006B5F7F4FCE0101960E94B7A28FEF809335
:1091B0000C0289CD10925B1110925C11823009F47F
:1091C000DDCD60E08EEC97E0D8CD8CE080939D0201
:1091D0008091C5049091C60401979093C604809332
:1091E000C50481E080933D02C8CE96E090939D0235
:1091F00091E090933D028F5F8093CD14D701C6011B
:109200008856954CAF4FBF4F8093C7049093C804C6
:10921000A093C904B093CA04C1CE8090C5049090B5
:10922000C604A12CB12C0E9407D0DC01CB018C1903
:109230009D09AE09BF0988169906AA06BB0668F4FF
:109240000E9407D06C197D097093C6046093C50411
:1092500004C0009709F4E9CEC9CE60960FB6F89421
:10926000DEBF0FBECDBFDF91CF911F910F91FF9059
:10927000EF90DF90CF90BF90AF909F908F907F90B6
:109280006F905F904F900895CF92DF92EF92FF9290
:109290000F931F930E9407D00091BC041091BD044E
:1092A0002091BE043091BF046B017C01C01AD10A29
:1092B000E20AF30AF7FC13C02091BB042095209327
:1092C000BB04DC01CB018A549C4FAF4FBF4F80934E
:1092D000BC049093BD04A093BE04B093BF0481E08E
:1092E0009091BB04911101C080E01F910F91FF90FC
:1092F000EF90DF90CF9008950E941F90A4E0B1E01E
:109300008C918F7D8C939FB7F894E5E0F1E080819C
:10931000806280839FBF8C918F7B8C939FB7F894E2
:109320008081806480839FBF6A98729A54985C9A07
:1093300082E08093D404E8DB1092D7040895CF93A1
:10934000DF931F921F92CDB7DEB789839A830E9465
:109350000A7A89819A810F900F90DF91CF910C94B6
:1093600064B36F927F928F929F92AF92BF92CF928F
:10937000DF92EF92FF920F931F93CF93DF9300D072
:109380001F92CDB7DEB76C013B014701580129831D
:109390003A834B835C830E940A7A83E080933D0288
:1093A000D092D505C092D4057092D3056092D205B3
:1093B00029813A814B815C81CA01B9010F94A31CB8
:1093C0006093CE057093CF058093D0059093D1051F
:1093D0000F942C176B017C019B01AC01C501B401FA
:1093E0000F945E1B0F94A31C6093CA057093CB056A
:1093F0008093CC059093CD05A7019601F301608180
:109400007181828193810F945E1B0F94A81C6093DD
:10941000AF107093B0108093B1109093B2108BEA9C
:1094200093E490933C0280933B020F900F900F9037
:109430000F90DF91CF911F910F91FF90EF90DF90F0
:10944000CF90BF90AF909F908F907F906F90089536
:10945000CF92DF92EF92FF920F931F93CF93DF9300
:109460008C01EB016A0179010E940A7A23E02093C2
:109470003D021093D5050093D405D093D305C09336
:10948000D205A601DD0C660B770B4093CE055093F9
:10949000CF056093D0057093D105C701FF0CAA0BCF
:1094A000BB0B841B950BA60BB70B8093CA0590933F
:1094B000CB05A093CC05B093CD0588819981092E69
:1094C000000CAA0BBB0B841B950BA60BB70B809350
:1094D000AF109093B010A093B110B093B21088E287
:1094E00094E490933C0280933B02DF91CF911F91D3
:1094F0000F91FF90EF90DF90CF900895EF92FF9241
:109500000F931F93CF93DF931F92CDB7DEB78C01DC
:109510007B0180E249830F94960249814F3F11F00D
:1095200084E501C082E40F9496028AE30F949602C8
:10953000F801608171818281938142E00F9455032B
:10954000F70140815181628173818BEE91E10E942C
:109550008F9162E070E080E090E00F90DF91CF911A
:109560001F910F91FF90EF900C94CFCF0F931F930B
:10957000CF93DF93EB01FC012381211102C080E036
:1095800040C02250223028F48FE28883198281E083
:1095900038C08C01FC01648575858685978540E01F
:1095A0000F94640C882359F3F8014089F0E24F9F2F
:1095B000A00111249A012F513A4F232B01F320E0EF
:1095C00030E090E06EE2F901E40FF51FEF51FA4F41
:1095D0007081703271F02830310529F4DE01A90F55
:1095E000B11D6C939F5F7081FE01E90FF11D7083C7
:1095F0009F5F2F5F3F4F2B30310529F7C90FD11DDA
:109600001882DF91CF911F910F910895CF93DF932F
:10961000EC010F94AC041B82DF91CF9108953F922F
:109620004F925F926F927F928F929F92AF92BF9272
:10963000CF92DF92EF92FF920F931F93CF93DF931E
:10964000CDB7DEB72C970FB6F894DEBF0FBECDBFF7
:109650005C01DC0159968D909C905A97F4018185AC
:109660009285A385B4859C01AD012F5F3F4F4F4F7D
:109670005F4F29873A874B875C87D5011496CD9039
:10968000DD90ED90FC901797C114D104E104F10432
:1096900039F0BFEFCB1ADB0AEB0AFB0A312C07C00B
:1096A000F401C080D180E280F3803324339426011A
:1096B00037011D821E821F821886F40181859285E2
:1096C000A385B4852D813E814F81588528173907A0
:1096D0004A075B0708F064C089859A85AB85BC851D
:1096E0008C159D05AE05BF0550F482E0C82ED12C27
:1096F000E12CF12C92E0492E512C612C712C9E0111
:109700002F5F3F4FB701A601C4010F942D0D882391
:1097100009F446C089819A81AB81BC81892B8A2B4F
:109720008B2B41F0260137019FEF491A590A690A2C
:10973000790A05C0C414D504E604F70491F02D811C
:109740003E814F8158852F5F3F4F4F4F5F4F2D8395
:109750003E834F8358873FEFC31AD30AE30AF30AC5
:10976000ACCF0FEF1FEF2FEF3FE0B301A201C40119
:109770000F949C0CF82E882399F0D50114964D91E6
:109780005D916D917C9117974115510561057105AA
:1097900049F093018201C4010F949C0C811102C015
:1097A000F12C29C0D50114964D925D926D927C9258
:1097B0001797332051F0D301C2010196A11DB11DAD
:1097C000F40180839183A283B383F501858996890F
:1097D000A789B08D892B8A2B8B2B69F4D5015596DF
:1097E0004D925D926D927C92589711968C91119743
:1097F000806811968C938F2D2C960FB6F894DEBF4F
:109800000FBECDBFDF91CF911F910F91FF90EF90D1
:10981000DF90CF90BF90AF909F908F907F906F9090
:109820005F904F903F9008954F925F926F927F921A
:109830009F92AF92BF92CF92DF92EF92FF920F93DF
:109840001F93CF93DF931F92CDB7DEB78C017B01BF
:109850006A01A22EDB0159968D919C915A97F801CD
:10986000928F818F40E050E0BA01C7010F94ED0460
:10987000912CF70180859185A285B3854189528914
:109880006389748984179507A607B70708F064C031
:1098900025E0B695A795979587952A95D1F7F82F46
:1098A000FF70BF2ED70113968C91823008F46AC0E6
:1098B00041E050E0BE016F5F7F4FC7010F94020788
:1098C000019719F4898190E002C08FEF9FEF019614
:1098D00009F458C0F70180859185A285B3854F961C
:1098E000A11DB11D80879187A287B387F0E2BF9E3B
:1098F000C0011124BC016F517A4F6115710509F443
:1099000041C0DB012C91222319F0253ED1F47EC108
:1099100091100EC04091E1075091E2076091E3077A
:109920007091E407F8014487558766877787B08A86
:10993000FC01EF51FA4F8081882361F099249394C0
:1099400098CF4BE050E0C6010F945E1E892B09F0C2
:1099500090CF1AC0992493948A2D8274823491F402
:10996000992009F49CC0D8015096BC9050971C9641
:109970006D917D918D919C911F9741E00F94640CA6
:10998000811180C080E045C1A7FCFCCFF0E2BF9E02
:10999000A00111249A012F513A4FD9011B968C91A5
:1099A000817121F08A2D827109F068C08091E107F0
:1099B0009091E207A091E307B091E407F801848752
:1099C0009587A687B787B08AFA01EF51FA4F448985
:1099D000558960E070E0BA0155274427D8015596B3
:1099E0004D935D936D937C935897828D938DA0E0FA
:1099F000B0E0482B592B6A2B7B2BD80155964D9301
:109A00005D936D937C935897D9011B968C918871C7
:109A100059F4848D958DA68DB78DF801818B928B2D
:109A2000A38BB48B81E010C0803141F598012F5E8B
:109A30003F4FD80159968D919C915A970F94AD0D37
:109A40008823E1F084E0F80183838A2D8F70D801A8
:109A500011968C931197F801148215821682178241
:109A600018961D921D921D921C921B97A4FEC1C0B8
:109A7000C8010E9495B48111BCC084CFD80113964F
:109A80001C9280CFF8016089F0E26F9FB001112431
:109A90006F517A4F6115710509F08BC073CFD701F3
:109AA00013968C911397823009F46CCF51968D9157
:109AB0009D910D90BC91A02D803E9F4FAF41B1056F
:109AC00008F060CFC701ABDD882309F45BCF0F94AA
:109AD000240C882309F456CFD70159962D913C9137
:109AE0005A9714968D919D910D90BC91A02D02973F
:109AF000A109B109F901058404C0880F991FAA1FA3
:109B0000BB1F0A94D2F74684578460887188480E38
:109B1000591E6A1E7B1E81E08093E9074092E1078F
:109B20005092E2076092E3077092E40780E092E0CF
:109B3000E1EEF5E0DF019C011D9221503040E1F79C
:109B4000BB24B394D7015996ED91FC915A97848127
:109B5000B81698F421EE35E0B301A2014B0D511D6A
:109B6000611D711D8091EA079091EB070E948FE2C1
:109B7000882309F407CFB394E5CF80E092E0A0E01A
:109B8000B0E0058404C0880F991FAA1FBB1F0A9468
:109B9000D2F7F7014189528963897489840F951F2F
:109BA000A61FB71F818B928BA38BB48B61EE75E0E0
:109BB000B12C80E2DB011D928A95E9F78BE0F6017A
:109BC000DB0101900D928A95E1F781E298E2FB01B9
:109BD000918B808B20E038E037872687938B828BB0
:109BE000918F808F378B268B0F94240C8111CECED2
:109BF000C9CEA5FE09C0F8014189528963897489DB
:109C0000C8010F94ED0405C081E003C0911096CE09
:109C100081CE0F90DF91CF911F910F91FF90EF9028
:109C2000DF90CF90BF90AF909F907F906F905F90AC
:109C30004F9008952F923F924F925F926F927F9232
:109C40008F929F92AF92BF92CF92DF92EF92FF924C
:109C50000F931F93CF93DF93CDB7DEB7C254D109D3
:109C60000FB6F894DEBF0FBECDBF4C015B018A0179
:109C7000322E1C8E1F8E19821C826115710511F403
:109C800010E0A4C0FC0183818111FACFFA01808128
:109C90008F3209F099C0F50183818250823060F0E3
:109CA000618D728DCE0101960F948508882341F352
:109CB000CE0101967C0101C07501C8018C0101969D
:109CC000F80120812F32D1F36E01FCE1CF0ED11CBF
:109CD0003601CE0101962C012396CFAE23972D2C71
:109CE0009BE09150E7E3F0E0EC0FFD1FE90FF11D61
:109CF00080E280839111F5CFD80127E04A2F3B2FD6
:109D00008D91811107C08FA9803209F4B9CF842FBA
:109D1000932F2CC08F32B9F38E3231F42A3009F4EC
:109D2000AFCF98E02AE0EACFE7EFF1E134913323B7
:109D300021F031963813FACFA3CF291708F4A0CF1A
:109D4000813208F49DCF8F3709F49ACF31E0390F73
:109D5000E7E3F0E0EC0FFD1FE90FF11D9FE9980F1D
:109D60009A3108F480528083932FC8CF8C01FC0174
:109D7000208101962F32D1F32223E9F021E0AE01B8
:109D8000495C5F4FB701C6014FDD882309F478CFE6
:109D9000EA14FB0411F0C70139DCC614D70441F002
:109DA00023969FAD2397822D7601C92ED82E98CF6A
:109DB000942D852DF9CF232DAE01495C5F4FB7015E
:109DC000C40132DD182F02C07B017ECFCE01019687
:109DD0000E940B45CE014C960E940B45812FCE5B15
:109DE000DF4F0FB6F894DEBF0FBECDBFDF91CF912E
:109DF0001F910F91FF90EF90DF90CF90BF90AF90A9
:109E00009F908F907F906F905F904F903F902F909A
:109E100008952F923F924F925F926F927F928F920E
:109E20009F92AF92BF92CF92DF92EF92FF920F93E9
:109E30001F93CF93DF93EC0149EE50E181E090E076
:109E4000FA0125913491C217D3070CF05DC09C0133
:109E500021503109220F331F220F331FD901A9517D
:109E6000BF4EFD01659174912B513F4EF901A590B4
:109E7000B490FC01EE0FFF1FEE0FFF1FE951FF4EE4
:109E8000E590F490FD01C590D490FA0105911491EC
:109E9000F90125903490072E000C880B990B0F9434
:109EA0002C172B013C01CA19DB09BE01DD0F880B01
:109EB000990B0F942C174B015C01B7016C197D09AC
:109EC000072E000C880B990B0F942C179B01AC01EB
:109ED000C501B4010F948B176B017C01B8016219A5
:109EE0007309072E000C880B990B0F942C179B01FC
:109EF000AC01C701B6010F943B1C9B01AC01C3012F
:109F0000B2010F945F1B11C001964C5F5F4F80320E
:109F1000910509F095CFE3E6F1E165917491072E83
:109F2000000C880B990B0F942C17DF91CF911F9188
:109F30000F91FF90EF90DF90CF90BF90AF909F90E8
:109F40008F907F906F905F904F903F902F900895EB
:109F500060919E0470919F048091A0049091A1044F
:109F600008950F931F93CF93DF93CDB7DEB7289754
:109F70000FB6F894DEBF0FBECDBF60919C04709108
:109F80009D04072E000C880B990B0F942C176D83E2
:109F90007E838F83988780919E0490919F04A091E7
:109FA000A004B091A10489839A83AB83BC834EEF54
:109FB000BE016B5F7F4FCE010196A0DA60919A04DB
:109FC00070919B04072E000C880B990B0F942C1793
:109FD0006D837E838F839887809190049091910404
:109FE000A0919204B091930489839A83AB83BC833C
:109FF0004FEFBE016B5F7F4FCE0101967FDAE3EF3B
:10A00000F1E184918F010F5F1F4F882321F00F949E
:10A010009602F801F6CFE0919404F0E0E050FB4F97
:10A02000608170E080E090E00E94EAA5EEEEF1E150
:10A0300084918F010F5F1F4F882321F00F949602A8
:10A04000F801F6CF6091010570E080E090E00E9499
:10A05000EAA528960FB6F894DEBF0FBECDBFDF91FC
:10A06000CF911F910F9108951F920F920FB60F92EB
:10A0700011240BB60F92EF92FF920F931F932F9321
:10A080003F934F935F936F937F938F939F93AF9380
:10A09000BF93CF93DF93EF93FF9380919210811141
:10A0A00090C181E08093921080916E008B7F8093AD
:10A0B0006E00789480910F028F37E0F08F57909167
:10A0C00000059093FF042FB7992329F0F8949091FD
:10A0D0000201906404C0F894909102019F7B9093D8
:10A0E00002012FBF909101059093FE04992391F0F6
:10A0F000759A11C09091FF04891740F02FB7F8941A
:10A10000909102019F7B909302012FBF9091FE04DA
:10A11000891708F075988F5F80930F029091FD0466
:10A1200081E089278093FD0481110E9484458091FC
:10A130000E02823079F1A0F4882341F1813009F0D8
:10A1400042C080917800909179002091F204309182
:10A15000F304820F931F9093F3048093F20433C0AF
:10A16000833019F1843079F58091FC04811103C0AA
:10A1700086E08093FC048091FC0481508093FC0471
:10A18000882309F183E080930E021DC010927B00AA
:10A1900080E403C010927B0082E480937C00809175
:10A1A0007A00806480937A000EC08091780090914C
:10A1B00079002091F0043091F104820F931F909365
:10A1C000F1048093F004C0910E02C11169C0809126
:10A1D0000D028F5F80311CF480930D0261C01092DC
:10A1E0000D028091EF04811113C08091F2049091CF
:10A1F000F3049093EE048093ED048091F004909129
:10A20000F1049093EC048093EB0481E08093EF04DD
:10A210008AE0E2EFF4E0DF011D928A95E9F71092FF
:10A22000F1041092F0040091ED041091EE041195E8
:10A2300001951109D1E080910005811101C0D0E0A4
:10A24000809161089091620891958195910980179C
:10A2500091070CF48AC0809121029091220291957D
:10A2600081959109081719070CF48AC011E08091B3
:10A270000105811101C010E0E090EB04F090EC04C6
:10A2800080915F08909160088E159F050CF083C047
:10A2900080911F0290912002E816F9060CF086C00A
:10A2A000CF5FC53018F4C0930E0202C010920E02A8
:10A2B00020E030E0ABE0B0E0C901880F991FFC015D
:10A2C000EA5DFB4F408151814115510509F43EC0C3
:10A2D000F894223041F56091090164701598EFB748
:10A2E000141615062CF4F89470910B01746004C0D8
:10A2F000F89470910B017B7F70930B01EFBF429A32
:10A30000FD013197F1F742987FB7662329F0F89461
:10A3100060910B01646004C0F89460910B016B7F45
:10A3200060930B017FBF7894FC01EA5DFB4F14162C
:10A3300015063CF4408151814150510951834083BD
:10A3400005C0808191810196918380832F5F3F4F6B
:10A350002330310509F0B0CFF8941092921080911B
:10A360006E00846080936E002CC0DD2309F473CFEF
:10A370004BED51E169EB71E180E00E94F35F6BCF3F
:10A38000DD2309F473CF48E951E166E771E180E02C
:10A390000E94F35F6BCF112309F47ACF48EA51E1B1
:10A3A00069EB71E18FEF0E94F35F72CF112309F423
:10A3B00077CF45E651E166E771E18FEF0E94F35FE9
:10A3C0006FCFFF91EF91DF91CF91BF91AF919F91AF
:10A3D0008F917F916F915F914F913F912F911F913D
:10A3E0000F91FF90EF900F900BBE0F900FBE0F904C
:10A3F0001F901895CF92DF92EF92FF92C090900439
:10A40000D0909104E0909204F090930480919A048B
:10A4100090919B040897BC01990F880B990B0F949E
:10A420002C179B01AC01C701B6010F94261787FFBB
:10A430001FC020E030E040E050E4C701B6010F94B7
:10A440005F1B0F94A81C7093EA046093E9040E94B8
:10A4500007D0DC01CB01805A9541AF4FBF4F8093AD
:10A46000E5049093E604A093E704B093E80408C0E1
:10A470001092E5041092E6041092E7041092E804AA
:10A48000FF90EF90DF90CF900895CF92DF92EF9200
:10A49000FF92C0909E04D0909F04E090A004F090A2
:10A4A000A10480919C0490919D044597BC01990F53
:10A4B000880B990B0F942C179B01AC01C701B601B7
:10A4C0000F94261787FF1FC020E030E040E251E4E0
:10A4D000C701B6010F945F1B0F94A81C7093E4048E
:10A4E0006093E3040E9407D0DC01CB01805C9346BB
:10A4F000AF4FBF4F8093DF049093E004A093E1043B
:10A50000B093E20408C01092DF041092E0041092AD
:10A51000E1041092E204FF90EF90DF90CF90089555
:10A5200010929D0410929C0480E0AFDF10929B0477
:10A5300010929A045FDF0E9483B210929D041092E1
:10A540009C0480E0A2DF109200059FB7F894E2E03F
:10A55000F1E080818F7B80839FBF10929B041092DB
:10A560009A04109201057598089560E08091ED04B9
:10A570009091EE044EDC60939E0470939F04809350
:10A58000A0049093A1048091EB049091EC040E94AC
:10A59000545F60939004709391048093920490931D
:10A5A0009304A8958FB7F8941092EF048FBF089585
:10A5B00090916905E92FF0E0EA59F74F80839F5F9A
:10A5C000953018F49093690502C010926905809146
:10A5D000680A8F5F8093680A0895EF920F931F9324
:10A5E000CF93DF93CDB7DEB72C970FB6F894DEBFCD
:10A5F0000FBECDBFE0907C14EAEAF4E1808591853E
:10A60000A285B3854481558166817781008111815E
:10A610002281338109831A832B833C834D835E839C
:10A620006F83788789879A87AB87BC87AE01475F3E
:10A630005F4FBE016B5F7F4FCE0101960E94FFA46A
:10A6400009E912E026EB34E1AE01475F5F4FBE013E
:10A650006B5F7F4FCE0101960E94B7A22C960FB67A
:10A66000F894DEBF0FBECDBFDF91CF911F910F9148
:10A67000EF900895CF93DF93CDB7DEB727970FB64E
:10A68000F894DEBF0FBECDBF0E94D3F381113BC053
:10A6900080E50E94FF44882319F00E94784401C09D
:10A6A00060E06F8383E50E94FF44882319F00E94D5
:10A6B000784401C06CE06E8384E50E94FF448823E7
:10A6C00019F00E94784401C063E06D8382E50E9426
:10A6D000FF44882319F00E94994404C060E070E0B0
:10A6E00080ED90E469837A838B839C839E012B5F4A
:10A6F0003F4FAE014F5F5F4FBE016A5F7F4FCE019C
:10A7000007960F94A90E27960FB6F894DEBF0FBEDA
:10A71000CDBFDF91CF9108954F925F926F927F925C
:10A72000AF92BF92CF92DF92EF92FF920F931F935F
:10A73000CF93DF9385E1A82E83E0B82E9CE6E92E27
:10A7400094E1F92E0AEA14E12DE7C22E24E1D22E7B
:10A75000C0E0D0E0F50181915F010E94D0448823E0
:10A7600071F10E949944FE01E055FB4F20812111B7
:10A7700004C02091B404222331F0F80120813181FA
:10A780004281538103C020E030E0A9010F945F1B98
:10A79000C330D10559F0F6012081318142815381C6
:10A7A0002B013C01C301B2010F945E1B462F572FB2
:10A7B000BC01F70140835183628373830AC0F801AF
:10A7C00080819181A281B381F70180839183A283EB
:10A7D000B3832196F4E0EF0EF11C0C5F1F4F84E071
:10A7E000C80ED11CC430D10509F0B4CF86E40E9454
:10A7F000FF448823C9F00E94994420E030E0A90179
:10A800000F94851D181684F40E94994420E030E0CE
:10A8100040E752E40F943B1C6093990270939A02B4
:10A8200080939B0290939C02DF91CF911F910F9197
:10A83000FF90EF90DF90CF90BF90AF907F906F90A0
:10A840005F904F90089580916E0590916F05A09153
:10A850007005B09171058093990290939A02A0932C
:10A860009B02B0939C0280916C0590916D05909332
:10A870009402809393020C944A9180919902909152
:10A880009A02A0919B02B0919C0280936E059093D6
:10A890006F05A0937005B09371058091930290911C
:10A8A000940290936D0580936C0584E690E09093FC
:10A8B0009402809393020C944A912F923F924F926C
:10A8C0005F926F927F928F929F92AF92BF92CF9240
:10A8D000DF92EF92FF920F931F93CF93DF9300D0FD
:10A8E0001F92CDB7DEB71C017A8369835C834B83EB
:10A8F00089018090990290909A02A0909B02B0905A
:10A900009C02F901C080D180E280F38020E030E039
:10A91000A901C701B6010F942617811106C0E0E115
:10A92000F3E2C590D590E590F490EB81FC81208115
:10A930003181428153816091B2147091B31480913E
:10A94000B4149091B5140F94261787FF17C0C092C6
:10A950009902D0929A02E0929B02F0929C02EB81C3
:10A96000FC8180819181A281B3818093B214909304
:10A97000B314A093B414B093B5142FDEF801408043
:10A9800051806280738020E030E0A901C301B201F0
:10A990000F942617811108C040909502509096029E
:10A9A00060909702709098024092990250929A0299
:10A9B00060929B0270929C02F10180819181A28140
:10A9C000B3818093AA149093AB14A093AC14B0936A
:10A9D000AD14E981FA8180819181A281B381809354
:10A9E000AE149093AF14A093B014B093B114F5DDEE
:10A9F000EB81FC8120813181428153816091B214CD
:10AA00007091B3148091B4149091B5140F94851D76
:10AA10001816BCF4C0929902D0929A02E0929B025E
:10AA2000F0929C02EB81FC8180819181A281B381B3
:10AA30008093B2149093B314A093B414B093B5144C
:10AA4000CCDD0E9425A78092990290929A02A09252
:10AA50009B02B0929C020F900F900F900F90DF918D
:10AA6000CF911F910F91FF90EF90DF90CF90BF900B
:10AA7000AF909F908F907F906F905F904F903F909E
:10AA80002F9008951F93CF93DF93CDB7DEB72C9708
:10AA90000FB6F894DEBF0FBECDBF9091B5049817E6
:10AAA00061F1182F0E94AFF48091AA149091AB1419
:10AAB000A091AC14B091AD1489879A87AB87BC87FD
:10AAC0008091AE149091AF14A091B014B091B114D4
:10AAD0008D839E83AF83B88719821A821B821C8262
:10AAE0009E012F5F3F4F42EB54E1BE016B5F7F4FF2
:10AAF000CE010996E2DE1093B50480E02C960FB6E5
:10AB0000F894DEBF0FBECDBFDF91CF911F910895A6
:10AB10009A0142EB54E1D1CE9B01AC016EEA74E1A3
:10AB20008AEA94E1CACEEF920F931F93CF93DF93FB
:10AB3000CDB7DEB760970FB6F894DEBF0FBECDBFBE
:10AB40006D877E878F87988BE0907C14ECE6F4E12C
:10AB500080859185A285B385448155816681778101
:10AB6000008111812281338109831A832B833C83E5
:10AB70004D835E836F83788789879A87AB87BC878D
:10AB8000AE01475F5F4FBE016B5F7F4FCE01019605
:10AB90000E94FFA48E01035F1F4F28E734E1AE013E
:10ABA000475F5F4FBE016B5F7F4FCE0101960E94F2
:10ABB000B7A260960FB6F894DEBF0FBECDBFDF918F
:10ABC000CF911F910F91EF9008950F931F93CF9303
:10ABD000DF9394E08902E00111248E0103581B4E9B
:10ABE000FE01E45DFB4FDE01AE5AB74F2D913D9162
:10ABF0004D915C9160817181828193810F945F1B83
:10AC0000F8016083718382839383FE01ED5BFC4EC8
:10AC100085919591A591B491FE01E25BFB4E8083F5
:10AC20009183A283B383FE01E15BFC4E85919591F4
:10AC3000A591B491CE5EDD4F88839983AA83BB83AF
:10AC4000DF91CF911F910F910895EF92FF920F9393
:10AC50001F93CF93DF937C0184E50E94FF44D82F9C
:10AC6000882349F10E948844C82F181604F5EAE3A6
:10AC7000F2E484918F010F5F1F4F882321F00F941E
:10AC80009602F801F6CF8DE40F949602B70180E0AA
:10AC900090E04AE00F94EF026C2FCC0F770B80E32B
:10ACA00093E10E94AC918AE00F94960208C08093D1
:10ACB0009404D0E004C080917C14809394048D2F80
:10ACC000DF91CF911F910F91FF90EF900895CF9357
:10ACD000FC0180818B33A1F08091680A853080F47B
:10ACE000C62FBF018091690520E6829FC001112413
:10ACF0008957974F0F949D1E8C2F5ADC81E001C01D
:10AD000080E0CF910895DF92EF92FF920F931F930F
:10AD1000CF93DF93CDB7DEB76E970FB6F894DEBF53
:10AD20000FBECDBF6091EC077091ED076115710505
:10AD300001F14DE150E0CE0101967C010F94961691
:10AD40001E8EF7018F010E191F09D190DD2019F019
:10AD50009AE0D912F7CFF701E00FF11F108260E0FF
:10AD6000C701B5DF882329F0C7010E94E382811162
:10AD700009C081E02091EC073091ED07232BA1F46D
:10AD800080E012C0DD2049F00F5F1F4F8091EC077B
:10AD90009091ED07080F191F02C000E010E010931A
:10ADA000ED070093EC07E5CF6E960FB6F894DEBF83
:10ADB0000FBECDBFDF91CF911F910F91FF90EF900C
:10ADC000DF9008954F925F926F927F928F929F9241
:10ADD000AF92BF92CF92DF92EF92FF920F931F93A9
:10ADE000CF93DF931F92CDB7DEB78DDF811158C2AD
:10ADF0008091680A853028F40F94C703AC0197FF4F
:10AE00004DC180915B11882309F44AC28091680A80
:10AE1000811102C010926B05EE24E3944091FE1361
:10AE20005091FF1360910014709101148091FA13F6
:10AE30009091FB13A091FC13B091FD134817590793
:10AE40006A077B0708F4E12C00E010E0BB24B39410
:10AE500080E6A82E94E6992E29E0C22E23E1D22E78
:10AE60003DE8832E8091680A853008F019C2E11010
:10AE700017C280916B05811113C280915513909177
:10AE80005613A0915713B09158138093FE139093CB
:10AE9000FF13A0930014B093011441E050E0BE01F1
:10AEA0006F5F7F4F8DE493E10F940207019719F4D0
:10AEB000898190E002C08FEF9FEFF82EEE24E3949B
:10AEC0004090FE135090FF13609000147090011496
:10AED0004091FA135091FB136091FC137091FD1394
:10AEE0004416550666067706C8F4E12C8F3FFFEF3F
:10AEF0009F0709F481C02AE0821709F4A2C08DE0FF
:10AF0000F81609F49EC093E2F91619F0EAE3FE126E
:10AF1000ABC080916A058111A7C088C00E9425A797
:10AF20008DE493E10E94064B80916813882359F1C8
:10AF3000815080936813889EC001112441E061E034
:10AF400083599C4E0E947E6EE091681324E0E29F3C
:10AF5000F0011124E759FC4E4081518162817381D7
:10AF60004093FE135093FF136093001470930114E9
:10AF70008DE493E10F94ED0480915C118823D9F066
:10AF8000B0925B1118C010925B1181E090E0909339
:10AF90009E1080939D100E9483B20E9498B26D33E0
:10AFA00071058105910528F0D092ED07C092EC075C
:10AFB000AADE9092A20480915B1181113BC0ECE16A
:10AFC000F3E184913F019FEF691A790A882321F008
:10AFD0000F949602F301F5CF1092061480915C1144
:10AFE000882319F00E94127121C00E94C3718091C0
:10AFF0005C118111F7CF1AC0E9E7F8E184913F01B4
:10B000002FEF621A720A882321F00F949602F3013F
:10B01000F5CFEDE0F3E184913F019FEF691A790AE2
:10B02000882321F00F949602F301F5CFE3E2FE129C
:10B0300008C005C023E2F2122EC100E010E0B09279
:10B040006B0510926A050115110509F40BCF80916B
:10B050006905A89E000D111D1124F801E957F74F4D
:10B06000108280E0A5DA19C10F35110508F0FACE7B
:10B07000FBE3FF1202C0B0926A0580916A0581115C
:10B08000F1CE80916905F801A89EE00DF11D112413
:10B09000E957F74FF0820F5F1F4FE4CE982F2091B2
:10B0A000DB053091DC058A3019F09D3009F0C1C014
:10B0B000109268052115310509F49ACEF901E85F6F
:10B0C000FA4F10821092DC051092DB0528E035E083
:10B0D0008901F90180812F5F3F4F8032C9F37801E8
:10B0E0008E3409F07BC00115110509F477C064E0C6
:10B0F00073E1C8010F94A516DD24D394892B11F4B4
:10B10000D12C09C06EE470E0C80104960F94921E21
:10B11000009709F08C014AE050E060E070E0C8015F
:10B1200001960F941A14609304057093050580939B
:10B130000605909307050091DD051091DE0520912D
:10B14000DF053091E0050F5F1F4F2F4F3F4F601716
:10B1500071078207930729F0D11003C087E092E1BD
:10B1600027C06AE270E0C7010F94C11E9C010097DE
:10B1700011F1982F9E1910E0992339F09150F701A1
:10B18000E90FF11D80811827F7CF4AE050E060E019
:10B1900070E0C90101960F941A14012F10E020E00D
:10B1A00030E0601771078207930741F085EE92E166
:10B1B0000E940A7326CE8BEB92E1FACF80910405B0
:10B1C00090910505A0910605B09107058093DD05D6
:10B1D0009093DE05A093DF05B093E00580910B020C
:10B1E000811122C067E470E0C7010F94921E00979E
:10B1F000D9F04AE050E060E070E001960F941A1434
:10B200006430710588F4E4E4F2E184918F010F5F0A
:10B210001F4F882321F00F949602F801F6CF60E0CB
:10B220008AE392E10E94F94561E088E095E04FDD14
:10B23000DFCD2F3531050CF0DBCD9C35C1F40F94FB
:10B24000C70397FDD5CD209168052111D1CD20915F
:10B25000DB053091DC05A9014F5F5F4F5093DC05A2
:10B260004093DB05F901E85FFA4F8083C1CD9B3342
:10B2700019F481E080936805809168058111B8CD4B
:10B28000C90101969093DC058093DB05F901E85F25
:10B29000FA4F4083ADCD10926A0500E010E0E2CD98
:10B2A0000F90DF91CF911F910F91FF90EF90DF9062
:10B2B000CF90BF90AF909F908F907F906F905F9056
:10B2C0004F9008950C9471F40F931F93CF93DF93D5
:10B2D000CDB7DEB72C970FB6F894DEBF0FBECDBF4B
:10B2E000EAEAF4E180859185A285B38544815581A0
:10B2F00066817781008111812281338109831A83DC
:10B300002B833C834D835E836F83788789879A87FD
:10B31000AB87BC87AE01475F5F4FBE016B5F7F4F5E
:10B32000CE0101960E94FFA426EB34E1AE01475FF7
:10B330005F4FBE016B5F7F4FCE0101960E94F5A16A
:10B340002C960FB6F894DEBF0FBECDBFDF91CF9124
:10B350001F910F9108958F929F92BF92CF92DF928B
:10B36000EF92FF920F931F93CF93DF93CDB7DEB78A
:10B3700064970FB6F894DEBF0FBECDBFB02EC12EBE
:10B38000D22EF32E94E0890280011124F801E655B3
:10B39000FB4E4F011082118212821382498B5A8B0D
:10B3A0006B8B7C8B91DF49895A896B897C89F4018D
:10B3B0004083518362837383E0907C1420E030E00B
:10B3C000A9016B2D7C2D8D2D9F2D0F94261781119A
:10B3D00008C0F801E85FFC4D85919591A591B49165
:10B3E00004C08B2D9C2DAD2DBF2D8D879E87AF87E3
:10B3F000B88B8091B2149091B314A091B414B09111
:10B40000B5144091AE145091AF146091B014709186
:10B41000B1140091AA141091AB142091AC14309186
:10B42000AD1409831A832B833C834D835E836F8322
:10B43000788789879A87AB87BC87AE01475F5F4F64
:10B44000BE016B5F7F4FCE0101960E94FFA48E016B
:10B45000035F1F4F26EB34E1AE01475F5F4FBE0134
:10B460006B5F7F4FCE0101960E94B7A20E9425A775
:10B470001092951464960FB6F894DEBF0FBECDBF40
:10B48000DF91CF911F910F91FF90EF90DF90CF90C0
:10B49000BF909F908F90089590910C04891791F020
:10B4A00080930C04811109C00E94968589E894E17B
:10B4B0000E94E1A30E940F6404C08AEA94E10E9402
:10B4C000E1A302CF08952F923F924F925F926F9225
:10B4D0007F928F929F92AF92BF92CF92DF92EF9224
:10B4E000FF920F931F93CF93DF93CDB7DEB7629791
:10B4F0000FB6F894DEBF0FBECDBF082F11E010933A
:10B50000B50424982C9A0898109A0E9425A7209197
:10B510000C04298B80E0C0DFB0D910934D140111C9
:10B5200019C088E50E94D044382E89E50E94D04495
:10B53000182F8AE50E94D044282E311006C0111120
:10B5400013C0882369F0312E10C0112369F0312E09
:10B55000082F0BC03324339411E02224239402C01B
:10B56000382E182F01E001C000E00E94194501119A
:10B5700005C0311003C0112309F409C180E090E037
:10B58000A0EAB0E48093741490937514A093761499
:10B59000B09377149C01AD016091B2147091B31413
:10B5A0008091B4149091B5140F94261787FF0AC0A8
:10B5B00019821A821B821C82BE016F5F7F4F84E753
:10B5C00094E1AADA01110CC0332009F48DC11111E4
:10B5D00007C080E00E940482002309F485C1CCC02A
:10B5E0001092AE141092AF141092B0141092B114C5
:10B5F0001092AA141092AB141092AC141092AD14C5
:10B6000063DEE3EDF2E084918A8BE9E4F3E2C59036
:10B61000D590E590F490EDE4F3E285909590A590B7
:10B62000B490A5019401C701B6010F94851D1816A9
:10B630002CF4A7019601C501B40104C0A501940131
:10B64000C701B6010F943B1C6D877E878F87988B4F
:10B6500088E0682E83E2782EF301659175918591DB
:10B6600094912CE0422E23E2522EF2012591359145
:10B67000459154910F94261787FF02C0F30101C032
:10B68000F20145905590659074902D853E854F85CB
:10B690005889CA01B9010F948B1720E030E040E8C7
:10B6A0005FE30F945F1B0F94CA1D9B01AC01C301A4
:10B6B000B2010F948B1769877A878B879C87E4ED9B
:10B6C000F2E094919D8720E030E040EC5FE3C5011B
:10B6D000B4010F948B172B013C012D85622F220F93
:10B6E000770B880B990B0F942C179B01AC01C301AE
:10B6F000B2010F948B1769837A838B839C8320E03C
:10B7000030E040EC5FE3C701B6010F948B176B018B
:10B710007C012A89622F220F770B880B990B0F94DB
:10B720002C179B01AC01C701B6010F948B176D83D9
:10B730007E838F839887AE01475F5F4FBE016F5F47
:10B740007F4FCE010596E4D9109295141092AE1455
:10B750001092AF141092B0141092B1141092AA1457
:10B760001092AB141092AC141092AD14011131CFA1
:10B7700031102FCF112359F081E00E940482002361
:10B7800009F4B8C080918D04811104C007C0211054
:10B79000F9CF5BC080918E0481111FC060E08AE602
:10B7A00093E10E94F945EAE3F2E484917F019FEF7F
:10B7B000E91AF90A882321F00F949602F701F5CFD0
:10B7C000EBE5F3E184917F012FEFE21AF20A88237F
:10B7D000E1F10F949602F701F5CF76DD80E090E07D
:10B7E000A8E9B1EC80936C1490936D14A0936E143F
:10B7F000B0936F1480E090E0A1E8B3E480937014FC
:10B8000090937114A0937214B09373148091B21436
:10B810009091B314A091B414B091B51480937414A2
:10B8200090937514A0937614B093771419821A82AA
:10B830001B821C82AE014F5F5F4F60E774E18CE6B4
:10B8400094E166D982E00E9404823EDD0023F1F09B
:10B850000E9425A71092B2141092B3141092B4143F
:10B860001092B51431DD1D821E821F82188680E081
:10B8700090E0A0E2B1E489839A83AB83BC83BE01EC
:10B880006B5F7F4FCE01019647D902C02110E0CFF8
:10B8900080914C1480934D148989FEDD0E942354BD
:10B8A00083E080933D020E94CFC71092B504249A92
:10B8B0002C98089A109862960FB6F894DEBF0FBEC7
:10B8C000CDBFDF91CF911F910F91FF90EF90DF904F
:10B8D000CF90BF90AF909F908F907F906F905F9030
:10B8E0004F903F902F900895112309F450CF81E09D
:10B8F0000E940482211046CFE7DCCACF80E0CCDD75
:10B90000E4EBF0E180E090E0A0E8BFE38083918386
:10B91000A283B38314821582168217821086118641
:10B92000128613861486158616861786808B918B51
:10B93000A28BB38B148A158A168A178A108E118EE1
:10B94000128E138E148E158E168E178E80A391A3D1
:10B95000A2A3B3A308958091020590910305892BBA
:10B9600039F00E94884491E0811103C090E001C049
:10B9700091E0892F08954F925F926F927F928F92FC
:10B980009F92AF92BF92CF92DF92EF92FF92CF93AE
:10B99000DF93CDB7DEB72C970FB6F894DEBF0FBE9E
:10B9A000CDBF8091900490919104A0919204B091A8
:10B9B000930489839A83AB83BC8360919A047091CA
:10B9C0009B04072E000C880B990B0F942C172981D0
:10B9D0003A814B815C810F945E1B6B017C0160930B
:10B9E000B1057093B2058093B3059093B40520918F
:10B9F00016043091170440911804509119040F94C3
:10BA00008B176D837E838F8398876093AD057093CA
:10BA1000AE058093AF059093B0052091A9053091B4
:10BA2000AA054091AB055091AC05C701B6010F9432
:10BA30005F1B4B015C016093A9057093AA0580937D
:10BA4000AB059093AC052091120430911304409102
:10BA50001404509115040F948B1769877A878B878C
:10BA60009C876093A5057093A6058093A705909386
:10BA7000A80520ED3CEC4CE45DE360910E04709170
:10BA80000F0480911004909111040F948B172B01D7
:10BA90003C012091A1053091A2054091A305509150
:10BAA000A40569817A818B819C810F945E1B9B0127
:10BAB000AC01C301B2010F948B172B013C0123E3AE
:10BAC00033E343E75FE360919D0570919E058091AC
:10BAD0009F059091A0050F948B179B01AC01C301AA
:10BAE000B2010F945F1B2B013C0160939D05709385
:10BAF0009E0580939F059093A00589819A81AB81D3
:10BB0000BC818093A1059093A205A093A305B09357
:10BB1000A40529853A854B855C856D817E818F8161
:10BB200098850F945F1BA30192010F945E1B2B015C
:10BB30003C0120E030E04EE453E40F94851D20E00A
:10BB400030E0A9011816ACF4C701B6010F94851DA9
:10BB500018166CF5A7019601C501B4010F945E1B80
:10BB60006093A9057093AA058093AB059093AC05EB
:10BB70001EC0C301B2010F94261787FF22C020E028
:10BB800030E0A901C701B6010F94261787FF16C040
:10BB9000A7019601C501B4010F945E1B6093A9052E
:10BBA0007093AA058093AB059093AC0507C0412C18
:10BBB000512C8EE4682E83E4782E03C0412C512C46
:10BBC0003201C301B2012C960FB6F894DEBF0FBE4E
:10BBD000CDBFDF91CF91FF90EF90DF90CF90BF90DE
:10BBE000AF909F908F907F906F905F904F9008954F
:10BBF0002F923F924F925F926F927F928F929F927D
:10BC0000AF92BF92CF92DF92EF92FF92CF93DF93EA
:10BC100000D01F92CDB7DEB760909C0470909D0459
:10BC200080909E0490909F04A090A004B090A104E6
:10BC3000B301072C000C880B990B0F942C17A5014E
:10BC400094010F945E1B6B017C01609399057093C6
:10BC50009A0580939B0590939C0520ED3CEC4CE469
:10BC60005DE360911A0470911B0480911C04909113
:10BC70001D040F948B171B012C0120919505309109
:10BC800096054091970550919805C501B4010F9410
:10BC90005E1B9B01AC01C201B1010F948B171B010C
:10BCA0002C0123E333E343E75FE360919105709157
:10BCB000920580919305909194050F948B179B01A9
:10BCC000AC01C201B1010F945F1B69837A838B833E
:10BCD0009C83609391057093920580939305909354
:10BCE00094058092950590929605A0929705B09242
:10BCF00098058091AA10882321F081E08093900517
:10BD0000B9C020E030E040E251E4C701B6010F9431
:10BD1000851D181624F481E080939005A4C020E0CE
:10BD200030E040E251ECC701B6010F94261787FDC1
:10BD3000E4CF672811F380919005882351F0109289
:10BD40008C0510928D0510928E0510928F05109221
:10BD500090052091220430912304409124045091B5
:10BD60002504C701B6010F948B172B013C0160938A
:10BD700088057093890580938A0590938B0520919F
:10BD80008C0530918D0540918E0550918F05C7012E
:10BD9000B6010F945F1B4B015C0160938C0570939F
:10BDA0008D0580938E0590938F0520911E04309110
:10BDB0001F0440912004509121040F948B179B0184
:10BDC000AC016093840570938505809386059093FC
:10BDD0008705C301B2010F945F1B29813A814B8112
:10BDE0005C810F945E1B2B013C0120E030E04FE7AB
:10BDF00053E40F94851D20E030E0A9011816ACF43F
:10BE0000C701B6010F94851D18166CF5A7019601A0
:10BE1000C501B4010F945E1B60938C0570938D0572
:10BE200080938E0590938F051EC0C301B2010F94BD
:10BE3000261787FF22C020E030E0A901C701B60124
:10BE40000F94261787FF16C0A7019601C501B401FC
:10BE50000F945E1B60938C0570938D0580938E0507
:10BE600090938F0507C0412C512C8FE7682E83E4F7
:10BE7000782E03C0412C512C3201C301B2010F9026
:10BE80000F900F900F90DF91CF91FF90EF90DF9088
:10BE9000CF90BF90AF909F908F907F906F905F906A
:10BEA0004F903F902F9008952F923F924F925F9224
:10BEB0006F927F928F929F92AF92BF92CF92DF92BA
:10BEC000EF92FF920F931F93CF93DF93EC014CE11E
:10BED00054E181E090E0FA0125913491C217D30733
:10BEE0000CF05DC09C0121503109220F331F220F3D
:10BEF000331FD901A65EBB4EFD0165917491285E8A
:10BF00003B4EF901A590B490FC01EE0FFF1FEE0F20
:10BF1000FF1FE65EFB4EE590F490FD01C590D490C6
:10BF2000FA0105911491F90125903490072E000C27
:10BF3000880B990B0F942C172B013C01CA19DB09B4
:10BF4000BE01DD0F880B990B0F942C174B015C0180
:10BF5000B7016C197D09072E000C880B990B0F9403
:10BF60002C179B01AC01C501B4010F948B176B0119
:10BF70007C01B80162197309072E000C880B990B1C
:10BF80000F942C179B01AC01C701B6010F943B1C09
:10BF90009B01AC01C301B2010F945F1B11C001965C
:10BFA0004C5F5F4F8A33910509F095CFEEEFF4E1D6
:10BFB00065917491072E000C880B990B0F942C1728
:10BFC000DF91CF911F910F91FF90EF90DF90CF9075
:10BFD000BF90AF909F908F907F906F905F904F90A9
:10BFE0003F902F900895CF92DF92FF920F931F936F
:10BFF000CF93DF931F921F92CDB7DEB7F82E8A0141
:10C0000080910B02882309F444C0E9E7F8E18491A8
:10C010006F019FEFC91AD90A882341F069837A8397
:10C020000F949602F60169817A81F1CFFB01849128
:10C030006F019FEFC91AD90A882321F00F94960245
:10C04000F601F5CFE7EBF3E184916F019FEFC91A99
:10C05000D90A882321F00F949602F601F5CFF7FC58
:10C060000BC06F2DFF0C770B880B990B0E94EAA574
:10C070008AE00F9496020DC0E2EBF3E184916F0128
:10C080009FEFC91AD90A882321F00F949602F6016E
:10C09000F5CF80918305811108C010920B0281E0D9
:10C0A00080938305C8010E9454830F900F90DF9105
:10C0B000CF911F910F91FF90DF90CF900C949052F1
:10C0C0008F3F29F0882331F048E851E105C045E66B
:10C0D00051E102C048E951E166E771E184CF8F3F49
:10C0E00029F0882331F04BEC51E105C048EA51E1D9
:10C0F00002C04BED51E169EB71E175CF4F925F9258
:10C100006F927F92AF92BF92CF92DF92EF92FF92A7
:10C110000F931F93CF93DF9300D01F92CDB7DEB75D
:10C120008091EF04811113C00F900F900F900F902A
:10C13000DF91CF911F910F91FF90EF90DF90CF9003
:10C14000BF90AF907F906F905F904F9008950E9446
:10C15000B5520E9407D069837A838B839C83809138
:10C16000100290911102181619060CF026C10197C1
:10C17000909311028093100240909E0450909F046F
:10C180006090A0047090A1048091AA10811119C040
:10C190008091070490910804A0910904B0910A04C9
:10C1A0000097A105B10569F029813A814B815C8135
:10C1B000281B390B4A0B5B0B57FD03C081E08093B2
:10C1C000AA1060919C0470919D04072E000C880BAE
:10C1D000990B0F942C17AEE1AA2EB12CC12C7B0128
:10C1E0008C01A30192016BEB75E08AEB95E00E9454
:10C1F00087B3C0909E04D0909F04E090A004F0907C
:10C20000A1048091630890916408BC01990F880B88
:10C21000990B0F942C179B01AC01C701B6010F9429
:10C22000851D1816CCF46091230270912402072E0C
:10C23000000C880B990B0F942C179B01AC01C701C4
:10C24000B6010F94261787FF07C080E0D1DC0F945A
:10C25000A31C7595679501C060E06093000580910F
:10C26000DF049091E004A091E104B091E204009712
:10C27000A105B10529F129813A814B815C81281BF7
:10C28000390B4A0B5B0B57FD1BC00E94A84F6B017B
:10C290007C018091E3049091E404BC0180E090E093
:10C2A0000F942A179B01AC01C701B6010F94261702
:10C2B00087FFA5C046E054E167EF73E180E093DEBD
:10C2C0008091E5049091E604A091E704B091E80420
:10C2D0000097A105B10529F149805A806B807C80C7
:10C2E000481A590A6A0A7B0A77FC1BC00E944191CE
:10C2F0006B017C018091E9049091EA04BC0180E02B
:10C3000090E00F942A179B01AC01C701B6010F946E
:10C31000261787FF71C045ED53E168EE73E18FEF9B
:10C3200062DE60919A0470919B04072E000C880BCA
:10C33000990B0F942C172091900430919104409107
:10C34000920450919304EAE0AE2EB12CCC24CA940E
:10C350007B018C0165EB75E089EB95E00E9487B36A
:10C360008091A110811126C0C0909004D0909104BA
:10C37000E0909204F090930420E030E040EA50E432
:10C38000C701B6010F94851D87FF04C060E060936C
:10C390000105CACE20E030E046E153E4C701B60112
:10C3A0000F942617181694F3E6DA0F94A31C7595CC
:10C3B0006795EDCF10920105B7CE40909E04509046
:10C3C0009F046090A0047090A10420E030E848E948
:10C3D00053E4C301B2010F94851D1816A4F020E0A8
:10C3E00030E040EA50E4C301B2010F94261787FF02
:10C3F000CBCE80E065DEC0CE0E94FA5192CF80E0C5
:10C400000E9445525DCF80E06ADE40909E045090CD
:10C410009F046090A0047090A104E1CF8F929F923E
:10C42000AF92BF92CF92DF92EF92FF920F931F9342
:10C43000CF93DF931F92CDB7DEB75C014B016A014A
:10C44000122FEDEAF5E084917F019FEFE91AF90AD6
:10C45000882321F00F949602F701F5CF8091AF0465
:10C4600083FD36C020E030E0A901F60160817181D2
:10C47000828193810F942617882351F1F0900D0447
:10C48000F11024C020919C0430919D048091000201
:10C490009091010228173907CCF4E9E7F8E184917B
:10C4A0008F010F5F1F4F882321F00F949602F80130
:10C4B000F6CFE9E8F3E184918F010F5F1F4F8823E6
:10C4C00009F493C00F949602F801F5CF0F94D6119A
:10C4D00091E09093A70480915B11882321F0109242
:10C4E0005B11909382050E946EB2002339F081E0C7
:10C4F0008093AE1085E99DE70E9464B30E9425A752
:10C5000090E1EAEAF4E1A2E7B5E001900D929A9594
:10C51000E1F720E030E0A901F501608171818281BD
:10C5200093810F942617882329F00E94048388237F
:10C5300009F453C082E08983B401CE0101960F94BF
:10C54000130E20E030E0A901F60160817181828143
:10C5500093810F942617882399F0002351F081E0EE
:10C560008093AE108FE39DE70E9464B380E00E9449
:10C57000BC8340E050E060E271E4C6010F949F117B
:10C58000002339F081E08093AE108DE39CE70E9498
:10C5900064B361E0812F0F94311280E00E94BC836C
:10C5A0000E94498364E670E080E090E00E9409E622
:10C5B0000E9407D0DC01CB0188539045AF4FBF4F9D
:10C5C0008093070490930804A0930904B0930A048D
:10C5D0001092AA10FF24F39408C040E050E060E7F6
:10C5E00072E4C5010F949F11A5CF8F2D0F90DF919D
:10C5F000CF911F910F91FF90EF90DF90CF90BF9060
:10C60000AF909F908F900895CF92DF92EF92FF921C
:10C610000F931F93CF93DF9300D01F92CDB7DEB758
:10C620007C016B01042F1091AA1010920704109244
:10C6300008041092090410920A041092AA1080E0D3
:10C640000E94455211110F94D61161E0802F0F9472
:10C6500031120E94194520E030E0A901F701608104
:10C660007181828193810F942617882341F11123D0
:10C6700039F081E08093AE108DE39CE70E9464B3B3
:10C6800081E08093A8048091A804882351F01123AD
:10C6900041F060E0802F0F94311281E00E94BC8352
:10C6A000F2CF81E08093AE1087EE9BE70E9464B3E7
:10C6B00040E050E060EC70E4C7010F949F110E94CD
:10C6C0000483811141C0F60180819181A281B381EF
:10C6D00089839A83AB83BC8311E0C12CD12C80EA7F
:10C6E000E82E81E4F82E20E030E0A90169817A810A
:10C6F0008B819C810F94851D181674F41093AE10D5
:10C7000081E99BE70E9464B340E050E060E87FE38A
:10C71000CE0101960F949F111092A8041093AE10B1
:10C72000109206048BEE9DE70E9464B3809106048C
:10C73000811104C081E00E94BC83F8CFC982DA82F3
:10C74000EB82FC82813079F281E08093AE1082E34B
:10C7500094E40E9464B380917E0590917F05A0913E
:10C760008005B09181058093B6149093B714A0937F
:10C77000B814B093B9148093781490937914A0935B
:10C780007A14B0937B140E9471F480E090E0A8ECDE
:10C79000B2E489839A83AB83BC83AE014F5F5F4F62
:10C7A00066E775E082E795E00E94885580E090E0BA
:10C7B000A0EAB0E489839A83AB83BC83BE016F5F38
:10C7C0007F4F8AE795E00E948C550E942A7AE8E71D
:10C7D000F3E184918F010F5F1F4F882321F00F94A5
:10C7E0009602F801F6CF80918205882349F0809166
:10C7F0005C11882319F081E080935B11109282050F
:10C800001092A7040F900F900F900F90DF91CF918F
:10C810001F910F91FF90EF90DF90CF9008958CE0E3
:10C82000E9E8F4E1AAEAB4E101900D928A95E1F712
:10C8300008956091340270913502072E000C880B28
:10C84000990B0F942C172AE037ED43E25CE30F9429
:10C850008B172091720B3091730B4091740B509198
:10C86000750B0F948B1760930702709308028093E7
:10C87000090290930A020895CF93DF9361E081E06B
:10C880000E94AB79D091BA04C0E0D1111EC0809152
:10C89000D504811106C080913D02882309F4A1C00E
:10C8A0000BC0809123088111F6CF0E94407A8091BD
:10C8B000AC10882381F39CC081E0909123089111F2
:10C8C00080E024E04BE057E189C0D13009F5809148
:10C8D000D504811106C080913D02882309F481C0EE
:10C8E0000DC0809123088130B1F78FE496E60E9455
:10C8F0009F498091AC10882371F37AC081E09091B8
:10C900002308913009F080E023E044E057E166C05D
:10C91000D23009F58091D504811106C080913D0285
:10C92000882309F45EC00DC0809123088230B1F7DE
:10C9300083E596E60E949F498091AC10882371F3AD
:10C9400057C081E090912308923009F080E023E005
:10C950004DEF56E143C0D33001F58091D5048111EC
:10C9600005C080913D028823E1F10DC0809123082C
:10C970008330B9F787E596E60E949F498091AC1015
:10C98000882379F335C081E090912308933009F032
:10C9900080E023E046EF56E121C0D43011F58091CC
:10C9A000D504811105C080913D028823D1F00DC0CE
:10C9B000809123088430B9F78BE596E60E949F4961
:10C9C0008091AC10882379F313C081E09091230803
:10C9D000943009F080E023E04DEE56E16C2F0E9488
:10C9E0003D45CF5FDF5FC53009F04FCFC093B9043D
:10C9F000DF91CF9108951F93CF93DF93182F7093FA
:10CA0000C9056093C80561E081E00E94AB79D091CF
:10CA1000BA04C0E091E0113071F1123009F454C051
:10CA200011117BC0D111A5C09923D9F09091230891
:10CA30001916BCF04091AF105091B0106091B11038
:10CA40007091B2104F5F5F4F6F4F7F4F4093AF10A9
:10CA50005093B0106093B1107093B2109F5F909399
:10CA6000230880913D02882309F40DC121E041E0B3
:10CA700066EE76E17AC0D1117CC09923D9F090910D
:10CA800023081916BCF04091AF105091B01060917E
:10CA9000B1107091B2104F5F5F4F6F4F7F4F409357
:10CAA000AF105093B0106093B1107093B2109F5FAD
:10CAB0009093230880913D02882309F4E4C021E08B
:10CAC00041E06FED76E151C0D11153C09923D9F007
:10CAD000909123081916BCF04091AF105091B010FE
:10CAE0006091B1107091B2104F5F5F4F6F4F7F4FE9
:10CAF0004093AF105093B0106093B1107093B21088
:10CB00009F5F9093230880913D02882309F4BBC066
:10CB100021E041E068ED76E128C0D1112AC09923D7
:10CB2000D9F0909123081916BCF04091AF105091A4
:10CB3000B0106091B1107091B2104F5F5F4F6F4FA6
:10CB40007F4F4093AF105093B0106093B11070932B
:10CB5000B2109F5F9093230880913D02882309F4CF
:10CB600092C021E041E06FEC76E18C2F0E947D7352
:10CB70008AC0D130F9F48091D504811106C080912A
:10CB80003D02882309F47FC00BC0809123088130C7
:10CB9000B1F70E94407A8091AC10882381F37BC06A
:10CBA00081E090912308913009F080E024E045EC89
:10CBB00056E166C0D23009F58091D504811106C0D6
:10CBC00080913D02882309F45EC00DC08091230846
:10CBD0008230B1F780E796E60E949F498091AC10C1
:10CBE000882371F358C081E090912308923009F0B6
:10CBF00080E023E04BEB56E143C0D33001F5809158
:10CC0000D504811105C080913D028823E1F10DC05A
:10CC1000809123088330B9F785E796E60E949F4903
:10CC20008091AC10882379F336C081E0909123087D
:10CC3000933009F080E023E042EB56E121C0D4308C
:10CC400011F58091D504811105C080913D028823A2
:10CC5000D1F00DC0809123088430B9F78AE796E6B9
:10CC60000E949F498091AC10882379F314C081E021
:10CC700090912308943009F080E023E047EA56E1E0
:10CC80006C2F0E943D45CF5FDF5F90E0C53009F01B
:10CC9000C2CEC093B904DF91CF911F91089563E88C
:10CCA00078E680E0A8CE6FE778E681E0A4CE6BE777
:10CCB00078E682E0A0CE65EB76E683E09CCE21E0CC
:10CCC0002093AE106093C4057093C5058093C6058C
:10CCD0009093C7058091C8059091C9050C9464B3E1
:10CCE00060E070E080E291E4EACF60E070E080E82C
:10CCF0009FE3E5CF6DEC7CEC8CEC9DE3E0CFCF9235
:10CD0000DF92EF92FF92CF93C82F0E9407D06B0162
:10CD10007C0124EA30E74DE75FE36091C405709140
:10CD2000C5058091C6059091C7050F94261787FD0C
:10CD300005C04AEF50E060E070E003C040E050E022
:10CD4000BA01C40ED51EE61EF71EC092C004D092D2
:10CD5000C104E092C204F092C304C0930C02CF91CC
:10CD6000FF90EF90DF90CF9008958091D5048111CE
:10CD70000C94407A6091AF107091B0108091B11016
:10CD80009091B210611571058105910569F10F94BB
:10CD90002C172091C4053091C5054091C6055091CE
:10CDA000C7050F948B179B01AC016091B61470916D
:10CDB000B7148091B8149091B9140F945F1B6093CD
:10CDC000B6147093B7148093B8149093B91483E099
:10CDD00096DF81E080933D021092AF101092B01068
:10CDE0001092B1101092B21080913D02882349F048
:10CDF00086EB94E10E9424E5BC018EE996E10C9457
:10CE0000437A08952F923F924F925F926F927F9252
:10CE10008F929F92AF92BF92CF92DF92EF92FF924A
:10CE20001F93CF93DF93CDB7DEB72A970FB6F89451
:10CE3000DEBF0FBECDBF1C01162F8091D504882305
:10CE400019F00E94407A3FC18091AF109091B010CC
:10CE5000A091B110B091B210892B8A2B8B2B09F4C1
:10CE6000A7C00E944A91A4E01A02C00111249E8327
:10CE70008D83FC01E655FB4E4080518062807380BB
:10CE800020E030E04AE754E4C301B2010F945F1B95
:10CE90006B017C0180911E02882301F1113069F041
:10CEA0001230A1F011111AC0C0901202D0901302DA
:10CEB000E0901402F090150211C0C0901602D090BC
:10CEC0001702E0901802F090190208C0C0901A02F0
:10CED000D0901B02E0901C02F0901D028091AF10D8
:10CEE0009091B010A091B110B091B2108F8398873B
:10CEF000A987BA87BC01CD010F942C172091C405D6
:10CF00003091C5054091C6055091C7050F948B1708
:10CF10009B01AC01C301B2010F945F1B4B015C018B
:10CF2000AD81BE81A655BB4EBE83AD83FD0160833E
:10CF30007183828393838F819885A985BA85B7FF92
:10CF400013C020E030E04AE754E4C301B2010F947B
:10CF50005E1B6B017C019B01AC01C501B4010F9408
:10CF6000261787FF18C010C08F819885A985BA85BC
:10CF7000892B8A2B8B2B79F0A7019601C501B4016F
:10CF80000F94851D18163CF4AD81BE81CD92DD92C3
:10CF9000ED92FC9213971092AF101092B010109275
:10CFA000B1101092B210812FAADE81E080933D0271
:10CFB00080913D02882309F486C0B4E01B02F00191
:10CFC0001124E655FB4EC080D180E280F380C982F7
:10CFD000DA82EB82FC822DEC3CEC4CEC5DE3609160
:10CFE000C4057091C5058091C6059091C7050F9441
:10CFF000851D87FD05C0CE0101960E9424E55FC016
:10D0000020E030E04AE754E4C701B6010F948B17E3
:10D010000F94A31C6B017C016115710581059105BD
:10D0200061F097FF0AC0F094E094D094C094C11CC2
:10D03000D11CE11CF11C8DE201C080E280936414DC
:10D04000C701B60128EE33E040E050E00F94231B07
:10D050008AE0882E912CA12CB12CCA01B901A5011E
:10D0600094010F94231B605D609365148EE280939E
:10D070006614C701B60124E630E040E050E00F94AA
:10D08000231BCA01B901A50194010F94231B605D04
:10D0900060936714C701B601A50194010F94231B87
:10D0A000162FCA01B901A50194010F94231B605DDD
:10D0B00060936814105D1093691484E694E1BC01D8
:10D0C000C1010E94437A2A960FB6F894DEBF0FBEC4
:10D0D000CDBFDF91CF911F91FF90EF90DF90CF9068
:10D0E000BF90AF909F908F907F906F905F904F9088
:10D0F0003F902F90089562E087E996E183CE61E04A
:10D1000080E996E17FCE60E089E896E17BCE80E021
:10D110000C9445520C94FA51FF920F931F93CF93A6
:10D12000DF9361E081E00E94AB79D091BA04C0E066
:10D13000FF24F394D1111EC08091D504811106C043
:10D1400080913D02882309F451C10BC080912308CE
:10D150008111F6CF0E94407A8091AC10882381F330
:10D160004DC181E090912308911180E024E044E8D2
:10D1700056E139C1D13071F58091D504811106C0D5
:10D1800080913D02882309F431C113C080912308A6
:10D190008130B1F727EE33E04AE050E063E972E016
:10D1A0008EE796E10E94284A8091AC10882341F3D3
:10D1B00025C111E080912308813009F010E08091B1
:10D1C0009302909194020E94D3E500E09C0148E70D
:10D1D00056E177C0D230D1F58091D504811106C0D7
:10D1E00080913D02882309F401C11FC0809123086A
:10D1F0008230B1F7F092CF041092CB041092CC049D
:10D200001092CD041092CE0407E818E622E231E035
:10D2100040E050E06CE974E081E796E10E945B74C5
:10D220008091AC108823E1F2E9C011E080912308DD
:10D23000823009F010E080919C0490919D040E943E
:10D24000D3E500E09C014AE656E13BC0D330F1F55E
:10D250008091D504811106C080913D02882309F494
:10D26000C5C01FC0809123088330B1F7F092CF046E
:10D270001092CB041092CC041092CD041092CE04E4
:10D280000AE818E627E830E040E050E06AE974E098
:10D2900086E696E10E945B748091AC108823E1F2EF
:10D2A000ADC011E080912308833009F010E0809137
:10D2B0009A0490919B040E94D3E500E09C0142E611
:10D2C00056E16C2F812F0E94077B90C0D430C1F5AE
:10D2D0008091D504811106C080913D02882309F414
:10D2E00085C01DC0809123088430B1F7F092CF042F
:10D2F0001092CB041092CC041092CD041092CE0464
:10D300002FEF30E040E050E063EA74E086E596E11C
:10D310000E94284A8091AC108823F1F26FC011E07E
:10D3200080912308843009F010E08091A30490914B
:10D33000A4040E94D3E500E09C014AE456E1C1CF79
:10D34000D53081F58091D504811106C080913D02D0
:10D35000882309F44BC015C0809123088530B1F7AC
:10D3600009E114E627EE33E04AE050E064E372E0BE
:10D3700085E496E10E945B748091AC10882331F3C0
:10D380003DC011E080912308853009F010E08091C4
:10D390003402909135020E94D3E500E09C0140E404
:10D3A00056E18FCFD63011F58091D504811105C09B
:10D3B00080913D028823D1F00DC0809123088630F2
:10D3C000B9F784E09AE60E949F498091AC108823C7
:10D3D00079F314C081E090912308963009F080E041
:10D3E00023E047E356E16C2F0E943D45CF5FDF5FAE
:10D3F000C53009F09FCE87E08093B904DF91CF91CB
:10D400001F910F91FF9008958F929F92AF92BF92BC
:10D41000CF92DF92EF92FF920F931F93CF93DF9300
:10D4200000D01F92CDB7DEB78091D504882309F4D0
:10D4300046C08091910290919202181619060CF044
:10D440003BC09A8389839E012D5F3F4F44E050E0AB
:10D4500066E974E1CE0101960E942EE1EAE3F2E46E
:10D4600084917F019FEFE91AF90A882321F00F9434
:10D470009602F701F5CF4091961450919714609160
:10D4800098147091991482E695E10E948F916091B1
:10D4900091027091920281E595E10E94AC91EFE4D6
:10D4A000F5E184917F019FEFE91AF90A882321F0C1
:10D4B0000F949602F701F5CF0E94407A69C181E08E
:10D4C0008093AE10C090AF10D090B010E090B1102B
:10D4D000F090B210C114D104E104F10409F454C075
:10D4E0001092AF101092B0101092B1101092B210B2
:10D4F000B6010D2C000C880B990B0F942C17209162
:10D5000073083091740840917508509176080F9413
:10D510008B17209196143091971440919814509144
:10D5200099140F945F1B4B015C0120E030E040E058
:10D5300050EC0F94851D87FD27C020E030E040EAC5
:10D5400050E4C501B4010F9426171816ECF0809131
:10D550000C04882371F080918F04882351F080910E
:10D560002A0490912B04C80ED91ED0922B04C0928D
:10D570002A048092961490929714A0929814B092D4
:10D58000991482E080933D0280913D02882309F442
:10D59000FFC020E030E048EC52E4609196147091B6
:10D5A000971480919814909199140F948B170F945D
:10D5B000A31C6B017C0197FD10C020E137E240E025
:10D5C00050E00F94231BCA01B9012AE030E040E08B
:10D5D00050E00F94231B605D09C0F094E094D09458
:10D5E000C094C11CD11CE11CF11C6DE26093641459
:10D5F000C701B60128EE33E040E050E00F94231B52
:10D600008AE0882E912CA12CB12CCA01B901A50168
:10D6100094010F94231B605D60936514C701B601EC
:10D6200024E630E040E050E00F94231BCA01B9012A
:10D63000A50194010F94231B605D609366148EE234
:10D6400080936714C701B601A50194010F94231BB1
:10D65000162FCA01B901A50194010F94231B605D27
:10D6600060936814105D1093691464E674E18EE2AF
:10D6700096E10E94437AC0909614D0909714E0905F
:10D680009814F09099148090C0059090C105A090D6
:10D69000C205B090C305A5019401C701B6010F945E
:10D6A0002617882301F120E030E0A901C701B60167
:10D6B0000F942617882351F0A5019401C701B601E4
:10D6C0000F94261787FD04C081E003C080E001C0ED
:10D6D0008FEF8093BF05C092C005D092C105E09244
:10D6E000C205F092C30580914614813120F48091E7
:10D6F00048148330C0F580914614853120F4809120
:10D7000048148431E0F5809146148F3308F040C00E
:10D71000809148148F32E0F103EE15E120E143E0FF
:10D720006FE285E00E9461B103EB15E120E143E087
:10D730006FE28AE50E9461B18091BF0560E3681BDA
:10D7400009E915E12DE042E08EE60E9461B1809189
:10D75000BF0561E3681B0FE715E12DE042E089E1B9
:10D760000E9461B115C08091BF0564E0681B06E1AD
:10D7700016E12CE042E082E40E9461B1BCCF03E1FB
:10D7800016E121E043E064E18CE30E9461B1BBCF8C
:10D790000F900F900F900F90DF91CF911F910F91ED
:10D7A000FF90EF90DF90CF90BF90AF909F908F90C1
:10D7B00008958091D504882321F01092AE100C9426
:10D7C0002E7A0C9440900F931F93CF93DF9361E0D8
:10D7D00081E00E94AB79D091BA04C0E000E015E18D
:10D7E000D1111EC08091D504811106C080913D02E7
:10D7F000882309F4BAC00BC0809123088111F6CFA9
:10D800000E94407A8091AC10882381F3B5C081E0FA
:10D8100090912308911180E024E04AE455E1A2C0F0
:10D82000D13009F58091D504811106C080913D0267
:10D83000882309F49AC00DC0809123088130B1F784
:10D8400088EE90E80E949F498091AC10882371F384
:10D8500093C081E090912308913009F080E023E0AB
:10D8600048E355E17FC0D23061F58091D504811144
:10D8700006C080913D02882309F477C018C08091CA
:10D8800023088230B1F70E9488ED882319F00E94A6
:10D890002D4508C048EB51E064E170E080E090E085
:10D8A0000F94FB0B8091AC10882319F365C081E0C5
:10D8B00090912308923009F080E020E248E155E1A0
:10D8C00051C0D33061F58091D504811106C080919B
:10D8D0003D02882309F449C018C080912308833091
:10D8E000B1F70E9477E8882319F00E942D4508C0FF
:10D8F00048EB51E064E170E080E090E00F94FB0BB6
:10D900008091AC10882319F337C081E090912308EF
:10D91000933009F080E020E24AE055E123C0D430A2
:10D9200021F58091D504811105C080913D028823A5
:10D93000E1F00FC0809123088430B9F71093ED0710
:10D940000093EC070E9483568091AC10882369F302
:10D9500013C081E090912308943009F080E020E228
:10D9600047E255E16C2F0E943D45CF5FDF5FC53038
:10D9700009F036CFC093B904DF91CF911F910F9179
:10D9800008954F925F926F927F928F929F92AF9283
:10D99000BF92FF920F931F93CF93DF93182F86E2CE
:10D9A00093E19093EB078093EA071092421382E091
:10D9B00090E0A0E0B0E080932B1390932C13A09301
:10D9C0002D13B0932E131092E9071092E5071092D1
:10D9D000E6071092E7071092E8078FEF9FEFDC0150
:10D9E0008093E1079093E207A093E307B093E407E5
:10D9F000112379F1153008F0F9C040E060E070E0E3
:10DA0000CB010F94640C882309F4F0C020E1129F2D
:10DA1000C00111248F529A4FFC01E254FE4F208125
:10DA20002F7709F0E3C03C96408151816281738178
:10DA3000443651056105710508F4D8C034978080DB
:10DA40009180A280B38081149104A104B10421F4D7
:10DA5000CDC0812C912C540140E0C501B4010F943C
:10DA6000640CF82E882309F4C1C08091EC059091D4
:10DA7000ED058115924009F0B9C0A091F105AA23E6
:10DA800009F4B4C06091EF057091F005611571055E
:10DA900009F4ACC02091EE05222309F4A7C0A0939D
:10DAA0003D1320932F1380E030E0E1E0F0E0C82F39
:10DAB000AF01082E02C0440F551F0A94E2F7241745
:10DAC000350741F0982F8F5F983089F789E0809370
:10DAD00038138CC0809338132091F7053091F805E6
:10DAE0002115310519F040E050E008C020910506ED
:10DAF0003091060640910706509108062093301396
:10DB00003093311340933213509333132401350172
:10DB1000460E571E611C711C40923E1350923F13DB
:10DB20006092401370924113E091F205F091F30579
:10DB3000F0934413E0934313B0E00F943F1B460E61
:10DB4000571E681E791E40924513509246136092EC
:10DB500047137092481385E0EE0FFF1F8A95E1F797
:10DB6000E150FE4FEF2FFF27E6954E0E5F1E611C22
:10DB7000711C4092391350923A1360923B13709289
:10DB80003C132091F4053091F5052115310521F064
:10DB9000890120E030E008C00091010610910206E2
:10DBA0002091030630910406B501A40144195509DA
:10DBB00066097709400F511F621F731F04C07695D5
:10DBC000679557954795CA95D2F74093341350936C
:10DBD00035136093361370933713453F2FE0520788
:10DBE0006105710528F48CE080934213F12C1AC072
:10DBF000453F5F4F6105710510F480E111C08091D0
:10DC00000D0690910E06A0910F06B091100680931C
:10DC1000451390934613A0934713B093481380E2A3
:10DC2000809342138F2DDF91CF911F910F91FF9021
:10DC3000BF90AF909F908F907F906F905F904F902C
:10DC40000895EF92FF920F931F93CF93DF93CDB779
:10DC5000DEB76F970FB6F894DEBF0FBECDBF7B0166
:10DC60000EEC11E120ED31E1F8013183208322E057
:10DC7000209307149093A01080939F1040E050E0F1
:10DC8000BA0184ED91E10F94ED04F8018081918156
:10DC90002BE1FC013496DE01159601900D922A9538
:10DCA000E1F7FC01828193819C838B8382EB93E07B
:10DCB0009A838983A701BE016F5F7F4F85EA93E056
:10DCC0000E9427B5CE0101960E9441836F960FB640
:10DCD000F894DEBF0FBECDBFDF91CF911F910F91A2
:10DCE000FF90EF90089510925B118091501388235C
:10DCF00021F08DE493E10C94064B08956F927F928E
:10DD00008F929F92AF92BF92DF92EF92FF920F930A
:10DD10001F93CF93DF93CDB7DEB7AE970FB6F894CE
:10DD2000DEBF0FBECDBF20915C11222309F406C2D5
:10DD3000D62E7C0180915013882309F4A5C044237A
:10DD400009F4CFC180916813882329F1E9E7F8E14C
:10DD500084918F010F5F1F4F882321F00F9496024B
:10DD6000F801F6CFE6E3F8E184918F010F5F1F4FD2
:10DD7000882321F00F949602F801F6CF61E070E05D
:10DD800080E090E00E94EAA58AE00F9496028DE27E
:10DD900098E10E9454838EE693E19EA78DA78FE2BF
:10DDA00080936D1381E0898310E00FE1809125134A
:10DDB000181778F4019FC0011124AE014F5F5F4F27
:10DDC000BE01635D7F4F81519E4E0E9498AE1F5FE2
:10DDD000EDCF898187FD0FC0AE014F5F5F4FBE0160
:10DDE000635D7F4F89E493E10E9498AE8DA59EA567
:10DDF00001979EA78DA7EDA5FEA51082E09168135F
:10DE000084E0E89FF0011124E759FC4E8091FE1355
:10DE10009091FF13A0910014B0910114808391831D
:10DE2000A283B383EAE3F2E484918F010F5F1F4F73
:10DE3000882321F00F949602F801F6CFB70184E110
:10DE400098E10E94C591609168139DE8699FB001B7
:10DE5000112463597C4E89E098E10E94C59140915C
:10DE6000FE135091FF13609100147091011483E030
:10DE700098E10E9455918AE00F9496028091681370
:10DE80008F5F8093681327C04423C1F0EAE3F2E474
:10DE900084918F010F5F1F4F882321F00F9496020A
:10DEA000F801F6CFE3EFF7E184918F010F5F1F4F89
:10DEB000882389F00F949602F801F6CF1092681328
:10DEC00082E0B82E10C1B7018AED97E10E94C5919A
:10DED0008AE00F94960207DF1D8218861C821B823F
:10DEE00082EB93E09A8389838FEA91E19093CF113B
:10DEF0008093CE11F70180818F3209F05CC08701D9
:10DF00000F5F1F4FCE0101964C010115110509F459
:10DF100058C06FE270E0C8010F94921E5C01009738
:10DF200009F450C00817190708F04CC03C01601AEA
:10DF3000710AA301B801CE0180960F94B21EE0E2EF
:10DF4000F0E0EC0FFD1FE60DF71D10826091CE1181
:10DF50007091CF116115710511F06C5F7F4F21E059
:10DF6000AE01405E5F4FCE0105960E941A4E8111B0
:10DF70001AC0E6ECF7E184918F010F5F1F4F81110A
:10DF800004C08E01005E1F4F04C00F949602F8017A
:10DF9000F2CFF80181918F01882319F00F94960236
:10DFA000F8CF8EE287C09092CF118092CE1185017A
:10DFB0000F5F1F4FAACF80ED91E19093CF11809317
:10DFC000CE1187019091CE118091CF11692F782FBA
:10DFD000DD2009F459C06115710511F06C5F7F4FA8
:10DFE00021E0A8018DE493E10E941A4E882309F4F0
:10DFF00047C080915E1390915F13A0916013B09120
:10E0000061138093FA139093FB13A093FC13B093C6
:10E01000FD131092FE131092FF1310920014109231
:10E020000114B80188EB97E10E94C5914091FA1361
:10E030005091FB136091FC137091FD1380EB97E1FD
:10E040000E9455918AE00F949602E1EAF7E18491EB
:10E050007F019FEFE91AF90A882321F00F949602B5
:10E06000F701F5CFB80180E090E0EBDD80916B1116
:10E07000882319F08BE691E101C0C80160E02AC055
:10E08000B8018DE897E110C06115710511F06C5F62
:10E090007F4F26E5A8018DE493E10E941A4E81117D
:10E0A0000CC0B80189E797E10E94C5918EE20F94F8
:10E0B00096028AE00F9496020FC081E08093591176
:10E0C000B70187E697E10E94C5918AE00F94960216
:10E0D00060E0C8010E941746CE0101960E9441836C
:10E0E0002DC0BB24B394EAE3F2E484918F010F5F67
:10E0F0001F4F882321F00F949602F801F6CFEEEE21
:10E10000F7E184918F010F5F1F4F882321F00F9457
:10E110009602F801F6CFE1E0BE1619F0E8EEF7E15D
:10E1200002C0E2EEF7E184918F010F5F1F4F882359
:10E1300009F4C9CE0F949602F801F5CFAE960FB64A
:10E14000F894DEBF0FBECDBFDF91CF911F910F912D
:10E15000FF90EF90DF90BF90AF909F908F907F9057
:10E160006F900895CF92DF92EF92FF920F931F93DB
:10E17000CF93DF93CDB7DEB7EDB6FEB6DC010D90E1
:10E180000020E9F79D01281B390B2C5F3F4F4DB74D
:10E190005EB7421B530B0FB6F8945EBF0FBE4DBF68
:10E1A0000DB71EB70F5F1F4F9F938F9380E697E1C8
:10E1B0009F938F931F930F930F94BF16680154E0A2
:10E1C000C50ED11C0F900F900F900F900F900F90D5
:10E1D000F6018081882339F090E00F94561EF601F5
:10E1E00081936F01F5CF60E0C8010E9467568823D4
:10E1F00019F0C8010E94E3828CE597E19093ED0746
:10E200008093EC070E9483560FB6F894FEBE0FBEB3
:10E21000EDBEDF91CF911F910F91FF90EF90DF90B6
:10E22000CF900895AF92BF92CF92DF92EF92FF927C
:10E230000F931F93CF93DF93CDB7DEB7AA970FB697
:10E24000F894DEBF0FBECDBF8091AE118F93809149
:10E25000AD118F9383E597E19F938F937E0181E2C8
:10E26000E80EF11CFF92EF920F94BF160F900F90E3
:10E270000F900F900F900F9010E0F7010190002089
:10E28000E9F73197EE19FF091E1774F46701C10E03
:10E29000D11C17FDDA94F601808190E00F94561E90
:10E2A000F60180831F5FE9CF40E050E0BA0183EBC5
:10E2B00091E10F94ED0400E0CE0101966C01809194
:10E2C000B611823028F4011114C08FEF9FEF16C0F1
:10E2D0008091BB119091BC11A091BD11B091BE1164
:10E2E0008F719927AA27BB27892B8A2B8B2B59F74C
:10E2F0001AC08091AD119091AE1101969093AE111C
:10E300008093AD11AA960FB6F894DEBF0FBECDBFB5
:10E31000DF91CF911F910F91FF90EF90DF90CF9001
:10E32000BF90AF90089540E050E0B60183EB91E1DB
:10E330000F94240818163CF6F60101900020E9F726
:10E3400031971E2F1C19115068F05601A10EB11CF7
:10E3500017FDBA94F501808190E00F94561EF501E7
:10E360008083F1CF8A858E3709F4A9CF45E050E04C
:10E37000B701C6010F94A41E892B09F0A0CFC701D5
:10E38000F1DE01E09CCFCF92DF92EF92FF921F93DC
:10E39000CF93DF9310925C118091B611882321F006
:10E3A00083EB91E10E94064B10922A1310922713DF
:10E3B00085E3809326130E9407D0EB01A8958091F6
:10E3C00026130E9408B186E293E10E94F5E12398AA
:10E3D000229A219A209A289A85E08093281382E530
:10E3E0008CBD1DBC1AE08FEF0E94FAE11150D9F7E5
:10E3F00020E030E0A90160E086E293E10E9420E2A3
:10E40000182F80932913813049F00E9407D06C1B8C
:10E410007D0B613D774060F381E054C02AEA31E032
:10E4200040E050E068E086E293E10E9420E282FF53
:10E4300003C010932A130EC014E00E94FFE18093E2
:10E4400029131150D1F78A3A11F082E03BC082E0E3
:10E4500080932A1380912A13823021F0C12CD12C71
:10E46000760105C0C12CD12CE12C80E4F82E20E0EF
:10E4700030E0A90167E386E293E10E9420E2A70170
:10E48000960169E286E293E10E9420E280932913DB
:10E49000882349F00E9407D06C1B7D0B613D7740BB
:10E4A00030F38AE00FC080912A13823011F520E00A
:10E4B00030E0A9016AE386E293E10E9420E288232A
:10E4C00051F088E08093271386E293E10E94F5E102
:10E4D000EAE3F2E419C00E94FFE1807C803C19F479
:10E4E00083E080932A130E94FFE10E94FFE10E94D3
:10E4F000FFE186E293E10E94F5E11092281381E0AA
:10E5000040DA811131C015C08491EF012196882332
:10E5100021F00F949602FE01F7CFE5E4F7E1849134
:10E52000EF012196882309F456C00F949602FE014C
:10E53000F6CF80E026DA811117C0E9E7F8E184918F
:10E54000EF012196882321F00F949602FE01F7CF68
:10E55000E1E3F7E18491EF012196882309F43BC0C0
:10E560000F949602FE01F6CF6BE273E183EB91E12B
:10E570000F948508811116C0E9E7F8E18491EF0155
:10E580002196882321F00F949602FE01F7CFE0E256
:10E59000F7E18491EF0121968823E9F00F94960228
:10E5A000FE01F7CF81E080935C11EAE3F2E484910D
:10E5B000EF012196882321F00F949602FE01F7CFF8
:10E5C000E4E1F7E18491EF012196882321F00F9493
:10E5D0009602FE01F7CF8BE1E3EBF1E1A4EDB1E1AF
:10E5E00001900D928A95E1F78091B1119091B2114D
:10E5F0009093D3118093D21180ED91E19093CF113C
:10E600008093CE11DF91CF911F91FF90EF90DF901B
:10E61000CF900895EF92FF921F93CF93DF931F92B5
:10E62000CDB7DEB7182FE9E7F8E184917F012FEF2E
:10E63000E21AF20A882331F099830F949602F701C7
:10E640009981F3CFE12FF92F84917F019FEFE91A90
:10E65000F90A882321F00F949602F701F5CF609113
:10E66000DD057091DE058091DF059091E0050E9447
:10E67000EAA58AE00F9496020E9475861092DC0546
:10E680001092DB050F90DF91CF911F91FF90EF90DB
:10E6900008950F931F93CF93DF938C01EB0190911B
:10E6A0000A1120910B11921307C08EEF90E10E9486
:10E6B000D28F0E947E60F3CFF801A081B1814881A2
:10E6C00059818091091134E0839FF0011124EE5F9C
:10E6D000FE4EB387A287558744879F5F90930A11A8
:10E6E0008F5F821719F08093091102C010920911EF
:10E6F000DF91CF911F910F910895EF92FF920F93A9
:10E700001F93CF93DF931F92CDB7DEB78B01622F9C
:10E71000498345D7909146148091DA05498189173C
:10E7200008F43FC0909148148091D905981708F4D7
:10E7300038C0442399F120E030E0F801E20FF31FE4
:10E74000E491EE2319F02F5F3F4FF7CF86E190E081
:10E75000821B930B97FD01969595879536E1F32ED5
:10E7600049EEE42EE80E8E2D8F0D87FD0EC080E25F
:10E770000E9463B2FA94F7CFF8018491882339F0AC
:10E780000E94A090F81A0F5F1F4F1F14ACF31F14C4
:10E7900044F480E20E9463B2FA94F9CF86E1F82E45
:10E7A000F4CF0F90DF91CF911F910F91FF90EF90D9
:10E7B0000895CF92DF92EF92FF920F931F93CF9322
:10E7C000DF9300D01F92CDB7DEB77C018B01298388
:10E7D0003A834B835C831ED683E080933D02F092A4
:10E7E000D505E092D4051093D3050093D205298175
:10E7F0003A814B815C81CA01B9010F942A172AE042
:10E8000037ED43E25CE30F948B170F94A31C6093E6
:10E81000CE057093CF058093D0059093D1050F94CA
:10E820002C176B017C019B01AC0160E070E887E76D
:10E8300094E40F945E1B0F94A31C6093CA0570931D
:10E84000CB058093CC059093CD05F8016081718153
:10E85000828193810F942A172AE037ED43E25CE32B
:10E860000F948B17A70196010F945E1B0F94A81CA1
:10E870006093AF107093B0108093B1109093B2106A
:10E8800085E492E490933C0280933B0281E59CEB0B
:10E890009093D8058093D7051092D6050F900F90CE
:10E8A0000F900F90DF91CF911F910F91FF90EF90FC
:10E8B000DF90CF900895AF92BF92CF92DF92EF9208
:10E8C000FF920F931F93CF93DF937C01EB015A01CB
:10E8D0006901A0D523E020933D02F092D505E09296
:10E8E000D405D093D305C093D205A501BB0C660B0C
:10E8F000770B4093CE055093CF056093D00570936E
:10E90000D105C601DD0CAA0BBB0B841B950BA60B16
:10E91000B70B8093CA059093CB05A093CC05B09319
:10E92000CD0588819981092E000CAA0BBB0B841B95
:10E93000950BA60BB70B8093AF109093B010A093DC
:10E94000B110B093B21089E294E490933C028093AA
:10E950003B021093D8050093D7051092D605DF919E
:10E96000CF911F910F91FF90EF90DF90CF90BF90CC
:10E97000AF9008954F925F926F927F928F929F9285
:10E98000AF92BF92FF920F931F93CF93DF93CDB7B8
:10E99000DEB72A970FB6F894DEBF0FBECDBF109238
:10E9A000CF048091D504882339F00E941F908CEE0B
:10E9B00090E00E9464B3BBC4209193023091940212
:10E9C0004091AF105091B0106091B1107091B210A1
:10E9D000C901840F951F2436310524F4853691052D
:10E9E0003CF416C02436310531F08436910584F4A8
:10E9F00084E690E00DC0473051056105710514F0C3
:10EA0000069706C04A3F5F4F6F4F7F4F6CF40696E4
:10EA100090939402809393021092AF101092B010D2
:10EA20001092B1101092B2108091930290919402C2
:10EA30008A3091053CF0883E43E094072CF087EE45
:10EA400093E002C08AE090E0909394028093930256
:10EA50000E944449F82E0E947C45809146148531DD
:10EA600098F4FF2049F08091A3049091A404892B8D
:10EA700019F00DED1EE102C000EC1DE123E14FE0B5
:10EA800061E089E00E9461B1809146148D3108F007
:10EA900084C1883008F03FC08091AA10F11002C0F4
:10EAA000811139C060919C0470919D04072E000C67
:10EAB000880B990B0F942C1720E030E040E05FE3C7
:10EAC0000F945F1B0F94A31C643671052CF46A30FD
:10EAD000710524F446E003C042E101C04CE022E1AC
:10EAE00030E0241B310937FF02C02F5F3F4F3595BF
:10EAF00027953195219531092B5F2093491427E003
:10EB000020934A14CB010E94D3E50E94D8908DEB4C
:10EB10009DE10E94CB90809146148D31D0F580917B
:10EB200048148531B0F120E030E040E05FE36091CF
:10EB30009E0470919F048091A0049091A1040F9471
:10EB40005F1B0F94A31C9B01643671050CF0D6C2A9
:10EB50002A3031050CF0D0C246E022E130E0241B1F
:10EB6000310937FF02C02F5F3F4F3595279531950B
:10EB7000219531092B5F209349142CE120934A14ED
:10EB8000CB010E94D3E50E94D8908DEB9DE10E94BD
:10EB9000CB9080914614853140F5809148148131A5
:10EBA00020F160919C0470919D04072E000C880B4D
:10EBB000990B0F942C1720919E0430919F04409143
:10EBC000A0045091A1040F94851D18160CF098C252
:10EBD0001092321402E022E041E16DE082E194E122
:10EBE0000E94D9CC81E08093321480914614883001
:10EBF00008F03FC08091A110F11002C0811139C00E
:10EC000060919A0470919B04072E000C880B990B5D
:10EC10000F942C1720E030E040E05FE30F945F1B7F
:10EC20000F94A31C643671052CF46A30710524F42A
:10EC300046E003C042E101C04CE022E130E0241B89
:10EC4000310937FF02C02F5F3F4F3595279531952A
:10EC5000219531092F5A2093491427E020934A1413
:10EC6000CB010E94D3E50E94D8908DEB9DE10E94DC
:10EC7000CB90809146148D31D0F580914814853128
:10EC8000B0F120E030E040E05FE3609190047091EB
:10EC9000910480919204909193040F945F1B0F94C0
:10ECA000A31C9B01643671050CF035C22A30310576
:10ECB0000CF02FC246E022E130E0241B310937FF7F
:10ECC00002C02F5F3F4F359527953195219531092A
:10ECD0002F5A209349142CE120934A14CB010E940F
:10ECE000D3E50E94D8908DEB9DE10E94CB9080915E
:10ECF0004614853140F580914814813120F16091AE
:10ED00009A0470919B04072E000C880B990B0F94AA
:10ED10002C172091900430919104409192045091CD
:10ED200093040F94851D18160CF0F7C1109232143D
:10ED300002E022E042E168E582E194E10E94D9CC60
:10ED400081E080933214809146148C3130F58091AB
:10ED50004814843110F18091A3049091A404019689
:10ED600044E6489F9001499F300D112437FF02C0AF
:10ED700021503F4F832F932F990F990B009769F0E4
:10ED800028E6209349142BE120934A140E94D3E5EE
:10ED90000E94D89085E20E9463B28091501388232C
:10EDA00049F080914614843328F4809148148A32C3
:10EDB00008F0BCC180914614853328F48091481432
:10EDC000813308F0D9C16091A204623048F080918B
:10EDD0004614843328F480914814823308F0D1C15A
:10EDE00080914614813308F060C0809148148932C4
:10EDF00008F45BC00E9498B22B013C018CE3882E82
:10EE0000912CA12CB12CC301B201A50194010F9446
:10EE1000011BCA01B901A50194010F94011BCA018C
:10EE2000B62EA72E49018E010F5F1F4F41E84416F1
:10EE300041E5540641E06406710408F4BDC1B9011E
:10EE400028E130E040E050E00F94011B29013A0135
:10EE5000AF92BF92C40168E170E00F94271E9F93A8
:10EE60008F935F924F9282E998E19F938F931F93C4
:10EE70000F930F94BF160FB6F894DEBF0FBECDBF31
:10EE80009AE0491651046104710408F0BFC197E08B
:10EE9000892F880F980F9195955A9093491480E384
:10EEA00080934A14C8010E94D890E0910C14F0910C
:10EEB0000D1484818111ECC020917D1430917E1459
:10EEC00040917F14509180146091AA147091AB14FA
:10EED0008091AC149091AD140F945F1B0F94A31C00
:10EEE000CB010E946CE5BC018EE198E00F949D1E61
:10EEF0002091811430918214409183145091841494
:10EF00006091AE147091AF148091B0149091B114CF
:10EF10000F945F1B0F94A31CCB010E946CE5BC01F6
:10EF200089E198E00F949D1E2091851430918614FC
:10EF300040918714509188146091B2147091B31469
:10EF40008091B4149091B5140F945F1B2CEA35ECAA
:10EF500047E257E30F945F1B20E030E048EC52E4B7
:10EF60000F948B170F94A31C4B015C0197FD19C0E4
:10EF700090E1891697E29906A104B104E4F0C50175
:10EF8000B40120E137E240E050E00F94231BCA01B6
:10EF9000B9012AE030E040E050E00F94231B605DAF
:10EFA0000BC0B094A09490948094811C911CA11CDF
:10EFB000B11C6DE201C060E26093641428EE821619
:10EFC00023E09206A104B10494F0C501B40128EE37
:10EFD00033E040E050E00F94231BCA01B9012AE05E
:10EFE00030E040E050E00F94231B605D01C060E220
:10EFF00060936514C501B40124E630E040E050E0C0
:10F000000F94231B9AE0492E512C612C712CCA01BC
:10F01000B901A30192010F94231B605D60936614F4
:10F02000C501B401A30192010F94231B4B015C01A4
:10F03000672B682B692B79F08EE280936714CA01E5
:10F04000B901A30192010F94231B605D60936814C2
:10F0500080E3880D15C0CA01B901A30192010F9484
:10F06000231B662339F08EE280936714605D609302
:10F07000681405C080E2809368148093671480E26E
:10F080008093691464E674E182E198E00F949D1E18
:10F09000809146148632A8F4809148148E3188F00D
:10F0A00008E020E84EE160E082E194E10E94D9CCE2
:10F0B00080914614863228F4809148148F3108F0EC
:10F0C000A7C080914614823328F4809148148C3272
:10F0D00008F00EC1809146148F3308F028C180914A
:10F0E0004814883308F423C1109249148EE38093A6
:10F0F0004A140E9420B31BC14CE02FCD42E12DCD1C
:10F1000002E022E041E16DE082E194E10E94D9CC8D
:10F110006CCD4CE0D0CD42E1CECD02E022E042E128
:10F1200068E582E194E10E94D9CC0DCE07E028E0A9
:10F130004AE26AE282E194E10E94D9CC05E022E051
:10F140004CE262E382E194E10E94D9CC6AE08AE277
:10F150000E94B7B1609114147091151482E38093EA
:10F160002E148BE280932F142EE234E142E382E1ED
:10F1700094E10E9417CB1ECE6AE486E30E94B7B1E9
:10F1800022CE48E4649FB0011124072E000C880BA6
:10F19000990B0F942C172AE037ED43E25CE30F94B0
:10F1A0008B170F94A81C262F02E042E367E382E14D
:10F1B00094E10E94D9CC14CE44E68416910498F4CC
:10F1C000AF92BF923F932F9388E898E19F938F93DC
:10F1D0001F930F930F94BF160FB6F894DEBF0FBEA8
:10F1E000CDBF95E055CEAF92BF923F932F9380E86D
:10F1F00098E19F938F931F930F930F94BF160FB6B1
:10F20000F894DEBF0FBECDBF96E042CE98E040CE70
:10F210001092321483E08093491485E280934A145B
:10F22000FF2029F08BEB9DE10E94CB900DC08091D7
:10F23000CA14811102C08FE305C080918D04811131
:10F24000F1CF80E20E9463B28BE08093491415E213
:10F2500010934A148EE198E00E94D8908BE280933C
:10F26000491410934A14FF2029F089EB9DE10E9474
:10F27000CB900DC08091CB14811102C08FE305C0EB
:10F2800080918E048111F1CF80E20E9463B283E30A
:10F290008093491415E210934A1489E198E00E9482
:10F2A000D89083E58093491410934A14FF2029F0E5
:10F2B00087EB9DE10E94CB900DC08091CC14811111
:10F2C00002C08FE305C080918F048111F1CF80E2ED
:10F2D0000E9463B28BE58093491485E280934A14BF
:10F2E00082E198E00E94D89081E080933214E9CEC8
:10F2F00084E00E94869083E08093491412E3109387
:10F300004A1486E00E94B7900E947C458CE080936E
:10F31000491410934A1480919302909194020E9490
:10F32000D3E50E94D89085E20E9463B2D3CE2A969C
:10F330000FB6F894DEBF0FBECDBFDF91CF911F9106
:10F340000F91FF90BF90AF909F908F907F906F90A4
:10F350005F904F900895282F8091AF109091B0103A
:10F36000A091B110B091B21081309048A105B105C3
:10F3700040F01092AF101092B0101092B110109295
:10F38000B2108091C404882331F08091AF10809333
:10F3900023081092AC108091B9041816FCF4082EC2
:10F3A000000C990B821B910920912308022E000C5E
:10F3B000330B2817390794F097FF02C080E090E0E4
:10F3C00080932308092E000CAA0BBB0B8093AF106F
:10F3D0009093B010A093B110B093B2108091230815
:10F3E0006623A9F09091BA04891714F48093BA04A3
:10F3F0002091BA04022E000C330B2C5F3F4F482F94
:10F40000082E000C550B241735071CF484508093EC
:10F41000BA0408958091AD108630D8F496E0899FA3
:10F42000F0011124E251F84F20913B0230913C024F
:10F43000318320834091AF105091B0106091B11092
:10F440007091B21042835383648375838F5F80937E
:10F45000AD1008958AEB94E70C9464B3E091AD107D
:10F46000EE2369F0E150E093AD1086E0E89FF001F3
:10F470001124E251F84F808191810C9464B3EACF5A
:10F480001092AE10EBCFAF92BF92CF92DF92EF927D
:10F49000FF920F931F93CF93DF935C017B0120E0DA
:10F4A00030E0F501E20FF31FE491EE2319F02F5F36
:10F4B0003F4FF7CFF701CF018E199F0941914111BD
:10F4C000FACF04E110E0081B1109332702171307D4
:10F4D0001CF0DD24D39402C082E0D82E8091131456
:10F4E00090E06D2D70E06F5F7F4F0F943B1EC62E36
:10F4F000C6E0C60F80914614C81750F0809148149A
:10F5000090E02C2F30E02B503109821793079CF5A7
:10F51000D0E0E114F104C1F18AE30E9463B282E019
:10F52000D8120FC0CC0D80914614C81768F12091F5
:10F53000481430E08C2F90E00B97281739071CF403
:10F5400023C0DD2309F1802F880F080F000F0093DF
:10F550004914C0934A1480E20E9463B2C701DF914C
:10F56000CF911F910F91FF90EF90DF90CF90BF90C0
:10F57000AF900C94D89010924914C0934A14C501CE
:10F580000E94CB90D1E0C5CFDF91CF911F910F9119
:10F59000FF90EF90DF90CF90BF90AF9008950F93C2
:10F5A0004CE0849F402D112421E0240F2093D905A5
:10F5B0008CE0840F8093DA05E0914614F0E090E04F
:10F5C00002968E179F070CF1822F90E0209148142D
:10F5D00030E082179307CCF4662371F081E08093CA
:10F5E00032144D5F0BE020E860E082E194E10E947C
:10F5F000D9CC1092321403C081E0809332148091F0
:10F60000DA051092491480934A140F910895CF920D
:10F61000DF92EF92FF920F93CF93DF93982F862F75
:10F620006A017901692FBBDF909146148091DA0558
:10F63000891708F453C0909148148091D905981700
:10F6400008F44CC0002359F060E070E0F701E60FC9
:10F65000F71FE491EE2351F06F5F7F4FF7CFD70193
:10F66000BD016E197F098D918111FACFC62FD4E1AA
:10F67000D61BF6018491882339F00E94A090D81BF4
:10F68000FFEFCF1ADF0AF5CF8AE30E9463B2DD23D2
:10F6900029F080E20E9463B2D150F9CF8091DA055F
:10F6A0006AEFC69F602D11246058609349148093BF
:10F6B0004A14C701002349F0DF91CF910F91FF90C9
:10F6C000EF90DF90CF900C94CB90DF91CF910F9182
:10F6D000FF90EF90DF90CF900C94D890DF91CF9176
:10F6E0000F91FF90EF90DF90CF9008950F93CF93FD
:10F6F000DF93CDB7DEB7ED85FE85608171818281B4
:10F7000093810F94A31CCB010E94D3E500E09C01E0
:10F7100049855A8568858F817ADFDF91CF910F9176
:10F7200008951F93CF93DF9360E085E014DED091BE
:10F73000BA04C0E012E0D11109C080913D028823D3
:10F74000D9F121E041E06EE472E215C0D13049F414
:10F7500080913D02882381F120E041E065E472E27E
:10F760000AC0D23061F480913D02882329F120E063
:10F7700041E064E372E28C2F0E947D731DC0D330A0
:10F7800049F480913D028823B9F020E041E062E332
:10F7900072E2F1CFD43081F480913D02882351F0A0
:10F7A00021E040E067E272E28C2F0E947D738C2F93
:10F7B0000E94E39010933D02CF5FDF5FC53009F0F8
:10F7C000BACFC093B904DF91CF911F9108951F93D1
:10F7D000CF93DF9360E085E0BEDDD091BA04C0E056
:10F7E00012E0D11109C080913D028823D9F121E0B6
:10F7F00041E06AE172E215C0D13049F480913D02E6
:10F80000882381F120E041E061E172E20AC0D23058
:10F8100061F480913D02882329F120E041E063E01A
:10F8200072E28C2F0E947D731DC0D33049F4809109
:10F830003D028823B9F020E041E061E072E2F1CFBF
:10F84000D43081F480913D02882351F021E040E0E2
:10F8500066EF71E28C2F0E947D738C2F0E94E390E3
:10F8600010933D02CF5FDF5FC53009F0BACFC09380
:10F87000B904DF91CF911F9108951F93CF93DF9328
:10F8800060E085E068DDD091BA04C0E012E0D111FB
:10F8900009C080913D028823D9F121E041E069EE61
:10F8A00071E215C0D13049F480913D02882381F185
:10F8B00020E041E069ED71E20AC0D23061F480914C
:10F8C0003D02882329F120E041E068EC71E28C2FB1
:10F8D0000E947D731DC0D33049F480913D0288237E
:10F8E000B9F020E041E069EB71E2F1CFD43081F46E
:10F8F00080913D02882351F021E040E06EEA71E200
:10F900008C2F0E947D738C2F0E94E39010933D02F8
:10F91000CF5FDF5FC53009F0BACFC093B904DF9184
:10F92000CF911F9108951F93CF93DF9360E085E0FF
:10F9300012DDD091BA04C0E012E0D11109C080916B
:10F940003D028823D9F121E041E061EA71E215C06E
:10F95000D13049F480913D02882381F120E041E0DB
:10F9600061E971E20AC0D23061F480913D028823DE
:10F9700029F120E041E064E871E28C2F0E947D7360
:10F980001DC0D33049F480913D028823B9F020E0B6
:10F9900041E062E871E2F1CFD43081F480913D0220
:10F9A000882351F021E040E067E771E28C2F0E944C
:10F9B0007D738C2F0E94E39010933D02CF5FDF5F39
:10F9C000C53009F0BACFC093B904DF91CF911F9130
:10F9D00008951F93CF93DF9360E085E0BCDCD09166
:10F9E000BA04C0E012E0D11109C080913D02882321
:10F9F000D9F121E041E06AE671E215C0D13049F465
:10FA000080913D02882381F120E041E06BE571E2C5
:10FA10000AC0D23061F480913D02882329F120E0B0
:10FA200041E06CE471E28C2F0E947D731DC0D330E5
:10FA300049F480913D028823B9F020E041E06AE476
:10FA400071E2F1CFD43081F480913D02882351F0EE
:10FA500021E040E06FE371E28C2F0E947D738C2FD8
:10FA60000E94E39010933D02CF5FDF5FC53009F045
:10FA7000BACFC093B904DF91CF911F9108951F931E
:10FA8000CF93DF9360E085E066DCD091BA04C0E0FC
:10FA900012E0D11109C080913D028823D9F121E003
:10FAA00041E062E371E215C0D13049F480913D023A
:10FAB000882381F120E041E069E271E20AC0D2309E
:10FAC00061F480913D02882329F120E041E069E161
:10FAD00071E28C2F0E947D731DC0D33049F4809158
:10FAE0003D028823B9F020E041E067E171E2F1CF07
:10FAF000D43081F480913D02882351F021E040E030
:10FB00006CE071E28C2F0E947D738C2F0E94E39039
:10FB100010933D02CF5FDF5FC53009F0BACFC093CD
:10FB2000B904DF91CF911F9108951F93CF93DF9375
:10FB300060E085E010DCD091BA04C0E012E0D111A1
:10FB400009C080913D028823D9F121E041E06FEFA7
:10FB500070E215C0D13049F480913D02882381F1D3
:10FB600020E041E060EF70E20AC0D23061F48091A1
:10FB70003D02882329F120E041E060EE70E28C2F05
:10FB80000E947D731DC0D33049F480913D028823CB
:10FB9000B9F020E041E069ED70E2F1CFD43081F4BA
:10FBA00080913D02882351F021E040E06EEC70E24C
:10FBB0008C2F0E947D738C2F0E94E39010933D0246
:10FBC000CF5FDF5FC53009F0BACFC093B904DF91D2
:10FBD000CF911F9108950F931F93CF93DF9361E00F
:10FBE00081E0B9DBD091BA04C0E081E011E002E02D
:10FBF000D1112AC08823D9F0809123081816BCF0AF
:10FC00004091AF105091B0106091B1107091B2104E
:10FC10004F5F5F4F6F4F7F4F4093AF105093B010C7
:10FC20006093B1107093B2108F5F8093230880911E
:10FC30003D02882309F44AC020E041E06EEB70E207
:10FC40008C2F0E947D7342C0D130F1F48091D50495
:10FC5000811105C080913D028823C1F10BC08091C4
:10FC600023088130B9F7009306048091AC108823F3
:10FC700089F335C081E090912308913009F080E04C
:10FC800020E241EB50E21FC0D23001F58091D50453
:10FC9000811105C080913D028823C1F00BC0809185
:10FCA00023088230B9F7109306048091AC108823A2
:10FCB00089F315C081E090912308923009F080E02B
:10FCC00020E244EA50E26C2F0E943D45CF5FDF5FA7
:10FCD00080E0C53009F08CCF83E08093B904DF91D8
:10FCE000CF911F910F9108951F93CF93DF9361E000
:10FCF00081E031DBD091BA04C0E081E012E0D111A3
:10FD000027C08823D9F0809123081816BCF04091B1
:10FD1000AF105091B0106091B1107091B2104F5F60
:10FD20005F4F6F4F7F4F4093AF105093B010609371
:10FD3000B1107093B2108F5F8093230880913D02C1
:10FD4000882309F470C021E041E065E970E255C004
:10FD5000D13039F58823D9F0809123088230BCF462
:10FD60004091AF105091B0106091B1107091B210ED
:10FD70004F5F5F4F6F4F7F4F4093AF105093B01066
:10FD80006093B1107093B2108F5F809323088091BD
:10FD90003D02882309F447C020E040E060E870E2BB
:10FDA0002CC0D23001F58091D504811105C080911D
:10FDB0003D028823C1F10AC0809123088230B9F73F
:10FDC0005FDB8091AC10882391F335C081E0909186
:10FDD0002308923009F080E024E04BE750E26C2FDA
:10FDE0000E943D4520C0D33061F480913D028823BC
:10FDF000D1F020E041E069E770E28C2F0E947D7332
:10FE000012C0D43081F480913D02882351F021E06A
:10FE100040E06EE670E28C2F0E947D738C2F0E9472
:10FE2000E39010933D02CF5FDF5F80E0C53009F0C3
:10FE300066CFC093B904DF91CF911F910895BF920F
:10FE4000CF92DF92EF92FF920F931F93CF93DF93A6
:10FE5000CDB7DEB76F970FB6F894DEBF0FBECDBF3C
:10FE600080ED91E19093CF118093CE1181E080934A
:10FE70000714109209141092081440E050E0BA01DF
:10FE800084ED91E10F94ED048091CE119091CF110A
:10FE90002BE1FC013496DE01159601900D922A9516
:10FEA000E1F7FC01828193819C838B8382EB93E059
:10FEB0009A83898340E050E0BE016F5F7F4F85EAFF
:10FEC00093E00E9427B5CE010196DBD3C0900814C1
:10FED000D090091461E081E03EDA1091BA0400E0AC
:10FEE000F1E0CF1AD10811111EC08091D504811103
:10FEF00005C080913D028823B1F00AC0809123089B
:10FF00008111F7CFBDDA8091AC10882391F350C1F5
:10FF100081E090912308911180E024E049E650E2CD
:10FF2000602F0E943D456EE571E184ED91E10E94F4
:10FF3000B64A80915E118F3209F45AC0113009F02F
:10FF400059C08091D504882309F441C080912308C9
:10FF50008130E9F580912513882319F18150809330
:10FF60002513882361F090E001974FE1489F9001AD
:10FF7000499F300D1124C90181519E4E02C08FEA64
:10FF800091E12BE1FC013496A4EDB1E101900D92D9
:10FF90002A95E1F7FC01828193819093D31180939C
:10FFA000D21181E090E0A0E0B0E020912513211172
:10FFB00003C080E090E0DC018093AF109093B0101C
:10FFC000A093B110B093B2101092BA042DC08091DA
:10FFD0003D02882379F081E090912308913009F067
:10FFE00080E020E245E650E2602F0E943D4502C0DD
:10FFF00091E001C092E07601BB24B394B10E33C00E
:020000021000EC
:100000008AE00F949602CE0101963BD31092BA0477
:1000100082E090E0A0E0B0E08093AF109093B01049
:10002000A093B110B093B21081E08093AC1083E044
:1000300080933D02BDC01913B2C060E070E0C701FB
:100040000E94216E90915D118091D504992309F44D
:1000500086C081110DC080913D02811179C09B2D18
:1000600041E0E41AF1088FEFE816F80621F799C08D
:10007000809123088113EFCF1D8218861C821B827A
:1000800082EB93E09A8389838091D711882319F0BA
:1000900060ED71E102C06FEA71E16C5F7F4F21E0BA
:1000A0004EE551E1CE0105960E941A4E811124C001
:1000B000EAE3F2E484918F010F5F1F4F882321F060
:1000C0000F949602F801F6CFEFE4F0E284918F01ED
:1000D0000F5F1F4F811103C00EE511E104C00F94A3
:1000E0009602F801F3CFF80181918F01882309F47A
:1000F00087CF0F949602F7CF8BE1FE013596A4EDE2
:10010000B1E101900D928A95E1F72B813C8130930A
:10011000D3112093D211809125138A3008F073CF28
:1001200091E0980F90932513FFE18F9FC001112458
:10013000DC01AD50BE4E4BE1E4EDF1E101900D92DA
:100140004A95E1F7FC01E151FE4E338322835BCFF8
:1001500081E090912308911380E041E01CC081115F
:1001600006C080913D02882309F479CF0EC08091AA
:1001700023088113F6CF8EE591E10E94B2706AD90F
:100180008091AC10882369F313C081E0909123081B
:10019000911380E040E0602F0E9442F360CF9F5FA8
:1001A0005FCF0F5F1F5F053009F09DCE9093B904BC
:1001B0006F960FB6F894DEBF0FBECDBFDF91CF9123
:1001C0001F910F91FF90EF90DF90CF90BF90089517
:1001D000FF920F931F93CF93DF9361E081E0BBD831
:1001E000D091BA04C0E011E083E0F82ED1111DC017
:1001F0008091D504811106C080913D02882309F4C5
:10020000F5C00AC0809123088111F6CF39D98091B9
:10021000AC10882389F3F2C081E0909123089111FA
:1002200080E024E04DE350E2AEC0D13009F580918A
:10023000D504811106C080913D02882309F4D6C0FF
:100240000DC0809123088130B1F784E09AE60E94C6
:100250009F498091AC10882371F3D0C081E09091C8
:100260002308913009F080E023E044E350E28BC0A2
:10027000D23009F58091D504811106C080913D02EC
:10028000882309F4B3C00DC0809123088230B1F7F0
:100290008CE898EB0E949F498091AC10882371F301
:1002A000ADC081E090912308923009F080E023E016
:1002B0004BE250E268C0D33009F58091D50481113A
:1002C00006C080913D02882309F490C00DC0809142
:1002D00023088330B1F783E59CEB0E949F4980910E
:1002E000AC10882371F38AC081E090912308933089
:1002F00009F080E023E04EE150E245C0D43009F53A
:100300008091D504811106C080913D02882309F4B3
:100310006DC00DC0809123088430B1F782EA9AEB5A
:100320000E949F498091AC10882371F367C081E0DF
:1003300090912308943009F080E023E049E150E2F5
:1003400022C0D53021F58091D504811106C080915D
:100350003D02882309F44AC00DC0809123088530EE
:10036000B1F783E097EB0E949F498091AC108823FE
:1003700071F344C081E090912308953009F080E04A
:1003800023E040E150E26C2F0E943D452FC0D63063
:1003900069F58091D504811105C080913D028111DC
:1003A00011C024C0809123088630B9F780910B04D6
:1003B000812780930B04F0923D028091AC1088233A
:1003C00061F31CC080910B04811103C02AEF3FE14F
:1003D00002C02EEF3FE181E090912308963009F0B2
:1003E00080E001E042E050E26C2F11D9CF5FDF5F87
:1003F000C53009F0FBCE87E08093B904DF91CF913F
:100400001F910F91FF9008954F925F926F927F928C
:100410008F929F92AF92BF92DF92EF92FF920F93D3
:100420001F93CF93DF93D82EE82E880FFF08F70194
:10043000ED52FD4F6491E701CC0FDD1FCC0FDD1FA6
:10044000FE01E75BFC4D4590559065907490062E3B
:10045000000C770B880B990B0F942C174B015C0148
:1004600020E030E040EC5FE3C301B2010F948B1752
:10047000A50194010F948B17AB01BC0100E010E0C3
:1004800098018D2D0E94AB59FE01E35CFC4D259136
:10049000359145915491C501B4010F948B174B01CF
:1004A0005C0120E030E0A9010F942617882309F4AD
:1004B0004BC000E010E09801B501A40170588D2DEB
:1004C0000E94AB59F701E65CFC4D649161111BC0C1
:1004D000EAE3F2E484913F019FEF691A790A8823E5
:1004E00021F00F949602F301F5CFE8E1F3E2849155
:1004F0003F019FEF691A790A882321F00F94960231
:10050000F301F5CF6AE0FE01E85FFC4D45905590A0
:100510006590749070E080E090E00F942C179B0140
:10052000AC01C301B2010F943B1C2B013C01A5019E
:100530009401C501B4010F945F1BAB01BC01930191
:1005400082018D2D0E94AB59F701E653FB4E81E0ED
:100550008083F701E357FB4F8083FE01EE5AF74F8C
:1005600010821182128213828D2D0E94E555FE01A8
:10057000E557FD4F85919591A591B4918E01065552
:100580001B4EF80180839183A283B3830E94645938
:10059000C459DB4EF80180819181A281B3818883A7
:1005A0009983AA83BB83DF91CF911F910F91FF9015
:1005B000EF90DF90BF90AF909F908F907F906F9063
:1005C0005F904F9008950F931F93CF93DF938C010B
:1005D000EAE3F2E48491EF012196882321F00F945D
:1005E0009602FE01F7CFB8018BEF92E20E94C5910F
:1005F00082E20F9496028AE00F94960281E0DF91E6
:10060000CF911F910F91089580910D0481111AC00F
:100610006091000270910102072E000C880B990B6B
:100620000F942C179B01AC0160919E0470919F0464
:100630008091A0049091A1040F942617881F882709
:10064000881F089580E00895CF93DF9389E493E1B4
:1006500018D08FEE91E1892B41F480ED91E111D01A
:100660008FEA91E1DF91CF910CC0C0E0D0E0CE01E4
:100670008A5F9C4E06D06F97CA3C8EEFD807B9F7B9
:10068000ECCF22EB33E0FC013183208304960C9401
:100690000B45149A0895179AEDE8F4E01082169A23
:1006A0001182159A1282F5CF8C01E9E7F8E1849165
:1006B000EF012196882321F00F949602FE01F7CFD7
:1006C000EBEDF2E28491EF012196882321F00F9463
:1006D0009602FE01F7CF0E949052DDDF0E947C4916
:1006E00061E0C8010E94F9450E942A7A0E942FB356
:1006F00084E00E94869080911314869586951092CE
:10070000491480934A140E9420B380911314869553
:100710008695880F1092491480934A148CEC92E2CB
:100720000E94CB908091131486958695982F990FEF
:10073000890F1092491480934A148FEB92E20E9421
:10074000CB900E9427B18111D3CF2FEF8BE49DE195
:10075000215080409040E1F700C00000F8942FEF56
:1007600084E39CE0215080409040E1F700C000000D
:100770000E949052A895FECFCF92DF92EF92FF9207
:100780000F931F93CF93DF93C82F0E94274680912A
:100790009904882391F00E9407D00091950410914C
:1007A00096042091970430919804DC01CB01801BC2
:1007B000910BA20BB30BB7FF34C18091680A85304F
:1007C00010F40E94E2560E9407D0C0908904D09095
:1007D0008A04E0908B04F0908C04C114D104E104ED
:1007E000F10469F10091AB041091AC042091AD04C7
:1007F0003091AE040C0D1D1D2E1D3F1D6B017C01A3
:10080000C01AD10AE20AF30AF7FC19C0E9E7F8E1D5
:100810008491EF012196882321F00F949602FE0126
:10082000F7CF609104047091050485E892E20E947C
:10083000C5918AE00F9496028CE792E235DF209111
:10084000A704211128C0C0900202D0900302E090BA
:100850000402F0900502C114D104E104F104D9F0BE
:100860000091AB041091AC042091AD043091AE0422
:100870000C0D1D1D2E1D3F1DDC01CB01801B910B9E
:10088000A20BB30BB7FD07C0C11105C00E941045F4
:10089000882309F4E5C00E9407D000914608109112
:1008A000470820914808309149086B017C01C01A23
:1008B000D10AE20AF30AF7FC3AC08B019C010C53FF
:1008C000164F2F4F3F4F0093460810934708209331
:1008D000480830934908079BCEC0069BCCC0059BB7
:1008E000CAC0209101052111C6C0049BC4C000915B
:1008F00042081091430820914408309145080115A1
:1009000011052105310509F4BFC0DC01CB01801BB5
:10091000910BA20BB30B80569A4EA109B109B7FFF8
:10092000B3C0749A6FEF70E082E00E9408CF0E941B
:100930001045811105C0D091A304C091A5041AC02F
:10094000E091FD108FE48E9FF0011124E751F44FE8
:10095000D081E091FD108E9FF0011124E551F44FFC
:10096000C0818091FD109091FC10891719F08F5F64
:100970008F70F9CFDD2329F10E9407D000914A083A
:1009800010914B0820914C0830914D08DC01CB01AF
:10099000011511052105310569F48C599F4FAF4FA1
:1009A000BF4F80934A0890934B08A0934C08B09394
:1009B0004D08B0C0801B910BA20BB30BB7FFABC0AF
:1009C000A9C010924A0810924B0810924C0810923D
:1009D0004D08CC2309F478C00E9407D000914E083E
:1009E00010914F082091500830915108DC01CB0143
:1009F000011511052105310569F48C599F4FAF4F41
:100A0000BF4F80934E0890934F08A0935008B09327
:100A100051083DC0801B910BA20BB30BB7FF38C030
:100A200036C00E9407D06B017C012091990430E010
:100A3000A8EEB3E00F944F1BDC01CB018C0D9D1D84
:100A4000AE1DBF1D8093950490939604A0939704C8
:100A5000B09398040E94B14F8AE00F949602ADCEF5
:100A6000179A10928D04169A10928E04159A10926D
:100A70008F040FDE10CF6093420870934308809379
:100A800044089093450833CF749860E04CCFCFEF83
:100A9000DD23D1F129EBD29FC00111246FEF70E06B
:100AA0000F943B1E6A5B7F4F88E00E9408CFCC23E7
:100AB000C1F029EBC29FC00111246FEF70E00F94C9
:100AC0003B1E6A5B7F4F0FC010924E0810924F087A
:100AD000109250081092510860E070E088E00E9487
:100AE00008CF60E070E086E00E9408CF0E947E6040
:100AF0008EEF90E1DF91CF911F910F91FF90EF90DA
:100B0000DF90CF900C94D28F60E070E088E00E947C
:100B100008CFCFCFDFEFC1115FCF10924E081092F8
:100B20004F081092500810925108B4CFCF93DF9322
:100B300080E00E9408A7C9E8D4E1688379838A83AA
:100B40009B8381E00E9408A76C837D838E839F83B3
:100B500082E00E9408A7688779878A879B87DF9150
:100B6000CF910895CF92DF92EF92FF92CF93DF93D0
:100B700020911E02222309F443C0EC01C09012020E
:100B8000D0901302E0901402F0901502A701960194
:100B9000688179818A819B810F94851D181624F4C0
:100BA000C882D982EA82FB82C0901602D0901702D6
:100BB000E0901802F0901902A70196016C817D81E6
:100BC0008E819F810F94851D181624F4CC82DD82BE
:100BD000EE82FF82C0901A02D0901B02E0901C02AD
:100BE000F0901D02A7019601688579858A859B850D
:100BF0000F94851D181624F4C886D986EA86FB86CC
:100C0000DF91CF91FF90EF90DF90CF900895CF9339
:100C1000DF930E944A91E091670AF0E0EA59F74FAA
:100C20008081882309F45EC0E9E7F2E28491EF0154
:100C30002196882321F00F949602FE01F7CFC091F0
:100C4000670A80E6C89FE0011124C957D74F888101
:100C50008E3419F0E6E7F2E210C080E20F949602BB
:100C600089910F949602899190ED980F9A30C8F36C
:100C70008D32B9F38B32A9F3EDCF8491EF01219638
:100C8000882321F00F949602FE01F7CF8091FC108B
:100C90009091FD10891B8F706FE070E0681B7109E7
:100CA000072E000C880B990B0E94EAA5E3E7F2E2FD
:100CB0008491EF012196882321F00F949602FE0182
:100CC000F7CF8091680A65E070E0681B7109072E14
:100CD000000C880B990B0E94EAA58AE0DF91CF9166
:100CE0000D949602DF91CF910895CF93DF938FB744
:100CF000F89490916A15909369158FBFEAE6F2E235
:100D00008491EF012196882321F00F949602FE0131
:100D1000F7CF8091DD059091DE05A091DF05B091C0
:100D2000E005BC01CD016F5F7F4F8F4F9F4F0E9449
:100D3000EAA58AE00F949602DF91CF9168CFEF92F7
:100D4000FF920F931F93CF93DF93C091670A80E6C2
:100D5000C89FE0011124C957D74F8091AF0480FF8D
:100D600019C0EAE3F2E484918F010F5F1F4F8111F4
:100D700002C08E0104C00F949602F801F4CFD8018E
:100D80008D918D01882319F00F949602F8CF8AE097
:100D90000F9496021092AA041092A9048FE38093F4
:100DA000B8041092B7041092B60410923E08109244
:100DB0003F081092400810924108FE018881219658
:100DC0008032D9F38E34B1F4818190ED980F9A304E
:100DD00020F08D3211F08B3269F43296DF013196BA
:100DE0002C9120532A30D0F3CD01FC0101962081B3
:100DF0002032D9F3F0930504E09304048F010F5FD0
:100E00001F4FC0816AE270E0C8010F94921E0097E4
:100E100031F0FC01319780818032E1F31182CD34D1
:100E200029F0C43519F0C73409F0E5C0F801808114
:100E30000F5F1F4F8032D1F380538A3008F0DBC040
:100E4000C093B8041092B7041092B6046AE080917F
:100E5000B6049091B704689FA001699F500D1124BA
:100E60005093B7044093B6043196DF0111978C91EB
:100E7000282F30E020533109240F351F3093B70459
:100E80002093B604808180538A3008F3DF013196C5
:100E90008C918032D9F3CD34B9F42E31310579F00B
:100EA0003CF42731310559F02C31310569F407C084
:100EB0002537310521F0203AE3E03E0729F4B093CD
:100EC000AA04A093A90497C01092AA041092A9049E
:100ED000D091040461E070E0CD0101964C9144236F
:100EE00009F489C0413299F4CD3489F420323105B6
:100EF00071F49093AA048093A90463E270E00F94C4
:100F0000921E009709F477C0DC011C9274C0415412
:100F10004A3108F043C0DC01FD015D915032E1F33C
:100F2000CF01A0EDA50FAA30C8F05E3229F451819F
:100F300050535A3098F067C05D3219F05B3209F0B7
:100F400062C05181A0EDA50FAA3048F05E3209F0D1
:100F50005AC0528150535A3010F055C0FC01042F32
:100F600010E0D80153E0B595A7955A95E1F7A25C3A
:100F7000B74F47707B0102C0EE0CFF1C4A95E2F7A9
:100F8000A7015C91452B4C93309711F0ED1B01C0EC
:100F9000E0E0D801AC5DB74FEC930AC04091A904E2
:100FA0005091AA04452B21F4B093AA04A093A9045C
:100FB000DC014C9141544A3110F4DC018DCFFC012D
:100FC0008E2FAF2F9191911103C0482F5A2F0BC034
:100FD00040ED490F4A30A0F343ED490F423080F312
:100FE0009B3271F3F2CFCA014F5F5F4FDC01EC918E
:100FF000E032C9F3E2CFDF91CF911F910F91FF90C3
:10100000EF900C943528A091A904B091AA04AB2BC1
:1010100029F43197F093AA04E093A904E0E0F0E00A
:101020009ECF81E080930B021092B31083E50E9463
:10103000FF44882319F00E94AB5C03C083E50E9443
:10104000D044811101C051CE0895CF93DF93E9E7D9
:10105000F8E18491EF012196882321F00F94960204
:10106000FE01F7CFEBE5F2E28491EF0121968823B0
:1010700021F00F949602FE01F7CFDF91CF910895F2
:101080000F931F93CF9383E50E94FF44882309F4B5
:1010900047C00E948844813039F0823009F040C056
:1010A00005E113E0C0E021C005E113E0C0E0F80174
:1010B00081918F010E94FF44882339F00E94884467
:1010C0004FEF682F8C2F0E9406A6CF5FC43079F7B0
:1010D00082E40E94FF44882319F10E9488444FEF64
:1010E000682F1BC0CF5FC43079F0F80181918F0168
:1010F0000E94FF448823B1F30E948844482F6FEF79
:101100008C2F0E9406A6EECF82E40E94FF44882323
:1011100039F00E948844482F6FEF84E00E9406A6B1
:10112000CF911F910F910C94A7E7CF93DF931F925C
:101130001F92CDB7DEB7789484B5826084BD84B544
:10114000816084BD85B5826085BD85B5816085BDC2
:1011500080916E00816080936E001092810080917A
:101160008100826080938100809181008160809302
:101170008100809180008160809380008091B10027
:1011800084608093B1008091B00081608093B00052
:1011900080919100826080939100809191008160A4
:1011A0008093910080919000816080939000809165
:1011B000A10082608093A1008091A1008160809352
:1011C000A1008091A00081608093A0008091210106
:1011D00082608093210180912101816080932101AF
:1011E0008091200181608093200180917A00846049
:1011F00080937A0080917A00826080937A00809157
:101200007A00816080937A0080917A008068809370
:101210007A001092C10082E08093C0001092C50055
:1012200087E08093C4008091C10080618093C100F9
:101230008091C10088608093C1008091C100806866
:101240008093C1008091C1008F7D8093C100109276
:101250005E08E0EDF4E284918F010F5F1F4F882359
:1012600021F00F949602F801F6CFEAE3F2E48491BC
:101270008F010F5F1F4F882321F00F949602F80112
:10128000F6CF14B710FF0DC0E7ECF4E284917F01B4
:101290009FEFE91AF90A882321F00F949602F701CB
:1012A000F5CF11FF0DC0E6EBF4E284917F019FEFD3
:1012B000E91AF90A882321F00F949602F701F5CF75
:1012C00012FF0DC0E4EAF4E284917F019FEFE91A76
:1012D000F90A882321F00F949602F701F5CF13FF46
:1012E0000DC0E3E9F4E284917F019FEFE91AF90A66
:1012F000882321F00F949602F701F5CF15FF0CC05B
:10130000E2E8F4E284918F010F5F1F4F882321F000
:101310000F949602F801F6CF14BEEBE7F4E2849145
:101320008F010F5F1F4F882321F00F949602F80161
:10133000F6CF80E20F949602E4E7F4E284918F0105
:101340000F5F1F4F882321F00F949602F801F6CF0C
:101350008AE00F949602EAE3F2E484918F010F5F32
:101360001F4F882321F00F949602F801F6CFE4E690
:10137000F4E284918F010F5F1F4F882321F00F94B7
:101380009602F801F6CFE0E5F4E284918F010F5F59
:101390001F4F882321F00F949602F801F6CFE7E162
:1013A000F4E284918F010F5F1F4F882321F00F9487
:1013B0009602F801F6CFEAE3F2E484918F010F5F21
:1013C0001F4F882321F00F949602F801F6CFE0E03A
:1013D000F4E284918F010F5F1F4F882321F00F9457
:1013E0009602F801F6CFEAE3F2E484918F010F5FF1
:1013F0001F4F882321F00F949602F801F6CF8091B9
:10140000921590919315BE016F5F7F4F009719F071
:10141000681B790B02C06859754181EF93E29CD734
:1014200060EF74E08AED93E297D78AE00F9496021A
:1014300081E08093660880936708809368088093B2
:10144000690880936A080E9477E88CE0ECE2F4E097
:10145000AAEAB4E101900D928A95E1F70E946459DD
:10146000809101018064809301018091010180617C
:1014700080930101809101018860809301016D9A40
:101480008091010180628093010188E00E944AF509
:101490008091010188608093010186E00E944AF5F5
:1014A0006C9A82E00E944AF587ED80937A00109250
:1014B0007E0010927D0080917E00816080937E008E
:1014C00080917E00846080937E0080E888BD80915A
:1014D0006E00846080936E006AEF70E080E090E0C0
:1014E0000E94CFCF85E090E09093640880936308DA
:1014F00060E080912102909122020E94094F20E039
:1015000030E040EA50E40F94261787FF0AC080912C
:10151000210290912202409790932202809321020F
:10152000E7CF81E391E0909324028093230260E06F
:1015300080916108909162080E94094F20E030E894
:1015400048E953E40F94851D181654F480916108FE
:101550009091620840969093620880936108E7CF6B
:1015600080911F02909120020E94545F20E030E0A1
:1015700040EA50E40F94261787FF0AC080911F02AB
:101580009091200240979093200280931F02E8CF11
:1015900080915F08909160080E94545F20E030E0E5
:1015A00046E153E40F94851D181654F480915F08AA
:1015B0009091600840969093600880935F08E8CF10
:1015C00098E288E10FB6F894A895809360000FBE6A
:1015D000909360001FB7F89480916508811124C032
:1015E000E3EFF2E48491E9E3F3E49491E82FF0E08F
:1015F000EE0FFF1FEC55FD4BA591B491EC91E92343
:1016000021F461E085E30E94D9CE85E30E9408B110
:101610008CB580618CBD8CB580648CBD84E30E94E8
:1016200008B183E30E9408B1809165088F5F8093C1
:1016300065081FBF579AB3E4EB2EB3E0FB2E10E012
:10164000F70161917F0170E0812F0E94BFA61F5FAB
:101650001530B1F7999A989A809107018068809324
:1016600007019A9A80910701806480930701809115
:101670000701806280930701809107018860809351
:101680000701809107018061809307018091070124
:101690008260809307018091070184608093070135
:1016A000A8E4EA2EA3E0FA2E10E0F70161917F0191
:1016B000812F0E945FE81F5F1530B9F780910A0102
:1016C000826080930A0180910A01816080930A01FF
:1016D00080910A01846080930A0180910A018064EC
:1016E00080930A0180910A01806880930A010F9A11
:1016F000179A0E9A169A0D9A159A0C9A149A0B9A92
:10170000139A26982E9A25982D9A24982C9A0A98FE
:10171000129A0998119A3F98479A0898109A389AFD
:101720004098179A10928D04399A4198169A1092FF
:101730008E043A9A4298159A10928F043B9A4398D5
:10174000149A3C9A4498809180008C7F809380000A
:1017500080918100877E88608093810080918000E5
:101760008F738093800080918100887F8260809356
:10177000810080E090E4909389008093880010922B
:1017800085001092840080916F00826080936F00CA
:1017900081E080934D1478940E9434A71092B50490
:1017A0006C9A0E947C496CD42091121430E079012B
:1017B000F8E3EF1AF108F7FE04C0790187E3E81AAD
:1017C000F108F594E7942E51310936952795F22EBC
:1017D0000E942FB305E513E223E147E06CE08E2D74
:1017E0000E9461B184E092D40091121410E002577B
:1017F00011091695079560911314625149E253E05F
:101800008F2D0E94E1B16091131466504FE253E0B6
:10181000802F0E94E1B10E9427B18111DBCF64ECDF
:1018200079E080E090E00E9409E630E6832E4DE00A
:10183000742E5EEEC52E54E2D52E60E0A62E60E03A
:10184000B62E2AE0922E8091680A853010F40E940C
:10185000E256809106148823F1F00E9407D000918F
:101860000214109103142091041430910514DC012A
:10187000CB01801B910BA20BB30BB7FD0CC01092D8
:10188000061480915C11811133C10E94C371809153
:101890005C1181112DC18091680A882309F496C0DA
:1018A00080915911882309F47FC00091670A809EB6
:1018B000800111240957174F65E375E2C8010F94A1
:1018C000A516892BF1F08DE493E10F94AC048DE41F
:1018D00093E10E94064B10925A1110925911E2E2C4
:1018E000F5E284918F010F5F1F4F882341F00F9421
:1018F0009602F801F6CF80915A11811155C087D90F
:1019000054C0F80101900020E9F731977F01E01AF7
:10191000F10A10924D136EE470E0C8010F94921E0C
:101920002C01009729F4F7013197E00FF11F0EC049
:1019300060E270E00F94921E8C010F5F1F4F6AE20D
:1019400070E0C2010F94921EFC0131977182928265
:101950001382F80101900020E9F73197AF01401B95
:10196000510BB8018DE493E10F94820580914D13E2
:10197000882309F4C0CFE9E7F8E184918F010F5F74
:101980001F4F882321F00F949602F801F6CFE7ED60
:10199000F4E284918F010F5F1F4F882309F4ABCFCE
:1019A0000F949602F801F5CFCAD98091680A88236E
:1019B00069F081508093680A8091670A8F5F853053
:1019C00018F48093670A02C01092670A80919514F8
:1019D000882309F483C0EAE3F2E484918F010F5F66
:1019E0001F4F882321F00F949602F801F6CFE3E110
:1019F000F5E284918F010F5F1F4F882321F00F9430
:101A00009602F801F6CF8091951480FD74C0809104
:101A1000951484FD70C090E2F92E8091951481FD9B
:101A200086C08091951485FD82C000E28091951456
:101A300082FD98C08091951486FD94C010E280913B
:101A4000951483FF1BC06091830870918408809176
:101A50008508909186080F942C1720917308309177
:101A6000740840917508509176080F948B17AB015C
:101A7000BC0183E095E253D490E501C090E28AE096
:101A80009A830F9496021F929A819F931F921F939D
:101A90001F920F931F92FF92DF92CF921F920E948C
:101AA00005B3109295140FB6F894DEBF0FBECDBFEC
:101AB00080910B04882391F010925B118DE493E1E7
:101AC0000F94AC048DE493E10E94064B10925A11DE
:101AD000109259110E9479BF0E94905280E00E949A
:101AE000BC83A114B10409F4AECE0E940000A9CEBB
:101AF0000E941271D0CE60917B0870917C08809119
:101B00007D0890917E080F942C1720916B083091DE
:101B10006C0840916D0850916E080F948B17AB01C3
:101B2000BC018FE095E2FBD388E5F82E76CF60917B
:101B30007F087091800880918108909182080F94AD
:101B40002C1720916F0830917008409171085091C6
:101B500072080F948B17AB01BC018BE095E2DFD3C9
:101B600009E564CF609183087091840880918508AD
:101B7000909186080F942C17209173083091740867
:101B800040917508509176080F948B17AB01BC01FA
:101B900087E095E2C4D31AE552CF2FB7F89490911D
:101BA00005019B7F909305012FBF87FD95C0A398EA
:101BB0002FB7F894909105019460909305012FBF81
:101BC000880F2FB7F894909105019B7F90930501A2
:101BD0002FBF87FD8DC0A3982FB7F8949091050172
:101BE0009460909305012FBF880F2FB7F8949091C0
:101BF00005019B7F909305012FBF87FD77C0A398B8
:101C00002FB7F894909105019460909305012FBF30
